:100000000C94F4220C9423230C9423230C94232388
:100010000C9423230C9423230C9423230C94232348
:100020000C9423230C9423230C9423230C94232338
:100030000C9423230C942D490C9423230C942323F8
:100040000C9423230C9423230C9423230C94232318
:100050000C9423230C9423230C9423230C94232308
:100060000C9423230C94E2D30C9423230C940ED4ED
:100070000C9423230C94629B0C9423230C94232331
:100080000C9423230C9423230C9423230C942323D8
:100090000C9423230C9423230C9423230C942323C8
:1000A0000C9423230C9423230C9423230C942323B8
:1000B0000C9423230C9423230C9423230C94F645B3
:1000C0000C9423230C9423230C9423230C94232398
:1000D0000C9423230C9423230C9423230C94232388
:1000E0000C942323353E5D3E623E3F3E673EB43E68
:1000F000B43E3F3E853EB43E8A3E923E973E9C3E95
:10010000713E763E7B3E3F3E803EB43E3A3E6C3E84
:10011000A13EA63EAA3EB43EB43EAE3E50726570CD
:100120006172696E6720666F7220736C6565703AE4
:1001300049276D20636F6D706C6574696E6720610F
:100140006E792020717565756564206D6F766573B5
:100150002E20202020202020004368616E67696ED9
:10016000672046696C616D656E743A202049276D81
:1001700020636F6D706C6574696E6720616E7920A5
:1001800020717565756564206D6F7665732E20200E
:10019000202020202000494E56414C494420544FF5
:1001A0004F4C3A2020202020202049207265636592
:1001B000697665642061204C656674202020546F48
:1001C0006F6C20636F6D6D616E642C20627574209E
:1001D00049206F6E6C792068617665206F6E6520AE
:1001E000546F6F6C2E2000494E56414C49442043B9
:1001F0004F4D4D414E443A202020204920726563E6
:100200006569766564206120636F6D6D616E6466FB
:100210006F7220612068656174656420706C617420
:10022000652C20627574204920646F6E27742068E5
:10023000617665206F6E65004920736177206120CB
:10024000676C6974636820696E206D79534420631C
:100250006172642E20496620746869732069732076
:10026000746865206669727374206572726F722C8F
:100270002074727974686973206D6F64656C206195
:100280006761696E2E20202000492074696D6564C5
:10029000206F7574207768696C6520202061747404
:1002A000656D7074696E6720746F20686561742075
:1002B000206D792065787472756465722E20202017
:1002C000202020202000492074696D6564206F750E
:1002D00074207768696C65202020617474656D7086
:1002E00074696E6720746F206865617420206D7971
:1002F00020706C6174666F726D2E2020202020208B
:10030000202000507265706172696E6720666F729E
:1003100020736C6565703A49276D20636F6F6C6957
:100320006E67206D7920202020202068656174652B
:10033000727320616E6420676F696E6720746F6DE1
:1003400079207761697420706F736974696F6E2E9C
:10035000202020004368616E67696E672046696CE3
:10036000616D656E743A202049276D20676F696E54
:100370006720746F206D792077616974706F73697D
:1003800074696F6E2E202020202020202020202025
:10039000004D7920686561746572732074696D65BC
:1003A00064206F75744920616D206E6F7720696ECF
:1003B00020536C65657020202028436F6C642050AA
:1003C00061757365292E20202020202020202020E8
:1003D000202020202020202020202020202020201D
:1003E000200052657374617274696E672074686569
:1003F000204275696C640054686973206973206ECB
:100400006F7420746865207833672076657273692D
:100410006F6E204920776F726B206265737420774E
:100420006974682E20466F722068656C7020736551
:10043000653A206D616B6572626F742E636F6D2F0C
:1004400068656C70202020004920616D2061205279
:1004500065706C696361746F722E202054686973D3
:10046000206275696C6420697320666F7220202099
:10047000616E6F7468657220626F742E20536565BB
:100480003A2020206D616B6572626F742E636F6D10
:100490002F68656C702020200054686520526570BC
:1004A0006C6963617430720049276D2043616E632B
:1004B000656C6C696E672E2020202020506C656171
:1004C000736520576169742E202020202020202071
:1004D00000200048656174657273207368757464E8
:1004E0006F776E2020202064756520746F20696E00
:1004F00061637469766974792020200048656174AD
:10050000696E67204661696C757265202331212010
:10051000536F6674776172652054656D70204C6905
:100520006D697420526561636865642120506C6553
:10053000617365202020202053687574646F776E86
:10054000206F722052657374617274200048656177
:1005500074696E67204661696C757265202332216B
:10056000204D7920657874727564657273206172AC
:1005700065206E6F7468656174696E672070726F54
:100580007065726C792E202020436865636B206D46
:100590007920636F6E6E656374696F6E7300486572
:1005A0006174696E67204661696C757265202333DA
:1005B00021204D79206578747275646572732061AD
:1005C0007265202020206C6F73696E672074656DE2
:1005D00070657261747572652E20436865636B2067
:1005E0006D7920636F6E6E656374696F6E7300481A
:1005F000656174696E67204661696C757265202358
:1006000035212049276D2072656164696E67206F0E
:100610007574206F66202072616E67652074656D49
:100620007065726174757265732E20436865636BC3
:10063000206D7920636F6E6E656374696F6E7300F1
:1006400048656174696E67204661696C75726520E2
:10065000233421204D792074656D70657261747545
:100660007265207265616473617265206661696C90
:10067000696E672120506C6561736520436865630E
:100680006B206D7920636F6E6E656374696F6E7336
:10069000009302690000006900EE01690000006932
:1006A000002601B80100000000200655000000559A
:1006B000002D085500000055004D0A55000000555A
:1006C00000400CAB000000AB002D095500000055A8
:1006D000002D085500000055004D0AAB00000055E4
:1006E0000000000001C00D5500000055002D085607
:1006F0000100000000C00D20015311BC005B12B1CD
:100700000100000000C00DC80000001400C00DC8AA
:100710000000001400910E9001000014005A109087
:100720000100001400C00D200300000000C805C82F
:100730000000001400C805C80000001400C805C867
:100740000000001400DD04B004000014007505C8AA
:1007500000000014007505C800000014007505C8ED
:1007600000000014009704B00400000000B8075512
:100770000000005500B909AB000000AB007D065534
:100780000000005500C805550000005500B807AB33
:10079000000000AB00C805550000005500DD045501
:1007A0000000005500C805550000005500B8075569
:1007B00000000055007D065601000000003F035573
:1007C0000000005500FA0C5500000055003F03558D
:1007D0000000005500B9095500000055003F0355C1
:1007E00000000055002D095500000055003F03553D
:1007F0000000005500EA0A5500000055003F03556F
:100800000000005500B909AB00000000005344206F
:10081000436172642052656D6F76656420202020EC
:100820000024F404D9201BC40C5C0E9804C4095F96
:100830000265077101F405F900FB04B30048048761
:1008400000C10369005803550003034500BE023A86
:10085000008402310053022A0029022500040220EC
:1008600000E4011C00C8011900AF01170098011431
:100870000084011300710110006101100051010E8C
:100880000043010D0036010B002B010B0020010B72
:1008900000150109000C01090003010800FB000814
:1008A00000F3000800EB000700E4000600DE00068D
:1008B00000D8000600D2000600CC000500C70005E5
:1008C00000C2000500BD000400B9000400B500042A
:1008D00000B1000400AD000400A9000400A500035D
:1008E00000A20003009F0004009B00030098000387
:1008F000009500020093000300900003008D0002A9
:10090000008B0003008800020086000200840003C0
:1009100000810002007F0002007D0002007B0002D7
:1009200000790002007700010076000200740002E6
:100930000072000100710002006F0002006D0001F2
:10094000006C0002006A00010069000200670001FB
:100950000066000100650001006400020062000101
:100960000061000100600001005F0002005D000105
:10097000005C0001005B0001005A00010059000109
:100980000058000100570001005600010055000109
:100990000054000100530000005300010052000108
:1009A0000051000100500001004F0001004E000006
:1009B000004E0001004D0001004C0001004B000002
:1009C000004B0001004A00010049000100480000FE
:1009D00000480001004700010046000000460001F9
:1009E00000450000004500010044000100430000F4
:1009F00000430001004200000042000100410000ED
:100A00000041000100400001003F0000003F0001E4
:100A1000003E0000003E0001003D0000003D0001DE
:100A2000003C0000003C0000003C0001003B0000D6
:100A3000003B0001003A0000003A000100390000CC
:100A400000390001003800000038000000380001C3
:100A500000370000003700010036000000360000BB
:100A600000360001003500000035000000350001AF
:100A700000340000003400000034000100330000A6
:100A8000003300000033000100320000003200009B
:100A9000003200010031000000310000003100018F
:100AA000003000000030000000300001002F000086
:100AB000002F0000002F0000002F0001002E00007A
:100AC000002E0000002E0001002D0000002D00006F
:100AD000002D0000002D0001002C0000002C000063
:100AE000002C0000002C0001002B0000002B000057
:100AF000002B0000002B0001002A0000002A00004B
:100B0000002A0000002A000100290000002900003E
:100B10000029000000290000002900010028000031
:100B20000028000000280000002800000028000124
:100B30000027000000270000002700000027000019
:100B4000002700010026000000260000002600000B
:100B500000260000002600010025000000250000FE
:100B600000250000002500000025000000250001F0
:100B700000240000002400000024000000240000E5
:100B800000240001002300000023000000230000D7
:100B900000230000002300000023000000230001C8
:100BA00000220000002200000022000000220000BD
:100BB00000220000002200010021000000210000AE
:100BC00000210000002100000021000000210000A1
:100BD0000021000100200000002000000020000093
:100BE0000020000000200000002000000020000085
:100BF00000200001001F0000001F0000001F000077
:100C0000001F0000001F0000001F0000001F000167
:100C1000001E0000001E0000001E0000001E00005C
:100C20000024F4D43050C38E20C2A24017828B70AF
:100C300011127A910D816CD90AA861E108C7586632
:100C400007615143061E4B5D05C145A7041A4111BA
:100C500004093D9803713931034036DB0265339155
:100C600002D4305402802E1D02632CEE01752AC579
:100C700001B028A001102781018F2564012B244B8E
:100C800001E0223401AC211F018D200D01801FFCE9
:100C900000841EED00971DDF00B81CD200E61BC6C5
:100CA00000201BBC00641AB200B219A8000A19A0E7
:100CB000006A189900D117910040178B00B516846F
:100CC0000031167E00B31579003A157300C7146F12
:100CD0000058146A00EE1366008813630025135E43
:100CE00000C7125B006C12570015125400C111515D
:100CF0000070114F0021114B00D61049008D104794
:100D0000004610440002104200C00F4000800F3E19
:100D100000420F3C00060F3B00CB0E3800930E370D
:100D2000005C0E3500270E3400F30D3200C10D318A
:100D300000900D3000600D2E00320D2D00050D2CA1
:100D400000D90C2B00AE0C2900850C29005C0C2767
:100D500000350C27000E0C2600E80B2400C40B24E1
:100D600000A00B23007D0B23005A0B2100390B211F
:100D700000180B2000F80A1F00D90A1E00BB0A1E2B
:100D8000009D0A1D00800A1D00630A1C00470A1B03
:100D9000002C0A1B00110A1A00F7091A00DD0919B4
:100DA00000C4091900AB091900920917007B091842
:100DB00000630917004C09160036091600200916B1
:100DC000000A091500F5081500E0081400CC081405
:100DD00000B8081400A4081400900813007D08123D
:100DE000006B08130058081200460812003408115E
:100DF00000230811001208110001081100F007106B
:100E000000E0071000D0071000C0071000B0070F67
:100E100000A107100091070E0083070F0074070F51
:100E20000065070E0057070E0049070E003B070D2F
:100E3000002E070E0020070D0013070D0006070DFA
:100E400000F9060C00ED060D00E0060C00D4060CBF
:100E500000C8060C00BC060C00B0060C00A4060B73
:100E60000099060C008D060B0082060B0077060B1E
:100E7000006C060B0061060A0057060B004C060AC0
:100E80000042060A0038060A002E060A0024060A56
:100E9000001A060A001006090007060A00FD0509E7
:100EA00000F4050900EB050900E2050900D9050970
:100EB00000D0050900C7050900BE050900B50508F1
:100EC00000AD050800A50509009C0508009405086B
:100ED000008C050800840508007C050800740508DE
:100EE000006C050700650508005D0507005605084C
:100EF000004E0507004705070040050800380507B4
:100F000000310507002A050700230507001C050618
:100F100000160507000F0507000805060002050773
:100F200000FB040600F5040700EE040600E80406D2
:100F300000E2040700DB040600D5040600CF040627
:100F400000C9040600C3040600BD040600B7040679
:100F500000B1040500AC040600A6040600A00405C8
:100F6000009B04060095040500900406008A040511
:100F70000085040500800406007A04050075040558
:100F800000700405006B040500660405006104059B
:100F9000005C04050057040500520405004D0405DB
:100FA0000048040500430405003E0404003A04051B
:100FB0000035040500300404002C04050027040457
:100FC00000230405001E0404001A0404001604058E
:100FD00000110404000D04040009040500040404C5
:100FE0000000040400FC030400F8030400F40304FC
:100FF00000F0030400EC030400E8030400E403042D
:1010000000E0030400DC030400D8030400D403045C
:1010100000D0030400CC030400C8030300C503038D
:10102000009502000000506C65617365207761696E
:10103000742E2E2E0084036901000014008304889E
:1010400000000014008C000000000000000030F8D8
:10105000FFFF00000000000000008E000000000004
:101060000000000000000000000000000000005729
:10107000290400188304DC0500001400901F891F58
:101080009502000000506C6561736520776169749A
:101090000084036901000014008304880000001428
:1010A000008C000000000000000030F8FFFF00008E
:1010B0000000000000008E000000000000000000A2
:1010C0000000000000000000000000572904001884
:1010D0008304DC05000014008CE5370000941B003D
:1010E000000000000000000000000000009500006B
:1010F000000046696E64207468652034206B6E6F52
:101100006273206F6E2000950100000074686520F6
:10111000626F74746F6E206F662074686520202083
:10112000009501000000706C6174666F726D206143
:101130006E64207469676874656E0095070000002E
:10114000666F7572206F722066697665207475729D
:101150006E732E00950000000049276D20676F69AF
:101160006E6720746F206D6F7665202020009501DA
:10117000000000746865206578747275646572207B
:10118000746F2020202020009501000000766172FD
:10119000696F757320706F736974696F6E73202047
:1011A00020009507000000666F722061646A757305
:1011B000746D656E742E009500000000496E206508
:1011C00061636820706F736974696F6E2C202020D2
:1011D00000950100000077652077696C6C206E65D2
:1011E000656420746F2020202020009501000000FD
:1011F00061646A7573742032206B6E6F6273206154
:101200007420202000950700000074686520736139
:101210006D652074696D652E0095000000004E6FAD
:101220007A7A6C65732061726520617420746865D8
:1012300020200095010000007269676874206865CD
:1012400069676874207768656E202020009501002A
:101250000000796F752063616E206A757374207366
:101260006C6964652061009507000000736865651E
:1012700074206F6620706170657200950000000038
:101280006265747765656E20746865206E6F7A7A22
:101290006C652020009501000000616E6420746878
:1012A0006520706C6174652E202020202020009520
:1012B00001000000477261622061207368656574F7
:1012C000206F66202020202000950700000070611C
:1012D00070657220746F2061737369737420757305
:1012E0002E009502000000506C65617365207761E7
:1012F0006974009502000000506C65617365207789
:10130000616974008EE6370000951B0000D007006D
:101310000000000000000000009AE90300188E00A1
:10132000000000CAE4FFFFD007000000000000003A
:101330000000002A0D3B00188E00000000C9E4FFE9
:10134000FF0000000000000000000000009AE90318
:101350000018950000000041646A75737420746879
:10136000652066726F6E742074776F0095010000BF
:10137000006B6E6F627320756E74696C20706170A3
:1013800065722020200095010000006A75737420AA
:10139000736C69646573206265747765656E20009F
:1013A00095070000006E6F7A7A6C6520616E64208C
:1013B000706C617465009502000000506C6561738B
:1013C000652077616974008E00000000CAE4FFFFA9
:1013D000D007000000000000000000009AE90300B0
:1013E000188E000000007A1A0000D00700000000EC
:1013F00000000000000051812800188E000000004D
:101400007A1A000000000000000000000000000048
:101410009AE9030018950000000041646A7573742E
:1014200020746865206261636B2074776F2000957B
:10143000010000006B6E6F627320756E74696C2022
:1014400070617065722020200095010000006A75AF
:10145000737420736C696465732062657477656565
:101460006E200095070000006E6F7A7A6C6520612F
:101470006E6420706C617465009502000000506C11
:10148000656173652077616974008E000000007AE1
:101490001A0000D007000000000000000000009AC1
:1014A000E90300188EC624000000000000D00700E9
:1014B000000000000000000000A82F2200188EC6C7
:1014C00024000000000000000000000000000000F8
:1014D0000000009AE9030018950000000041646ACA
:1014E00075737420746865207269676874207477F6
:1014F0006F0095010000006B6E6F627320756E7453
:10150000696C2070617065722020200095010000D8
:10151000006A75737420736C696465732062657406
:101520007765656E200095070000006E6F7A7A6C13
:101530006520616E6420706C617465009502000026
:1015400000506C656173652077616974008EC624F4
:10155000000000000000D0070000000000000000B4
:1015600000009AE90300188E3ADBFFFF000000003C
:10157000D007000000000000000000008B7C370056
:10158000188E3ADBFFFF00000000000000000000A2
:101590000000000000009AE9030018950000000018
:1015A00041646A75737420746865206C6566742084
:1015B00074776F200095010000006B6E6F627320DE
:1015C000756E74696C2070617065722020200095C2
:1015D000010000006A75737420736C696465732080
:1015E0006265747765656E200095070000006E6F78
:1015F0007A7A6C6520616E6420706C617465009508
:1016000002000000506C65617365207761697400A9
:101610008E3ADBFFFF00000000D007000000000052
:1016200000000000009AE90300188E00000000008E
:10163000000000D00700000000000000000000458E
:10164000BE1B00188E00000000000000000000001B
:101650000000000000000000009AE9030018950057
:10166000000000436865636B2074686174207061DA
:10167000706572202020200095010000006A7573BB
:101680007420736C69646573206265747765656E38
:10169000200095070000006E6F7A7A6C6520616EFD
:1016A0006420706C61746500891F95020000005011
:1016B0006C6561736520776169740084036901005A
:1016C00000140083048800000014008C0000000057
:1016D0000000000030F8FFFF0000000000000000E4
:1016E0008E0000000000000000000000000000006C
:1016F000000000000057290400188304DC050000E6
:1017000014008CE5370000941B000000000000006E
:1017100000000000000000950000000046696E64B3
:10172000207468652034206B6E6F6273206F6E20AA
:1017300000950100000074686520626F74746F6E1C
:10174000206F66207468652020200095010000004D
:10175000706C6174666F726D20616E64207469676D
:101760006874656E009507000000666F7572206FE3
:10177000722066697665207475726E732E0095000E
:1017800000000049276D20676F696E6720746F2025
:101790006D6F76652020200095010000007468655B
:1017A00020657874727564657220746F2020202023
:1017B00020009501000000766172696F75732070DA
:1017C0006F736974696F6E732020200095070000A5
:1017D00000666F722061646A7573746D656E742E35
:1017E000009500000000496E206561636820706FFD
:1017F000736974696F6E2C20202000950100000031
:1018000077652077696C6C206E65656420746F2045
:101810002020202000950100000061646A75737427
:101820002032206B6E6F627320617420202000953F
:10183000070000007468652073616D652074696D30
:10184000652E0095000000004E6F7A7A6C6573205B
:101850006172652061742074686520200095010024
:10186000000072696768742068656967687420772A
:1018700068656E202020009501000000796F7520BA
:1018800063616E206A75737420736C69646520618E
:101890000095070000007368656574206F6620700E
:1018A000617065720095000000006265747765657F
:1018B0006E20746865206E6F7A7A6C6520200095C2
:1018C00001000000616E642074686520706C6174B2
:1018D000652E202020202020009501000000477266
:1018E00061622061207368656574206F6620202026
:1018F0002020009507000000706170657220746FF1
:10190000206173736973742075732E009502000053
:1019100000506C6561736520776169740095020001
:101920000000506C656173652077616974008EE515
:10193000370000941B0000D00700000000000000EA
:101940000000009AE90300188E11060000CAE4FFA7
:10195000FFD00700000000000000000000DADF37C1
:1019600000188E12060000CAE4FFFF00000000000D
:10197000000000000000009AE90300189500000034
:101980000041646A757374207468652066726F6EB6
:10199000742074776F0095010000006B6E6F6273A6
:1019A00020756E74696C2070617065722020200053
:1019B00095010000006A75737420736C6964657327
:1019C000206265747765656E200095070000006EE3
:1019D0006F7A7A6C6520616E6420706C617465004A
:1019E0009502000000506C65617365207761697431
:1019F000008E11060000C9E4FFFFD00700000000C0
:101A00000000000000009AE90300188E1106000093
:101A10007B1A0000D007000000000000000000005A
:101A200051812800188E110600007A1A000000006B
:101A3000000000000000000000009AE90300189573
:101A40000000000041646A75737420746865206248
:101A500061636B2074776F200095010000006B6E4E
:101A60006F627320756E74696C207061706572208E
:101A700020200095010000006A75737420736C6962
:101A8000646573206265747765656E200095070054
:101A900000006E6F7A7A6C6520616E6420706C61F4
:101AA0007465009502000000506C656173652077D5
:101AB000616974008E120600007A1A0000D00700D7
:101AC0000000000000000000009AE90300188E2AC0
:101AD00027000000000000D0070000000000000008
:101AE000000000CFF91F00188E2A27000000000018
:101AF000000000000000000000000000009AE90360
:101B00000018950000000041646A757374207468C1
:101B1000652072696768742074776F009501000012
:101B2000006B6E6F627320756E74696C20706170EB
:101B300065722020200095010000006A75737420F2
:101B4000736C69646573206265747765656E2000E7
:101B500095070000006E6F7A7A6C6520616E6420D4
:101B6000706C617465009502000000506C656173D3
:101B7000652077616974008E29270000000000004D
:101B8000D007000000000000000000009AE90300F8
:101B9000188EF9E4FFFF00000000D00700000000ED
:101BA00000000000000017F03100188EF9E4FFFF7C
:101BB0000000000000000000000000000000000025
:101BC0009AE9030018950000000041646A75737477
:101BD00020746865206C6566742074776F200095AA
:101BE000010000006B6E6F627320756E74696C206B
:101BF00070617065722020200095010000006A75F8
:101C0000737420736C6964657320626574776565AD
:101C10006E200095070000006E6F7A7A6C65206177
:101C20006E6420706C617465009502000000506C59
:101C3000656173652077616974008EF9E4FFFF00C8
:101C4000000000D007000000000000000000009A23
:101C5000E90300188E1106000000000000D0070004
:101C60000000000000000000000BF81800188E11A2
:101C7000060000000000000000000000000000005E
:101C80000000009AE9030018950000000043686511
:101C9000636B20746861742070617065722020200D
:101CA000200095010000006A75737420736C6964EC
:101CB0006573206265747765656E20009507000086
:101CC000006E6F7A7A6C6520616E6420706C61744E
:101CD0006500891F99000000006E6F7A7A6C654379
:101CE000616C6962726174696F6E009600008600B3
:101CF00084033E01000014008304A60000001400C9
:101D00008C000000000000000030F8FFFF00000021
:101D100000000000008B0000000000000000000038
:101D200000000000000000000000A6000000830486
:101D3000DC0500001400901F8CE5370000941B00A8
:101D4000000000000000000000000000008BD1D661
:101D5000FFFF28E5FFFF60EA000000000000000030
:101D6000000080000000910114910014910414916E
:101D7000031488001F026E008D0064005802880062
:101D80000302E60088010302E600870064005802AF
:101D900087016400580291017F91007F91047F9137
:101DA000037F8B43E6FFFFB8E9FFFF6801000000F7
:101DB00000000000000000800000008B43E6FFFFF1
:101DC000B8E9FFFF68010000E4FFFFFF000000002A
:101DD0000C0300008B43E6FFFFB8E9FFFFF00000B3
:101DE00000D0FFFFFF000000003E0000008B43E634
:101DF000FFFFB8E9FFFFF0000000B3FFFFFF0000A6
:101E00000000850100008B8DD7FFFFB8E9FFFFF0D0
:101E10000000004FFEFFFF000000004A0300008B9F
:101E200043E6FFFF6EEDFFFFF00000007FFEFFFFC7
:101E300000000000C70000008B43E6FFFF6EEDFFCF
:101E4000FFF000000063FEFFFF00000000850100BE
:101E5000008B3BDBFFFF6EEDFFFFF0000000FEFCA0
:101E6000FFFF000000004C0300008B43E6FFFF254E
:101E7000F1FFFFF00000002EFDFFFF00000000CB8F
:101E80000000008B43E6FFFF25F1FFFFF00000009C
:101E900012FDFFFF00000000850100008B3BDBFF0F
:101EA000FF25F1FFFFF0000000ADFBFFFF00000089
:101EB000004C0300008B43E6FFFFDCF4FFFFF00063
:101EC0000000DDFBFFFF00000000CB0000008B43A3
:101ED000E6FFFFDCF4FFFFF0000000C1FBFFFF00A6
:101EE000000000850100008B3BDBFFFFDCF4FFFFFF
:101EF000F00000005CFAFFFF000000004C0300004F
:101F00008B43E6FFFF93F8FFFFF00000008DFAFF20
:101F1000FF00000000CB0000008B43E6FFFF93F8BA
:101F2000FFFFF000000070FAFFFF000000008501D5
:101F300000008B3BDBFFFF93F8FFFFF00000000B7E
:101F4000F9FFFF000000004C0300008B43E6FFFF99
:101F50004AFCFFFFF00000003CF9FFFF000000001A
:101F6000CB0000008B43E6FFFF4AFCFFFFF00000C0
:101F7000001FF9FFFF00000000850100008B3BDB24
:101F8000FFFF4AFCFFFFF0000000BAF7FFFF000070
:101F900000004C0300008B43E6FFFF00000000F050
:101FA000000000EBF7FFFF00000000CB0000008BFB
:101FB00043E6FFFF00000000F0000000CEF7FFFF47
:101FC00000000000850100008B3BDBFFFF000000EC
:101FD00000F000000069F6FFFF000000004C030065
:101FE000008B43E6FFFFB6030000F00000009AF606
:101FF000FFFF00000000CB0000008B43E6FFFFB6B0
:10200000030000F00000007DF6FFFF0000000085E7
:102010000100008B3BDBFFFFB6030000F000000077
:1020200019F5FFFF000000004C0300008B43E6FFA2
:10203000FF6D070000F000000049F5FFFF00000001
:1020400000CB0000008B43E6FFFF6D070000F000AF
:1020500000002CF5FFFF00000000850100008B3B15
:10206000DBFFFF6D070000F0000000C8F3FFFF007A
:102070000000004C0300008B43E6FFFF240B000030
:10208000F0000000F8F3FFFF00000000CB000000AC
:102090008B43E6FFFF240B0000F0000000DBF3FFA2
:1020A000FF00000000850100008B3BDBFFFF240BDD
:1020B0000000F000000077F2FFFF000000004C037A
:1020C00000008B43E6FFFFDB0E0000F0000000A7DE
:1020D000F2FFFF00000000CB0000008B43E6FFFF93
:1020E000DB0E0000F00000008AF2FFFF000000009D
:1020F000850100008B3BDBFFFFDB0E0000F00000E2
:102100000026F1FFFF000000004C0300008B43E6B7
:10211000FFFF92120000F000000056F1FFFF0000E8
:102120000000CB0000008B43E6FFFF92120000F09E
:1021300000000039F1FFFF00000000850100008B66
:102140003BDBFFFF92120000F0000000D5EFFFFF25
:10215000000000004C0300008B43E6FFFF48160020
:1021600000F000000005F0FFFF00000000CB0000C1
:10217000008B43E6FFFF48160000F0000000E8EF88
:10218000FFFF00000000850100008B3BDBFFFF48E4
:10219000160000F000000084EEFFFF000000004C7D
:1021A0000300008BC0F4FFFFA6F8FFFF68010000EA
:1021B000B4EEFFFF00000000FE0000008BC0F4FF43
:1021C000FFA6F8FFFFF000000084EEFFFF00000014
:1021D000009C0000008BC0F4FFFFA6F8FFFFF0009A
:1021E000000067EEFFFF00000000850100008BC0CB
:1021F000F4FFFF5A070000F000000003EDFFFF00AE
:102200000000004A0300008B77F8FFFFA6F8FFFFED
:10221000F000000033EDFFFF00000000C7000000E9
:102220008B77F8FFFFA6F8FFFFF000000016EDFF28
:10223000FF00000000850100008B77F8FFFFAD0371
:102240000000F0000000B2EBFFFF000000004C03B4
:1022500000008B2DFCFFFFA6F8FFFFF0000000E25E
:10226000EBFFFF00000000CB0000008B2DFCFFFF08
:10227000A6F8FFFFF0000000C5EBFFFF0000000024
:10228000850100008B2DFCFFFFAD030000F0000076
:102290000061EAFFFF000000004C0300008BE4FF38
:1022A000FFFFA6F8FFFFF000000091EAFFFF00002B
:1022B0000000CB0000008BE4FFFFFFA6F8FFFFF05B
:1022C00000000074EAFFFF00000000850100008BA1
:1022D000E4FFFFFFAD030000F000000010E9FFFF86
:1022E000000000004C0300008B9A030000A6F8FFDA
:1022F000FFF000000040E9FFFF00000000CB0000FD
:10230000008B9A030000A6F8FFFFF000000023E90D
:10231000FFFF00000000850100008B9A030000AD64
:10232000030000F0000000BFE7FFFF000000004CCA
:102330000300008B51070000A6F8FFFFF00000002B
:10234000EFE7FFFF00000000CB0000008B5107000B
:1023500000A6F8FFFFF0000000D2E7FFFF0000003A
:1023600000850100008B51070000AD030000F00064
:1023700000006EE6FFFF000000004C0300008B0829
:102380000B0000A6F8FFFFF00000009EE6FFFF0034
:10239000000000CB0000008B080B0000A6F8FFFF38
:1023A000F000000081E6FFFF000000008501000052
:1023B0008B080B0000AD030000F00000001DE5FFDE
:1023C000FF000000004C0300008BBF0E0000A6F8C9
:1023D000FFFFF00000004DE5FFFF00000000CB0014
:1023E00000008BBF0E0000A6F8FFFFF000000030D9
:1023F000E5FFFF00000000850100008BBF0E00001C
:10240000AD030000F0000000CCE3FFFF000000007F
:102410004C0300008B75120000A6F8FFFFF00000CF
:1024200000FCE3FFFF00000000CB0000008B7512F2
:102430000000A6F8FFFFF0000000DFE3FFFF000050
:102440000000850100008B75120000AD030000F054
:102450000000007BE2FFFF000000004C0300008B47
:102460002C160000A6F8FFFFF0000000ABE2FFFF13
:1024700000000000CB0000008B2C160000A6F8FF27
:10248000FFF00000008EE2FFFF0000000085010069
:10249000008B2C160000AD030000F00000002AE1C4
:1024A000FFFF000000004C0300008BE3190000A6B2
:1024B000F8FFFFF00000005AE1FFFF00000000CB32
:1024C0000000008BE3190000A6F8FFFFF0000000F9
:1024D0003DE1FFFF00000000850100008BE31900D3
:1024E00000AD030000F0000000D9DFFFFF00000096
:1024F000004C0300008B9A1D0000A6F8FFFFF000BF
:10250000000009E0FFFF00000000CB0000008B9AF4
:102510001D0000A6F8FFFFF0000000ECDFFFFF0049
:10252000000000850100008B9A1D0000AD03000033
:10253000F000000088DEFFFF000000004C030000F8
:102540008B51210000A6F8FFFFF0000000B8DEFF6D
:10255000FF00000000CB0000008B51210000A6F816
:10256000FFFFF00000009BDEFFFF00000000850180
:1025700000008B51210000AD030000F00000003787
:10258000DDFFFF000000004C0300008B5121000024
:10259000AD030000F000000067DDFFFF0000000059
:1025A0000C0300008C51210000AD030000F000007E
:1025B000000000000000000000860189188B43E63F
:1025C000FFFFF0E9FFFF68010000000000000000CD
:1025D0000000D20000008B43E6FFFFF0E9FFFF6838
:1025E00001000000000000E4FFFFFF0C0300008B6F
:1025F00043E6FFFFF0E9FFFFF000000000000000ED
:10260000D0FFFFFF3E0000008B43E6FFFFF0E9FF35
:10261000FFF000000000000000B3FFFFFF85010095
:10262000008B4BF1FFFFF0E9FFFFF000000000001E
:1026300000004FFEFFFF4C0300008B43E6FFFF9EB0
:10264000EDFFFFF0000000000000007FFEFFFFCB69
:102650000000008B43E6FFFF9EEDFFFFF00000004F
:102660000000000063FEFFFF850100008B4BF1FFBF
:10267000FF9EEDFFFFF000000000000000FEFCFFE9
:10268000FF4C0300008B43E6FFFF4BF1FFFFF00020
:102690000000000000002EFDFFFFCB0000008B4378
:1026A000E6FFFF4BF1FFFFF000000000000000120A
:1026B000FDFFFF850100008B4BF1FFFF4BF1FFFF9A
:1026C000F000000000000000ADFBFFFF4C03000025
:1026D0008B43E6FFFFF8F4FFFFF00000000000006E
:1026E00000DDFBFFFFCB0000008B43E6FFFFF8F4AB
:1026F000FFFFF000000000000000C1FBFFFF8501AC
:1027000000008B4BF1FFFFF8F4FFFFF0000000002A
:102710000000005CFAFFFF4C0300008B43E6FFFF64
:10272000A6F8FFFFF0000000000000008DFAFFFF98
:10273000CB0000008B43E6FFFFA6F8FFFFF0000090
:10274000000000000070FAFFFF850100008B4BF1D4
:10275000FFFFA6F8FFFFF0000000000000000BF9EB
:10276000FFFF4C0300008B43E6FFFF53FCFFFFF02D
:10277000000000000000003CF9FFFFCB0000008BD0
:1027800043E6FFFF53FCFFFFF000000000000000E5
:102790001FF9FFFF850100008B4BF1FFFF53FCFF8A
:1027A000FFF000000000000000BAF7FFFF4C03003C
:1027B000008B43E6FFFF00000000F0000000000077
:1027C0000000EBF7FFFFCB0000008B43E6FFFF00AC
:1027D000000000F000000000000000CEF7FFFF85C1
:1027E0000100008B4BF1FFFF00000000F000000033
:1027F0000000000069F6FFFF4C0300008B43E6FF7A
:10280000FFAD030000F0000000000000009AF6FF9A
:10281000FFCB0000008B43E6FFFFAD030000F0009C
:102820000000000000007DF6FFFF850100008B4BDB
:10283000F1FFFFAD030000F00000000000000019F0
:10284000F5FFFF4C0300008B43E6FFFF5A07000033
:10285000F00000000000000049F5FFFFCB00000081
:102860008B43E6FFFF5A070000F000000000000065
:10287000002CF5FFFF850100008B4BF1FFFF5A078D
:102880000000F000000000000000C8F3FFFF4C0350
:1028900000008B43E6FFFF080B0000F00000000083
:1028A000000000F8F3FFFFCB0000008B43E6FFFFC2
:1028B000080B0000F000000000000000DBF3FFFF49
:1028C000850100008B4BF1FFFF080B0000F00000BA
:1028D000000000000077F2FFFF4C0300008B43E68E
:1028E000FFFFB50E0000F000000000000000A7F29E
:1028F000FFFFCB0000008B43E6FFFFB50E0000F0AA
:10290000000000000000008AF2FFFF850100008B3C
:102910004BF1FFFFB50E0000F000000000000000CA
:1029200026F1FFFF4C0300008B43E6FFFF6212001D
:1029300000F00000000000000056F1FFFFCB000097
:10294000008B43E6FFFF62120000F0000000000071
:10295000000039F1FFFF850100008B4BF1FFFF62A2
:10296000120000F000000000000000D5EFFFFF4C57
:102970000300008B43E6FFFF10160000F00000008C
:102980000000000005F0FFFFCB0000008B43E6FFD6
:10299000FF10160000F000000000000000E8EFFF4C
:1029A000FF850100008B4BF1FFFF10160000F000C7
:1029B00000000000000084EEFFFF4C0300008BF8D5
:1029C000F4FFFF9EEDFFFF6801000000000000B46F
:1029D000EEFFFFC10000008BF8F4FFFF9EEDFFFF4C
:1029E000F00000000000000084EEFFFF9C000000EB
:1029F0008BF8F4FFFF9EEDFFFFF0000000000000E9
:102A00000067EEFFFF850100008BF8F4FFFFA6F8DA
:102A1000FFFFF00000000000000003EDFFFF4C038B
:102A200000008BA6F8FFFF9EEDFFFFF00000000006
:102A300000000033EDFFFFCB0000008BA6F8FFFF86
:102A40009EEDFFFFF00000000000000016EDFFFF0C
:102A5000850100008BA6F8FFFFA6F8FFFFF000003D
:102A60000000000000B2EBFFFF4C0300008B53FCA2
:102A7000FFFF9EEDFFFFF000000000000000E2EB12
:102A8000FFFFCB0000008B53FCFFFF9EEDFFFFF02C
:102A900000000000000000C5EBFFFF850100008B77
:102AA00053FCFFFFA6F8FFFFF0000000000000004D
:102AB00061EAFFFF4C0300008B000000009EEDFF69
:102AC000FFF00000000000000091EAFFFFCB0000D3
:102AD000008B000000009EEDFFFFF00000000000F2
:102AE000000074EAFFFF850100008B00000000A6D3
:102AF000F8FFFFF00000000000000010E9FFFF4CAD
:102B00000300008BAD0300009EEDFFFFF00000000E
:102B10000000000040E9FFFFCB0000008BAD030088
:102B2000009EEDFFFFF00000000000000023E9FF21
:102B3000FF850100008BAD030000A6F8FFFFF00049
:102B4000000000000000BFE7FFFF4C0300008B5AAD
:102B50000700009EEDFFFFF000000000000000EF06
:102B6000E7FFFFCB0000008B5A0700009EEDFFFF40
:102B7000F000000000000000D2E7FFFF8501000028
:102B80008B5A070000A6F8FFFFF0000000000000CD
:102B9000006EE6FFFF4C0300008B080B00009EED6B
:102BA000FFFFF0000000000000009EE6FFFFCB00EA
:102BB00000008B080B00009EEDFFFFF000000000FE
:102BC00000000081E6FFFF850100008B080B00007C
:102BD000A6F8FFFFF0000000000000001DE5FFFF69
:102BE0004C0300008BB50E00009EEDFFFFF00000CF
:102BF00000000000004DE5FFFFCB0000008BB50E8C
:102C000000009EEDFFFFF00000000000000030E536
:102C1000FFFF850100008BB50E0000A6F8FFFFF056
:102C200000000000000000CCE3FFFF4C0300008B1D
:102C3000621200009EEDFFFFF000000000000000A7
:102C4000FCE3FFFFCB0000008B621200009EEDFF53
:102C5000FFF000000000000000DFE3FFFF8501003F
:102C6000008B62120000A6F8FFFFF00000000000D9
:102C700000007BE2FFFF4C0300008B101600009E5B
:102C8000EDFFFFF000000000000000ABE2FFFFCB13
:102C90000000008B101600009EEDFFFFF00000000A
:102CA000000000008EE2FFFF850100008B1016007F
:102CB00000A6F8FFFFF0000000000000002AE1FF7E
:102CC000FF4C0300008BBD1900009EEDFFFFF000DC
:102CD0000000000000005AE1FFFFCB0000008BBDA8
:102CE0001900009EEDFFFFF0000000000000003D15
:102CF000E1FFFF850100008BBD190000A6F8FFFF72
:102D0000F000000000000000D9DFFFFF4C030000CE
:102D10008B6B1D00009EEDFFFFF000000000000027
:102D20000009E0FFFFCB0000008B6B1D00009EED53
:102D3000FFFFF000000000000000ECDFFFFF850156
:102D400000008B6B1D0000A6F8FFFFF000000000E4
:102D500000000088DEFFFF4C0300008B18210000FC
:102D60009EEDFFFFF000000000000000B8DEFFFF56
:102D7000CB0000008B182100009EEDFFFFF000004B
:102D800000000000009BDEFFFF850100008B182182
:102D90000000A6F8FFFFF00000000000000037DD93
:102DA000FFFF4C0300008B18210000A6F8FFFF3046
:102DB000F200000000000037DDFFFFC500000089C1
:102DC0000088000302000088010302000088001F41
:102DD0000200005F002A062A06FF102020546865C2
:102DE000205265706C696361746F7220202020002E
:102DF0002020546865205265706C696361746F723D
:102E00002020202000202020202D2D2D2D2D2D2D87
:102E10002D2D2D20202020202000202020202020AB
:102E2000202020202020202020202020202000469C
:102E300069726D776172652056657273696F6E2075
:102E4000372E2000436F6F6C210053746172742021
:102E50005072656865617421005269676874205416
:102E60006F6F6C004E4120004F4E20004F464600D1
:102E70004578747275646572004C65667420546F91
:102E80006F6C00506C6174666F726D0057656C6397
:102E90006F6D652120202020202020202020202050
:102EA00049276D20546865205265706C69636174B0
:102EB0006F722E205072657373207468652072657E
:102EC00064204D20746F20206765742073746172D4
:102ED0007465642120202020202020200057656C6C
:102EE000636F6D65212020202020202020202020BD
:102EF0002049276D20546865205265706C696361B4
:102F0000746F722E2050726573732074686520721E
:102F10006564204D20746F20206765742073746190
:102F20007274656421202020202020202000412070
:102F3000626C696E6B696E6720274D27206D656135
:102F40006E7349276D2077616974696E6720616EC1
:102F5000642077696C6C636F6E74696E7565207739
:102F600068656E20796F75202020707265737320FC
:102F700074686520627574746F6E2E2E2E20004169
:102F800020736F6C696420274D27206D65616E7317
:102F900020202049276D20776F726B696E67206152
:102FA0006E642077696C6C757064617465206D79EE
:102FB00020737461747573202020207768656E20FB
:102FC00049276D2066696E69736865642E2E2E0030
:102FD0004F7572206E6578742073746570732077F6
:102FE000696C6C20676574206D652073657420754D
:102FF000702120202020202046697273742C2077B5
:1030000065276C6C20726573746F72656D792062D0
:1030100075696C6420706C6174666F726D2E2E2EF3
:1030200000736F2069742773206E69636520616E79
:1030300064202020206C6576656C2E2049742773EF
:103040002070726F6261626C796120626974206FB6
:1030500066662066726F6D202020202020736869CC
:103060007070696E672E2E2E2020202020202020B8
:103070002000416161682C20746861742066656578
:103080006C73202020206D75636820626574746500
:10309000722E20202020202020204C6574277320B1
:1030A000676F206F6E20616E64206C6F6164736F58
:1030B0006D652066696C616D656E7421202020202D
:1030C0002020005765276C6C20747279206167613D
:1030D000696E212020202020202020202020202058
:1030E00020202020202020202020202020202020E0
:1030F00020202020202020202020202020202020D0
:1031000020202020202020202020202020202020BF
:10311000202020005765276C6C206B656570206748
:103120006F696E6720202020616E64206C6F61647F
:1031300020736F6D652020202020202066696C613F
:103140006D656E742C466F722068656C7020676FB9
:10315000746F206D616B6572626F742E636F6D2F7B
:1031600068656C70005765276C6C20676F20746F02
:1031700020746865206D61696E6D656E752E2049DD
:103180006620796F75206E65656420202068656C07
:103190007020676F20746F3A20202020202020208C
:1031A000206D616B6572626F742E636F6D2F686541
:1031B0006C7020202000417765736F6D65212020A1
:1031C000202020202020202020205765276C6C20E4
:1031D000676F20746F2074686520534420206361FA
:1031E0007264206D656E7520616E6420796F752044
:1031F000202063616E2073656C6563742061206DAF
:103200006F64656C21200049276D20676F696E67C8
:1032100020746F206D616B652020206120736572C2
:10322000696573206F66206C696E657320736F77B4
:10323000652063616E2066696E64206D79202020B0
:103240002020206E6F7A7A6C6520616C69676E6DE4
:10325000656E742E202020004C6F6F6B20666F729D
:103260002074686520626573742020206D6174632A
:10327000686564206C696E6520696E2065616368AD
:1032800061786973207365742E204C696E657320B4
:10329000617265206E756D626572656420312D31D5
:1032A0003320616E642E2E2E006C696E65206F6E69
:1032B000652069732065787472612020206C6F6EC0
:1032C000672E2054686520592061786973207365E2
:1032D000746973206C656674206F6E207468652055
:1032E000706C617465616E64205820617869732028
:1032F00069732072696768742E0047726561742172
:1033000020204927766520736176656420207468E3
:103310006573652073657474696E677320616E648C
:10332000202049276C6C20757365207468656D20BA
:10333000746F202020206D616B65206E69636520AD
:103340006D6F64656C73212020200053656C65638C
:10335000742062657374206C696E65732E0058204A
:1033600041786973204C696E65002D2D3E00202048
:103370002000592041786973204C696E6500446FC4
:103380006E6521004D792074656D7065726174758C
:1033900072652077617320206368616E67656420C1
:1033A00065787465726E616C6C792E2052657365F8
:1033B0006C6563742066696C616D656E7420202095
:1033C0006D656E7520746F20747279206167616914
:1033D0006E2E2020004D79206578747275646572B8
:1033E0007320617265202020206E6F7420686561F3
:1033F00074696E672075702E202020202043686538
:10340000636B206D79202020202020202020202088
:1034100020636F6E6E656374696F6E732120202068
:10342000202020202000507265737320646F776E17
:10343000206F6E2074686520202067726579207285
:10344000696E677320617420746F70206F66746892
:10345000652065787472756465727320616E64208E
:10346000202070756C6C2074686520626C61636BE1
:103470002E2E2E20202000507265737320646F77EB
:103480006E206F6E20746865202020677265792039
:1034900072696E6720617420746F70206F6620748B
:1034A000686520657874727564657220616E642049
:1034B00020202070756C6C2074686520626C6163DC
:1034C0006B2E2E2E20202000506C656173652077B6
:1034D000616974207768696C65204920686561744A
:1034E000206D7920657874727564657221202020C2
:1034F00020202020202020202020202020202020CC
:1035000020202020202020202020202020202020BB
:103510002020202020202020006775696465207409
:1035200075626573206F75742E204E6F77666565C2
:10353000642066696C616D656E742066726F6D20C3
:1035400020746865206261636B207468726F7567B0
:103550006820746865747562657320756E74696C33
:103560002069742E2E2E2020200067756964652046
:1035700074756265206F75742E20204E6F776665B6
:1035800065642066696C616D656E742066726F6D2E
:103590002020746865206261636B207468726F75A7
:1035A0006768207468657475626520756E74696CEF
:1035B0002069742E2E2E2020202000706F70732022
:1035C0006F757420696E2066726F6E742E202049AC
:1035D000276D2068656174696E67207570206D794C
:1035E000202020657874727564657220736F20776F
:1035F000652063616E20206C6F61642074686520B3
:1036000066696C616D656E742E2E2E005468697348
:10361000206D696768742074616B652061202020CB
:10362000666577206D696E757465732E2020202085
:1036300020202020416E64207761746368206F75BC
:10364000742C2074686520206E6F7A7A6C65207700
:10365000696C6C2067657420484F5421004865618F
:1036600074696E672050726F67726573733A2020B9
:10367000202020202020202020202020202020204A
:10368000202020202020202020202020202020203A
:10369000202020202020202020202020202020202A
:1036A00020202020202020202020202020004F4BE0
:1036B0002049276D20726561647921202020202017
:1036C00020204669727374207765276C6C206C6FBC
:1036D00061642074686572696768742065787472C3
:1036E000756465722E202020202050757368206636
:1036F000696C616D656E7420696E2E2E2E200047F8
:103700007265617421204E6F77207765276C6C207D
:103710002020206C6F616420746865206C6566747D
:103720002020202020202065787472756465722E18
:10373000205075736820202020202066696C616D00
:10374000656E74207468726F7567682E2E2E200067
:103750004F4B2049276D207265616479212020201C
:103760002020202050757368207468652066696C7D
:10377000616D656E742020207468726F7567682EA5
:103780002E2E20202020202020202020202020201D
:103790002020202020202020202020202020202029
:1037A0000049276D207265616479212050756C6C29
:1037B000207468652067756964652074756265208A
:1037C0006F666620616E642020707573682074686F
:1037D000652066696C616D656E7420202074687266
:1037E0006F7567682E2E2E2020202020202020207C
:1037F000200049276D207265616479212050756C25
:103800006C207468652067756964652074756265ED
:10381000206F666620616E64202070756C6C207469
:1038200068652066696C616D656E7420202067652F
:103830006E746C792E2E2E20202020202020202017
:1038400020200049276D207265616479212044653C
:1038500074616368202020746865206775696465F9
:1038600020747562652C206F70656E746865206CBD
:10387000657665722061726D20616E642020207013
:10388000756C6C2066696C616D656E74206672651E
:10389000652E200049276D207265616479212044DE
:1038A00065746163682020207468652067756964A9
:1038B0006520747562652C206F70656E7468652074
:1038C0006C657665722061726D20616E64202020C7
:1038D00070756C6C2066696C616D656E74206672C3
:1038E00065652E2000756E74696C20796F75206691
:1038F00065656C2074686520206D6F746F7220742C
:10390000756720697420696E2E2020202050757301
:103910006820666F72206120666577206D6F726522
:10392000207365636F6E64732C207468656E2077F6
:103930006169742E20005768656E2066696C616D40
:10394000656E74206973202020206265696E67208F
:1039500065787472756465642066726F6D20746832
:1039600065206E6F7A7A6C652C20507265737320B7
:103970004D20746F2073746F702065787472756455
:10398000696E672E2020005768656E2066696C613D
:103990006D656E74206973202020206265696E67F2
:1039A0002065787472756465642066726F6D20742A
:1039B0006865206E6F7A7A6C652C2020202020208C
:1039C000202020507265737320274D2720746F20AC
:1039D000657869742E2020005768656E206D792007
:1039E00066696C616D656E742069732072656C65C3
:1039F000617365642C20202020202020202020209E
:103A0000507265737320274D2720746F2065786985
:103A1000742E202020202020202020202020202044
:103A20002020202020202020005768656E206D79FE
:103A30002066696C616D656E742069732072656CB7
:103A400065617365642C2020202020202020202008
:103A500020507265737320274D2720746F2065787E
:103A600069742E20202020202020202020202020AB
:103A70002020202020202020200047726561742112
:103A8000202049276C6C2073746F70202020727581
:103A90006E6E696E67206D792065787472756465E5
:103AA000722E5072657373204D20746F20636F6E99
:103AB00074696E75652E2020202020202020202073
:103AC00020202020202020202020004F4B21204992
:103AD000276C6C206B656570206D79202020206D2F
:103AE0006F746F722072756E6E696E672E20596FDB
:103AF0007520206D6179206E65656420746F20707B
:103B0000757368202020206861726465722E2E2EE5
:103B10002020202020202020202020005765276CF6
:103B20006C206B65657020676F696E672E202020A2
:103B30004C6574732074727920746865206C6566B6
:103B40007420202065787472756465722E2050751B
:103B5000736820202020202066696C616D656E747A
:103B600020646F776E2E2E2E202020200057652790
:103B70006C6C206B65657020676F696E672E202006
:103B800020496620796F7527726520686176696EB5
:103B9000672020202074726F75626C652C2063682A
:103BA00065636B206F757420206D616B6572626F49
:103BB000742E636F6D2F68656C70202020004D7926
:103BC000206D6F746F722074696D6564206F7574F9
:103BD000202061667465722035206D696E7574658C
:103BE000732E202020205072657373204D20746F37
:103BF00020657869742E202020202020202020207D
:103C000020202020202020202020202020200048AC
:103C10006F77276420697420676F3F205265616465
:103C200079202000746F206D616B6520736F6D6566
:103C30007468696E673F202000596573202020005A
:103C40004E6F2020202000446F6573206D79206E18
:103C50006F7A7A6C652000686569676874206368AC
:103C600065636B206F75743F20004D79206865692E
:103C700067687420697320676F6F64212020004C8F
:103C8000657427732074727920616761696E2E00F4
:103C900044696420706C6173746963206578747220
:103CA000756465200066726F6D20746865206E6FA4
:103CB0007A7A6C653F20202020004C6F616420726E
:103CC00069676874004C6F616400556E6C6F616465
:103CD00020726967687400556E6C6F6164004C6F88
:103CE0006164206C65667400556E6C6F6164206C55
:103CF0006566740020202020204A6F67206D6F6465
:103D0000652020202020202000202020202020208E
:103D100020582B2020202020202020202000202080
:103D200020202020284261636B29202020592D3E2D
:103D30002020002020202020202020582D2020205E
:103D40002020202020202000202020202020202093
:103D5000592B202020202020202020200020203C23
:103D60002D5820284261636B2920205A2D3E2020A7
:103D700020002020202020202020592D202020201D
:103D80002020202020200020202020202020205A19
:103D90002D202020202020202020200020203C2D0D
:103DA0005920284261636B292020202020202020D8
:103DB0000020202020202020205A2B2020202020DE
:103DC00020202020200047414D45204F56455221BC
:103DD0000048656174696E673A2020202020202009
:103DE00020202020200048656174696E673A002019
:103DF000202020202000202D2D25006572726F725A
:103E000021002020202020202020202020202020D1
:103E10002020202020200045787472756465723A55
:103E20002020202D2D2D2F2D2D2D43005220457883
:103E30007472756465723A202D2D2D2F2D2D2D4312
:103E4000004C2045787472756465723A202D2D2DD2
:103E50002F2D2D2D4300506C6174666F726D3A20CA
:103E600020202D2D2D2F2D2D2D430020204E4120A3
:103E70002020200077616974696E6720002F202060
:103E80002043004320202020006820206D00205087
:103E90007265686561742053657474696E67732018
:103EA000202000526967687420546F6F6C202020B6
:103EB00020202020202020004C65667420546F6F45
:103EC0006C202020202020202020202000506C6109
:103ED00074666F726D202020202020202000205248
:103EE000657365742053657474696E677320746FAD
:103EF0002020002044656661756C742076616C75C5
:103F000065733F00556E5061757365202020202039
:103F10002020202020202000506175736520202063
:103F200020202020202020202020200043616E63BC
:103F3000656C204275696C642020202020202000C0
:103F400057616974696E6720666F7220486F6D698A
:103F50006E6720004368616E67652046696C616D1D
:103F6000656E742020202000536C65657020284306
:103F70006F6C6420506175736529200052657375FC
:103F80006D65204275696C6420202020202020006F
:103F90005A205061757365204865696768742020F0
:103FA000202020004C454420436F6C6F722020205D
:103FB0002020202020202000524544202020004F97
:103FC00052414E47450050494E4B20200047524534
:103FD000454E2000424C5545202000505552504C33
:103FE000450057484954452000435553544F4D0010
:103FF0004F46462020200046696C616D656E742036
:1040000046616E20202020202020004275696C64CB
:1040100020537461746973746963732020200042B3
:1040200061636B20746F204D6F6E69746F72202016
:104030002020004275696C642046696E697368656A
:10404000642120202020202020202020202020202B
:1040500020202020202020202020204275696C6410
:104060002054696D652020202020206820206D00CC
:104070004275696C642054696D653A2020202020C7
:104080006820206D004C696E653A20202020202099
:1040900020202020202020202000457374696D619D
:1040A000746564204275696C642054696D654C695F
:1040B000666574696D6520546F74616C3A202020C8
:1040C0002068004C617374204275696C643A20204A
:1040D0002020206820206D0043616E63656C207491
:1040E000686973206275696C643F0051756974205A
:1040F000746869732070726F636573733F004275F3
:10410000696C642066726F6D20534420202020204B
:1041100020005072656865617420202020202020D6
:104120002020202020005574696C69746965732013
:1041300020202020202020202000496E666F206152
:104140006E642053657474696E67732020004D6F30
:104150006E69746F72204D6F6465202020202020CE
:1041600020004368616E67652046696C616D656E0D
:104170007420202020004C6576656C204275696CA7
:104180006420506C6174652020004A6F67204D6F79
:104190006465202020202020202020202000486F3F
:1041A0006D6520417865732020202020202020206C
:1041B000200052756E2053746172747570205363C1
:1041C000726970742000456E61626C65205374657D
:1041D0007070657273202020200044697361626CE6
:1041E00065205374657070657273202020005374CD
:1041F0006F7020426C696E6B696E672120202020F1
:104200002000426C696E6B204C45447320202020B6
:1042100020202020200043616C6962726174652057
:104220004E6F7A7A6C657320200065786974206D12
:10423000656E752020202020202020202000426F45
:10424000742053746174697374696373202020202F
:10425000200047656E6572616C2053657474696EE9
:104260006773202020005072656865617420536573
:104270007474696E67732020200056657273696FCD
:104280006E204E756D6265722020202020005265E0
:1042900073746F72652044656661756C7473202059
:1042A00020002020205A20506175736520486569E0
:1042B000676874202020005A20506F736974696FFA
:1042C0006E2020202020206D6D20005061757365C8
:1042D000204163746976652020202020202000532F
:1042E0006F756E6420202020202020202020202098
:1042F00020200048656174656420506C617465001D
:10430000546F6F6C20436F756E7420202020202026
:104310002020200053494E474C45004455414C2035
:10432000200048656174204C4544732020202020E3
:104330002020202020004865617420486F6C642094
:1043400020202020206D2020200048656C70205403
:104350006578742020202020202020202000416328
:1043600063656C6572617465202020202020202008
:1043700020004E6F205344206361726420666F7585
:104380006E6400534420636172642072656164202E
:104390006572726F7200492063616E2774207265C6
:1043A0006164207468697320202053442063617223
:1043B0006420666F726D6174212020202020547269
:1043C00079207265666F726D617474696E67202002
:1043D0002020746865206361726420746F204641F8
:1043E0005431362E202000492063616E27742072DC
:1043F000656164205344202020202063617264732F
:1044000020776974682073746F7261676520206C0F
:104410006172676572207468616E203247422E2097
:10442000202020202020202020202020202020208C
:10443000202020202020200020534420636172642B
:104440002072656164206572726F720049276D2069
:10445000616C7265616479206275696C64696E670C
:10446000005761726E696E673A4275696C642073B9
:104470007065656473666173746572207468616EDB
:104480002035306D6D2F73202072657175697265EE
:104490002078336720666F726D61742020666F72BA
:1044A000206265737420726573756C74732E20209E
:1044B0002000D0FEC0FF18FFD0FF63FFE0FFB1FF78
:1044C000F0FF0000000051001000A4002000F800E0
:1044D000300040014000A2015000F70160004B0293
:1044E00070009F028000F20290004503A000970335
:1044F000B000E803C0003A04D0008C04E000DF0400
:10450000F0003205000186051001DB0520012F06B1
:104510003001DA0650013007600186077001DC07C0
:1045200080016808900120F9C9FFE0FCE7FFF8FF6F
:1045300000000000000008000000200319004006F1
:10454000320060094B00000A5000800C640000102B
:104550008000010049033600FF006B00D100A0007D
:10456000B800D500A6000A0199003F018E00740131
:104570008400A9017C00DE01740013026C00480273
:1045800065007D025D00B2025600E7024E001C038A
:10459000460051033D0086033200BB032200F003B6
:1045A000030067328E324036F63F5A40794A194C42
:1045B000934FF0507F6415762479308462854B8662
:1045C00034876088BF8A77962697FD9A8F9B789C60
:1045D000359D5F9E87A3D3A3CEA7A1AB69CD27CF7F
:1045E000AED0B1D26AD346D411241FBECFEFD1E2F0
:1045F000DEBFCDBF15E0A0E0B2E0E0E3F6EB01E006
:104600000BBF02C007900D92A23BB107D9F72DE175
:10461000A2EBB5E001C01D92AB33B207E1F715E4A0
:10462000C8EED5E400E006C022970109FE010BBFE9
:104630000E9405DAC23AD10780E00807A9F70E9474
:1046400046400C9416DB0C940000FA01DC0102C019
:1046500005900D9221503040D8F70895F89480913C
:10466000F6059091F7052091F4053091F505281B8A
:10467000390B7894C90108958093ED05089581E080
:104680008093EB0508958091ED0508958091EC05E8
:1046900008952091F6053091F70581E0232B09F06C
:1046A00080E008951092F7051092F6051092F90532
:1046B0001092F8051092FC051092FD051092EF057E
:1046C0001092F0051092F1051092F2051092EE058D
:1046D0001092ED051092EC051092E6051092E70598
:1046E0001092E8051092E9051092D1051092E505A7
:1046F0001092E4051092E305089581E02091E3050E
:104700003091E4052630310509F080E0089560918C
:10471000EF057091F0058091F1059091F2050895F3
:104720001092EF051092F0051092F1051092F2052B
:1047300008954F925F926F927F928F929F92AF9265
:10474000BF92CF92DF92EF92FF920F931F93CF937E
:10475000DF93CDB7DEB7C256D1090FB6F894DEBFEE
:104760000FBECDBFCE018D5B9F4F0E94647B84E165
:10477000FE01ED5BFF4FA5EBB5E001900D928A9530
:10478000E1F745E06FE57AE1CE01CD960E944CD08D
:10479000CE01CD960E948ED08093B40564E070E087
:1047A00085EB95E00E94794CDC016D917D918D91B6
:1047B0009C910E94CAD62B013C0184E00E94A07803
:1047C0009B01AC0163E070E085EB95E0A0962FAF14
:1047D000A097A1963FAFA197A2964FAFA297A3969D
:1047E0005FAFA3970E94794CFC0180809180A280EA
:1047F000B38083E00E94A0786B966CAF7DAF8EAFE4
:104800009FAF6B9762E070E085EB95E00E94794C7A
:10481000DC01CD90DD90ED90FC9061E070E085EBE7
:1048200095E00E94794CDC018D919D910D90BC9199
:10483000A02D6F968CAF9DAFAEAFBFAF6F9760E00E
:1048400070E085EB95E00E94794C8C016B966CAD25
:104850007DAD8EAD9FAD6B970E949CD6860E971E48
:10486000A81EB91ED8018D919D910D90BC91A02DCF
:104870006B968CAF9DAFAEAFBFAF6B97A0962FADD1
:10488000A097A1963FADA197A2964FADA297A396F0
:104890005FADA397C301B2010E947AD50E9497D65B
:1048A0009F938F937F936F936F960CAD1DAD2EAD3D
:1048B0003FAD6F976B964CAD5DAD6EAD7FAD6B97B9
:1048C000CE0189960E943D4C48E052E060E070E0E5
:1048D000CE0189960E94FA7B8CE099E00E946FA13C
:1048E0009093CC058093CB058CEB99E00E946FA14F
:1048F0009093CE058093CD058CEF9BE00E946FA135
:104900009093CA058093C9050F900F900F900F9058
:104910008091EA05882391F060E070E08CE099E0F6
:104920000E9499A060E070E08CEB99E00E9499A051
:1049300060E070E08CEF9BE00E9499A084E1FE01B2
:10494000B996DE01559601900D928A95E1F762E0E5
:1049500070E0CE0145960E94794C8C0182E00E9465
:10496000A0780E9497D69B01AC01A6E9B0E00E9416
:10497000CCD8F801608371838283938384E1FE0144
:104980007596DE01119601900D928A95E1F760E02F
:1049900070E0CE0101960E94794C8C0180E00E946B
:1049A000A07820E030E04DED52EC0E94CED70E947E
:1049B00097D6D8016D937D938D939C93139761E067
:1049C00070E0CE0101960E94794C8C0181E00E943A
:1049D000A07820E030E044E952EC0E94CED70E945B
:1049E00097D6F80160837183828393834CE850E00B
:1049F00060E070E0CE0145960E94FA7B42E850E00C
:104A000060E070E0CE0101960E94FA7B60E08CECE1
:104A100098E00E94494ACE59DF4F0FB6F894DEBFA6
:104A20000FBECDBFDF91CF911F910F91FF90EF90FF
:104A3000DF90CF90BF90AF909F908F907F906F90BE
:104A40005F904F9008950F931F93CF93DF93CDB74F
:104A5000DEB764970FB6F894DEBF0FBECDBFCE01B0
:104A600001960E94647B63E070E0CE0101960E9493
:104A7000794C8C0163E070E085EB95E00E94794C05
:104A8000FC014081518162817381F801408351832F
:104A90006283738364E070E0CE0101960E94794CDA
:104AA0008C0164E070E085EB95E00E94794CFC019C
:104AB0004081518162817381F80140835183628317
:104AC0007383CE0101960E94E77962E070E0CE0127
:104AD00001960E94794C8C0162E070E085EB95E0D4
:104AE0000E94794CFC014081518162817381F801FF
:104AF00040835183628373834CE850E060E070E050
:104B0000CE0101960E94FA7B42E850E060E070E03E
:104B100085EB95E00E94FA7B6091B4058CEC98E0FF
:104B20000E94494A64960FB6F894DEBF0FBECDBF0F
:104B3000DF91CF911F910F9108956091CB057091F6
:104B4000CC058CE099E00E9499A06091CD05709110
:104B5000CE058CEB99E00E9499A06091C9057091F7
:104B6000CA058CEF9BE00E9499A08CEF9BE00E940D
:104B700083A1882329F18CEF9BE00E949DA18111E4
:104B80001FC017C061E08CE099E00E94CFA181E0D6
:104B90008093EE058CEB99E00E949DA1811110C0DD
:104BA00061E08CEB99E00E94CFA181E08093EE055B
:104BB00008958CE099E00E949DA18111EBCFE2CF96
:104BC0000895CF93DF93EB01709305026093040285
:104BD0009091EC05981709F44BC0882329F1209790
:104BE00081F481E08093EA056CE171E081EB9AE069
:104BF0000E9403A581E090E09093D0058093CF05BB
:104C00000FC06130710561F41092EA0569E571E049
:104C100081EB9AE00E9403A5D093D005C093CF0505
:104C200081E08093EC0524C08091CF059091D00560
:104C30008130910529F41092D0051092CF0516C04D
:104C40008230910529F40E949D2584E090E006C001
:104C5000039749F40E949D2585E090E09093D0054C
:104C60008093CF0505C06230710511F41092EC05F8
:104C7000DF91CF910895CF93FC01C62F828193815C
:104C8000608171818617970798F4428153818481EE
:104C90009581840F951F0E944DD8A681B781A80FDA
:104CA000B91FCC938281938101969383828302C042
:104CB00081E08087CF910895682F84EF95E00C9470
:104CC0003B26CF93DF93FC0182819381892B21F4D2
:104CD00081E0818780E019C08481958120813181C4
:104CE000B9010E944DD8C681D781C80FD91F8481D0
:104CF00095810196B9010E944DD895838483828164
:104D000093810197938382838881DF91CF91089566
:104D10001F93CF93DF9300D0CDB7DEB784EF95E03C
:104D20000E946126682F84EF95E06A830E946126C5
:104D3000782F84EF95E079830E946126182F84EF05
:104D400095E00E946126982F6A817981812F0F90CA
:104D50000F90DF91CF911F910895CF9384EF95E04D
:104D60000E946126C82F84EF95E00E946126982F4B
:104D70008C2FCF91089584EF95E00C946126CF930A
:104D8000DF930E94BB26D82F0E94BB26C82F0E940B
:104D9000BB26CA3009F4E8C098F4C63009F4E1C073
:104DA00048F4C43009F4E0C008F0DEC0C33009F0B4
:104DB000DEC01AC0C83009F4D7C008F0D5C0D1C0D1
:104DC000CE3009F4D1C030F4CC3009F46CC008F016
:104DD00078C0CAC0C73109F45FC0CF3109F47AC0C6
:104DE000CF3009F0C4C0C0C08091B3058823A1F0C2
:104DF0008CE099E00E949F9F8CEB99E00E949F9F1E
:104E00008091B205811104C08CEF9BE00E949F9FAE
:104E10001092B2051092B3050E94AD26BC01D130AC
:104E200019F483EA99E002C083EF98E049960E9462
:104E300099A08CEF9BE00E9483A1882309F4A2C073
:104E40008CEF9BE00E949DA181119CC0D13019F490
:104E500083EA99E002C083EF98E049960E949DA101
:104E6000811190C086C083EA99E061E003C083EAC3
:104E700099E060E049960E94CFA140E061E070E0D7
:104E80008CEC98E00E948B43D13009F08EC00E94D8
:104E9000F73381117DC089C09091ED0581E08927AC
:104EA0000E944C3A82C00E94BB26682F6170D130AC
:104EB00019F483EA99E002C083EF98E00E94EC873E
:104EC00074C00E94BB26682F61708CEC98E00E9431
:104ED000494A6BC061E08CEC98E00E94444A8091A2
:104EE000B305882319F081E08093B2050E94AD26B6
:104EF000BC018CEF9BE00E9499A08CEF9BE00E948C
:104F00009DA1C1E0C827C093EE056C2F8CE099E00D
:104F10000E94CFA16C2F8CEB99E00E94CFA140E0C2
:104F200061E070E08CEC98E00E948B430E94E434D6
:104F300081113BC00E94D739059739F040E067EEF8
:104F400071E08CEC98E00E946D4360E070E08CEFC3
:104F50009BE00E9499A060E08CEC98E00E94444A9B
:104F600024C00E94882621C00E94BB261EC080E06B
:104F70001DC081E08093EE05D13009F474CF83EF3A
:104F800098E073CFD13009F472CF83EF98E071CFFE
:104F900040E066E971E08CEC98E00E946D4360E0CF
:104FA00070E08CEB99E00E9499A081E0DF91CF91B5
:104FB00008952F923F924F925F926F927F928F92BD
:104FC0009F92AF92BF92CF92DF92EF92FF920F9398
:104FD0001F93CF93DF93CDB7DEB7E7970FB6F89463
:104FE000DEBF0FBECDBF0E94FA4D882309F492C0E8
:104FF0008091F6059091F7052091F4053091F50523
:105000002817390711F40C9446310E94674E81111C
:105010000C944C310C944631C090E605D090E705D5
:10502000E090E805F090E9050E94A94DC616D70664
:10503000E806F90610F00C9473318091D1058111C6
:105040000C9473310C94683181EB9AE00E9429A48E
:1050500040E068E372E08CEC98E00E946D4381E0F0
:105060008093D1050E9432811092F7051092F605C7
:105070001092F9051092F8051092FC051092FD05AA
:1050800060E070E08CE099E00E9499A060E070E040
:105090008CEB99E00E9499A060E070E08CEF9BE0BF
:1050A0000E9499A0CE0101960E94D07A62E070E041
:1050B000CE0101960E94794C8C0182E00E94A0787A
:1050C00020E030E046E153E40E94CED70E9497D61C
:1050D000F80160837183828393831092ED0546E922
:1050E00050E060E070E0CE0101960E94FA7B0E94E1
:1050F000794E1092E5050EC08091F6059091F70566
:10510000892B41F48091E3059091E405892B11F4FA
:105110000C947A310E94E384882311F18091F60582
:105120009091F7052091F4053091F505281739077E
:1051300011F40C947E310E94EC8481110C94853121
:105140000C947E318091F6059091F705892B41F4FE
:105150008091E3059091E405892B11F40C948E3134
:105160008091EE05882391F08CEF9BE00E944BA18B
:10517000882361F060E08CE099E00E94CFA160E0BC
:105180008CEB99E00E94CFA11092EE058091ED0585
:1051900081110C944E328091EB0581110C944E32AA
:1051A0008091E3059091E405039789F40E94437987
:1051B000811101C008C084ED95E00E94E0D28823EF
:1051C00031F00E9432811092E4051092E305809143
:1051D000E3059091E405019741F40E944379811120
:1051E00004C01092E4051092E3058091E3059091CC
:1051F000E405029751F484ED95E00E94E0D2882303
:1052000021F01092E4051092E3058091E30590915E
:10521000E405049709F049C084ED95E00E94E0D2CE
:10522000882349F040E069E872E08CEC98E00E9445
:105230006D430C949F318091F305813019F483EA1A
:1052400099E002C083EF98E049960E944BA1882321
:1052500011F40C9492318091F305813019F483EAB2
:1052600099E002C083EF98E0FC01E157FF4F808195
:1052700081110C9492310C949C3183EF98E0499603
:105280000E9483A1811111C08091F305813019F42E
:1052900083EA99E002C083EF98E0FC01E157FF4FF9
:1052A0008081882311F40C949F318091E3059091C3
:1052B000E4050597F9F484ED95E00E94E0D2882397
:1052C00041F040E066EC72E08CEC98E00E946D43A7
:1052D0000DC08CEF9BE00E9483A1811101C006C02C
:1052E0008CEF9BE00E944BA1882321F01092E405F3
:1052F0001092E3058091E3059091E405069709F08B
:105300003FC084ED95E00E94E0D28823B1F0809107
:10531000D20581FF06C060E08CEC98E00E94534803
:105320002FC01092E4051092E30540E060E170E0C8
:105330008CEC98E00E948B4323C081EB9AE00E94A2
:10534000C6A78823E9F08091D20582FF04C081EBD3
:105350009AE00E9498A540E050E060E070E08CEC9C
:1053600098E00E94574640E060E170E08CEC98E0E5
:105370000E948B430E94198A1092E4051092E30563
:105380008091E3059091E405892B09F064C7809131
:10539000EC05882309F4E2C08091CF059091D005F7
:1053A000019709F0D2C70E944D638111D5C7CDC7BF
:1053B00063E073E004C0019731F464E573E081EBCE
:1053C0009AE00E9403A50E94992382E090E096C093
:1053D0000E944D638111D1C7C7C740E059EE64EA0E
:1053E00075E384ED95E00E94BCD286E00E94DC4B20
:1053F0008091040290910502892B11F00C944E3299
:1054000064E180E00E94498064E181E00E9449807B
:1054100064E183E00E94498064E184E00E94498065
:105420000C944E328091040290910502019711F084
:105430000C944E3284ED95E00E94E0D28111ADC70C
:105440000C944E32049749F08091CF059091D0058D
:105450008530910509F0DEC7E2C70E944D638111D6
:10546000DEC7F2CF6FE780E00E9449806FE781E0FE
:105470000E9449808091040290910502892B41F499
:105480006FE783E00E9449806FE784E00E944980D3
:1054900062EE73E081EB9AE00E9403A51092F3059F
:1054A00085E090E09093E4058093E30540E052EDC1
:1054B00069E47BE684ED95E00E94BCD286E090E052
:1054C0009093D0058093CF0524E140E063E08CEC1D
:1054D00098E00E94B443E2C71092F30584E090E0A4
:1054E0009093E4058093E30540E052ED69E47BE6A8
:1054F00084ED95E00E94BCD287E090E09093D005C7
:105500008093CF05CBC787309105A1F481E08093CC
:10551000F30584E090E09093E4058093E30540E098
:1055200052ED69E47BE684ED95E00E94BCD288E010
:1055300090E0E4CF8830910549F48CEC98E00E942B
:10554000CA430E94232589E090E0D8CF099709F04B
:10555000A5C70E944D6381116AC7A0C78091F60557
:105560009091F705892B09F476C68CEC98E00E949F
:10557000EF458091F8059091F9056091F4057091DF
:10558000F5050E944DD8E091FA05F091FB05E80F72
:10559000F91F10811B3809F45DC71E3809F462C772
:1055A0001B3909F44FC7193809F464C7163909F4CF
:1055B00032C3163809F46AC71C3841F48091F605E5
:1055C0009091F705459708F446C6CEC11C3909F4F9
:1055D00022C3103909F41FC3133809F41CC314384B
:1055E00009F419C3183809F416C30E944D638111D8
:1055F00049C754C78CEC98E00E94EF450E94BB2637
:1056000081E090E09093E4058093E3050E94882672
:1056100068A779A78AA79BA70E9488266CA77DA761
:105620008EA79FA70E9488266B017C010E94882676
:105630004B015C010E948826162F072F382E292E39
:105640000E9488262B013C018091EF059091F00586
:10565000A091F105B091F2050196A11DB11D8093B5
:10566000EF059093F005A093F105B093F2052F920A
:105670003F920F931F930CA51DA52EA53FA548A5EE
:1056800059A56AA57BA5CE0101960E943D4CB301A8
:10569000A201CE0101960E94FA7B58C08CEC98E0E2
:1056A0000E94EF450E94BB2681E090E09093E405C4
:1056B0008093E3050E94882668A779A78AA79BA7FD
:1056C0000E9488266CA77DA78EA79FA70E94882688
:1056D0006B017C010E9488264B015C010E94882698
:1056E000162F072F282E9EAB0E9488262B013C01E7
:1056F0000E94BB26382E8091EF059091F005A09175
:10570000F105B091F2050196A11DB11D8093EF0541
:105710009093F005A093F105B093F2052EA92F9375
:105720002F920F931F930CA51DA52EA53FA548A54D
:1057300059A56AA57BA5CE0101960E943D4C232D5B
:10574000B301A201CE0101960E94E97C0F900F9057
:105750000F900F9080C58CEC98E00E94EF450E945E
:10576000BB2681E090E09093E4058093E3050E94DE
:10577000882668A779A78AA79BA70E9488266CA776
:105780007DA78EA79FA70E9488266B017C010E949F
:1057900088264B015C010E948826162F072F282E91
:1057A0009EAB0E9488262B013C010E94BB26382E0E
:1057B0000E94882668AB79AB8AAB9BAB0E94AD2672
:1057C0009DAB8CAB8091EF059091F005A091F10518
:1057D000B091F2050196A11DB11D8093EF05909344
:1057E000F005A093F105B093F2052EA92F932F9207
:1057F0000F931F930CA51DA52EA53FA548A559A540
:105800006AA57BA5CE0101960E943D4CCCA8DDA8DF
:10581000E8A8F9A80AA91BA9232DB301A201CE016A
:1058200001960E94F97D92CF0E94BB260E94BB2662
:105830008093F3054091EF055091F0056091F105DB
:105840007091F2054F5F5F4F6F4F7F4F4093EF05B1
:105850005093F0056093F1057093F2050E94578014
:10586000FAC40E94BB260E94BB26E82E4091EF0599
:105870005091F0056091F1057091F2054F5F5F4F17
:105880006F4F7F4F4093EF055093F0056093F10504
:105890007093F2050E944D63882309F4DCC4DE2C6A
:1058A000DD1CDD24DD1C00E010E0F12CC701002E22
:1058B00002C0959587950A94E2F780FF04C06D2D8C
:1058C000802F0E9430800F5F1F4F0530110571F748
:1058D000C2C48091F6059091F7050B9708F4BBC4FC
:1058E0000E94BB260E94BB26182F0E94BB26282F91
:1058F00030E0F4E61F9F200D311D112424363105C0
:1059000039F040E067EF73E08CEC98E00E946D4363
:105910000E94BB260E9488260E94AD268431934DAA
:1059200039F040E068E474E08CEC98E00E946D434C
:105930000E94AD260E9488260E9488260E94BB26CF
:105940008091EF059091F005A091F105B091F205DD
:105950000196A11DB11D8093EF059093F005A093D2
:10596000F105B093F20577C40E94BB260E948826F9
:105970002B013C010E94882668A779A78AA79BA7CC
:105980000E9488266B017C010E9488264B015C01E5
:105990000E9488269B014091EF055091F00560918F
:1059A000F1057091F2054F5F5F4F6F4F7F4F40934E
:1059B000EF055093F0056093F1057093F2059F9306
:1059C0008F933F932F9308A519A52AA53BA5B30153
:1059D000A201CE0101960E943D4CCE0101960E948B
:1059E000E779B4CE153849F58091F6059091F70521
:1059F000059708F430C482E090E09093E40580932A
:105A0000E3050E94BB260E9488269B01AC01809181
:105A1000EF059091F005A091F105B091F205019686
:105A2000A11DB11D8093EF059093F005A093F105A2
:105A3000B093F205A8EEB3E074C1143909F047C081
:105A40008091F6059091F705059708F404C40E942B
:105A5000BB260E94BB268093D3050E94AD268C01F5
:105A60000E94BB268093D2054091EF055091F0052E
:105A70006091F1057091F2054F5F5F4F6F4F7F4F5F
:105A80004093EF055093F0056093F1057093F20594
:105A90000115110571F0D80120E432E44FE050E027
:105AA0000E94CCD8AB01BC0184ED95E00E94BCD231
:105AB00096C0CE0145960E94B8D28FE0FE01759641
:105AC000A4EDB5E001900D928A95E1F788C01539F3
:105AD00009F0A1C081EB9AE00E944AA48C01809158
:105AE000F6059091F705069708F4B5C30E94BB260A
:105AF0000E94BB26E82E0E94BB26C82E0E94BB2611
:105B0000D82E0E94BB26F82E4091EF055091F0054B
:105B10006091F1057091F2054F5F5F4F6F4F7F4FBE
:105B20004093EF055093F0056093F1057093F205F3
:105B3000E0FC03C0C8010E949AC9F801C282D38266
:105B400064EF75E0C8010E94FEC8E1FE84C3E091E5
:105B5000E00BEE0FFF0BEE52F44F20813181201746
:105B6000310731F0B80181EB9AE00E9466A403C0CE
:105B7000C8010E94E3C98E2D8470FF2039F0811185
:105B800005C06F2DC8010E94D3C965C3882309F4DD
:105B900062C3FF2079F0AF2DB0E020E432E44FE0A3
:105BA00050E00E94CCD8AB01BC0184ED95E00E948E
:105BB000BCD20DC0CE0145960E94B8D28FE0FE0146
:105BC0007596A4EDB5E001900D928A95E1F781E01C
:105BD0008093D3058091D20584708093D2054FE0E5
:105BE00050E069E170E08CEC98E00E9457466091CB
:105BF000D30581EB9AE00E94C1A741E060E170E02B
:105C00008CEC98E00E948B4386E090E09093E40552
:105C10008093E30520C3812F8358823008F043C06E
:105C20008091F6059091F705089708F414C30E9437
:105C3000BB260E94BB26082F0E9488266B017C0190
:105C40000E94AD26DC014091EF055091F005609176
:105C5000F1057091F2054F5F5F4F6F4F7F4F40939B
:105C6000EF055093F0056093F1057093F20583E022
:105C700090E09093E4058093E30520E432E44FE064
:105C800050E00E94CCD8AB01BC0184ED95E00E94AD
:105C9000BCD281E0143809F080E0A7019601602FA2
:105CA0000E94967FD8C2173851F48091F6059091E2
:105CB000F705069708F4CFC284E090E00BC01D38CA
:105CC000C9F58091F6059091F705069708F4C3C2CF
:105CD00085E090E09093E4058093E3050E94BB2665
:105CE0000E94BB268093F3050E94AD260E94AD263C
:105CF0004091EF055091F0056091F1057091F2052A
:105D00004F5F5F4F6F4F7F4F4093EF055093F0050C
:105D10006093F1057093F205DC0120E432E44FE07A
:105D200050E00E94CCD8AB01BC0184ED95E00E940C
:105D3000BCD291C21F3809F06EC08091F6059091D7
:105D4000F705029708F487C20E94BB260E94BB2673
:105D50004091EF055091F0056091F1057091F205C9
:105D60004F5F5F4F6F4F7F4F4093EF055093F005AC
:105D70006093F1057093F20524E2E22E22E0F22E08
:105D800000E010E0C82ED12C38EE832E33E0932EA5
:105D9000A12CB12CC601002E02C0959587950A94BE
:105DA000E2F780FF2EC0CE0101960E94647BB8010D
:105DB000CE0101960E94714CFC016081718182814B
:105DC00093816CA37DA38EA39FA3402F0E94B678DE
:105DD00020E030E04AE754E40E94CED70E9497D6F4
:105DE000A50194010E9497D82CA33DA34EA35FA3C5
:105DF000F89444E050E0B701CE0184960E94E9DABD
:105E000078940F5F1F4FF4E0EF0EF11C0530110581
:105E100009F0C0CF20C2103909F06DC08091F6059D
:105E20009091F705029708F416C20E94BB260E94C3
:105E3000BB26C82E4091EF055091F0056091F10509
:105E40007091F2054F5F5F4F6F4F7F4F4093EF05AB
:105E50005093F0056093F1057093F205AA24A39482
:105E6000B12CAC0EBD1EC5010E94647B94E2E92EEC
:105E700092E0F92E00E010E0D12C9A2C8B2CC60178
:105E8000002E02C0959587950A94E2F780FF26C000
:105E9000F894B801892D982D0E94794C44E050E087
:105EA000B7010E94D3DA7894B801892D982D0E9409
:105EB000794C5C01B801892D982D0E94794CFC0128
:105EC00060817181828193810E94CAD6402F0E9495
:105ED000CF78F50160837183828393830F5F1F4FB7
:105EE000F4E0EF0EF11C0530110549F6CE010196E4
:105EF0000E94737AB0C1113939F58091F6059091FD
:105F0000F705039708F4A7C10E94BB260E94BB2691
:105F1000182F0E94BB264091EF055091F00560912B
:105F2000F1057091F2054F5F5F4F6F4F7F4F4093C8
:105F3000EF055093F0056093F1057093F205682F1B
:105F4000812F0E94498087C11239A9F58091F605F9
:105F50009091F705069708F47EC10E94BB260E9427
:105F6000BB26182F0E94BB268FAB0E94BB268EAB90
:105F70000E94BB26082F0E94BB26C090EF05D09040
:105F8000F005E090F105F090F2052FEFC21AD20A69
:105F9000E20AF20AC092EF05D092F005E092F10514
:105FA000F092F205802F0E94B78A4EA96FA9812F27
:105FB0000E94088A50C1133951F58091F6059091DD
:105FC000F705069708F447C10E94BB260E94AD263C
:105FD0008C010E94AD267C010E94BB264091EF05FA
:105FE0005091F0056091F1057091F2054F5F5F4FA0
:105FF0006F4F7F4F4093EF055093F0056093F1058D
:106000007093F205B701C8010E94754B24C118387E
:10601000D9F58091F6059091F705049708F41BC116
:106020008091F8059091F9052091F6053091F705DA
:1060300003966091F4057091F5050E944DD8E091AA
:10604000FA05F091FB05E80FF91F808190E00496B6
:106050002817390708F4FFC00E94BB268091EF057E
:106060009091F005A091F105B091F2050196A11D66
:10607000B11D8093EF059093F005A093F105B093C7
:10608000F2050E94BF26E7C0163931F58091F6056A
:106090009091F705039708F4DEC00E94BB260E948A
:1060A000BB26182F0E94BB264091EF055091F005AA
:1060B0006091F1057091F2054F5F5F4F6F4F7F4F19
:1060C0004093EF055093F0056093F1057093F2054E
:1060D000812F0E94B3A3BFC0173911F58091F60537
:1060E0009091F705029708F4B6C00E94BB260E9463
:1060F000BB264091EF055091F0056091F10570913C
:10610000F2054F5F5F4F6F4F7F4F4093EF05509306
:10611000F0056093F1057093F2050E94DC4B9BC083
:10612000183931F58091F6059091F705029708F43A
:1061300092C00E94BB260E94BB268091EF059091E1
:10614000F005A091F105B091F2050196A11DB11DD8
:106150008093EF059093F005A093F105B093F205BD
:106160000E944C3460E08CEC98E00E94534873C06D
:10617000193931F58091F6059091F705059708F4E6
:106180006AC00E94BB260E9488268091EF059091EC
:10619000F005A091F105B091F2050196A11DB11D88
:1061A0008093EF059093F005A093F105B093F2056D
:1061B00084EF95E00E94B03A81E08093B3054BC034
:1061C0001A3911F58091F6059091F705029708F4B8
:1061D00042C00E94BB260E94BB264091EF05509111
:1061E000F0056091F1057091F2054F5F5F4F6F4FC1
:1061F0007F4F4093EF055093F0056093F105709346
:10620000F2050E94C93B27C01C3929F58091F6058B
:106210009091F7050297F8F00E94BB260E94BB26DA
:106220004091EF055091F0056091F1057091F205F4
:106230004F5F5F4F6F4F7F4F4093EF055093F005D7
:106240006093F1057093F20591E0813009F090E0E0
:10625000892F0E9454808091EF059091F005A091C4
:10626000F105B091F20581309A4CAA49BB4308F47C
:1062700015C181E09AECAAE9BBE38093EF05909306
:10628000F005A093F105B093F20508C10E94674E96
:10629000811129C00C940C288091E6059091E705A6
:1062A000A091E805B091E9050196A11DB11D80936B
:1062B000E6059093E705A093E805B093E9050E94F1
:1062C0006A4E682F84EF95E00E943B260C94F827D5
:1062D0008091E5058F5F8093E505863010F40C947E
:1062E0008A280C9424280E94674E81110C948A28D5
:1062F0000C947C280E94794E0C948A280E94EC848D
:1063000081110C94B0280C94A2280E94FA84682F62
:1063100084EF95E00E943B260C948E280E945C85B9
:106320000C94B0288091F305813011F00C943D2934
:1063300083EA99E00C943F2987E00E94DC4B10929D
:10634000E4051092E3050C9455298091CF059091B6
:10635000D005029749F43CC880910402909105024F
:10636000009709F028C824C88091CF059091D005E6
:106370008330910509F066C855C80E94C6A383E022
:1063800090E09093D0058093CF0580910402909186
:106390000502019709F02CC820C8CE0145960E943D
:1063A000B8D28FE0FE017596A4EDB5E001900D9294
:1063B0008A95E1F710920502109204020E94C6A38A
:1063C00040E061E973E08CEC98E00E946D4364E189
:1063D00080E00E94498064E181E00E94498064E19C
:1063E00083E00E94498064E184E00E94498060E08B
:1063F00070E08CE099E00E9499A060E070E08CEB86
:1064000099E00E9499A060E070E08CEF9BE00E9410
:1064100099A044C08630910509F075C85DC8809187
:10642000040290910502019709F01CC823C881EB72
:106430009AE00E948AA71092D0051092CF05109280
:10644000EC052CC08091F6059091F705809708F433
:1064500002CF81C98091F6059091F705499708F41C
:10646000FACEC8C88091F6059091F7054A9708F4CE
:10647000F2CE14C98091F6059091F705029708F0C5
:10648000F0C9E9CE1D3909F0ADCA23CA8091F605DD
:106490009091F705029708F0C7C9DDCEE7960FB6D1
:1064A000F894DEBF0FBECDBFDF91CF911F910F914A
:1064B000FF90EF90DF90CF90BF90AF909F908F9024
:1064C0007F906F905F904F903F902F90089540E0A5
:1064D0006DE57AE18EEF97E00E944CD080E092E08B
:1064E0009093F5058093F4051092F7051092F60548
:1064F0001092F9051092F8058EEF95E09093FB0548
:106500008093FA051092FC051092FD0584ED95E04C
:106510000E94B8D285EB95E00C943C4C40E06DE5D0
:106520007AE18AE298E00E944CD084E098E00C94F2
:10653000C6CFCF93DF9300D0CDB7DEB721E029835C
:1065400022E32A8342E050E0BC01CE0101960E9482
:10655000E9DA0F900F90DF91CF910895CF93DF93F9
:10656000EC0140E050E060EE70E40E94239E46E6BD
:1065700056E666EA7EE3CE0102960E94239E40E044
:1065800050E060E172E4CE010496DF91CF910C946B
:10659000239E0F931F93CF93DF93EB018B01085E34
:1065A0001F4F892B31F467E0CE010E94F3DA6CE0D3
:1065B00005C068E3CE010E94F3DA60E2C8010E94E0
:1065C000F3DACE010A960E94AE32CE0140960E94C6
:1065D000AE32CE014A960E94993264EF71E0CE014C
:1065E00006960E9409DB65E070E0CE0102960E94EB
:1065F00009DB64EF71E0CE0104960E9409DB6CE2D6
:1066000071E0CE010896DF91CF911F910F910C940C
:1066100009DB0F931F93CF93DF9300D01F92CDB769
:10662000DEB78C0160E00E94F3DA61E0C8010296F7
:106630000E94F3DA8FEF89831B821A82B8016C5FA4
:106640007F4F43E050E0CE0101960E94E9DA0F90BF
:106650000F900F90DF91CF911F910F910895FF92AE
:106660000F931F93CF93DF9300D000D0CDB7DEB749
:10667000F82E062F1FB7F89468E080E491E04C8371
:106680000E94F3DAF9820A834C814B8343E050E0A5
:1066900064E471E0CE0101960E94E9DA1FBF0F9019
:1066A0000F900F900F90DF91CF911F910F91FF905E
:1066B000089561E00C94F3DACF93DF93EC0166EE7A
:1066C00070E00E9409DB66EE70E0CE0102960E9447
:1066D00009DB6EE670E0CE0104960E9409DB65E0FE
:1066E000CE010696DF91CF910C94F3DA61E08EE64D
:1066F00091E00E94F3DA68EE73E082E791E00E9495
:1067000009DB68EE73E084E791E00E9409DB66E94B
:1067100070E086E791E00E9409DB60EA7FE088E7AD
:1067200091E00E9409DB60EA7FE08AE791E00E9445
:1067300009DB60ED77E080E791E00E9409DB60EA29
:106740007FE086E891E00E9409DB6AE070E08CE778
:1067500091E00E9409DB6AE070E08EE791E00E9420
:1067600009DB6AE070E080E891E00E9409DB6EE1FD
:1067700070E082E891E00E9409DB6EE170E084E85D
:1067800091E00E9409DB42E553E060E070E088EDB3
:1067900091E00E9401DB44E853E060E070E08CEDA2
:1067A00091E00E9401DB60E070E080EE91E00E94E9
:1067B00009DB60E070E082EE91E00E9409DB61E0BD
:1067C00084EE91E00E94F3DA60E888E891E00C94AE
:1067D000F3DACF93CFB7F89440E150E062E270E093
:1067E00089EF92E00E94E9DACFBFCF91089561E08E
:1067F00082E490E00E94729D91E0813009F090E087
:10680000892F08951F93CF93DF93CDB7DEB7649799
:106810000FB6F894DEBF0FBECDBF84E1EBEBF2E024
:10682000DE01119601900D928A95E1F70E94F733EF
:10683000882381F088E990E0A0E0B0E089839A8322
:10684000AB83BC8388E490E0A0E0B0E08D839E83BE
:10685000AF83B8871FB7F89444E150E064E272E078
:10686000CE0101960E94E9DA1FBF64960FB6F89434
:10687000DEBF0FBECDBFDF91CF911F910895CF93A3
:10688000CFB7F894682F82E490E00E94F3DA0E9478
:106890000234CFBFCF9108951F93CF93DF93CDB72D
:1068A000DEB729970FB6F894DEBF0FBECDBF85E0E7
:1068B000EFECF2E0DE01119601900D928A95E1F77E
:1068C0000E94E9331FB7F89481EC93E29F838E8393
:1068D00084E193ED9987888745E050E066E070E0B9
:1068E000CE0101960E94E9DA6FE984E090E00E940F
:1068F000F3DA6BE18CE090E00E94F3DA60E084E48C
:1069000092E00E94F3DA0E94023460E080E592E0B7
:106910000E94F3DA44E150E060E172E088E093E045
:106920000E94E9DA44E150E064EA71E08CE193E02E
:106930000E94E9DA4AE050E066E472E080E393E026
:106940000E94E9DA0E94763360E070E080EA91E02C
:106950000E9409DB60E082EA91E00E94F3DA61E0E4
:1069600080E691E00E94F3DA88E591E00E945C33D2
:1069700044E050E064E470E0CE0106960E94E9DA5B
:1069800060E071E080E090E00E94C9326CE171E06B
:1069900081E090E00E94C93280E491E00E940933D6
:1069A0008AE491E00E94593360E086E591E00E941C
:1069B000F3DA1FBF29960FB6F894DEBF0FBECDBF26
:1069C000DF91CF911F91089561E08CE490E00E94E7
:1069D000729D91E0813009F090E0892F0895CF9366
:1069E000CFB7F89480E491E00E9409338AE491E003
:1069F0000E94593388E591E00E945C3361E080E6B3
:106A000091E00E94F3DA61E08EE691E00E94F3DA11
:106A100081E00E943F3460E084E492E00E94F3DA77
:106A200060E080E592E00E94F3DA61E08CE490E0BF
:106A30000E94F3DACFBFCF9108951F93CF93DF93D6
:106A4000CDB7DEB72C970FB6F894DEBF0FBECDBF23
:106A50001FB7F89488EE90E8A0E0B0E089839A83AD
:106A6000AB83BC831D821E821F82188619861A86FC
:106A70001B861C864CE050E068E372E0CE01019674
:106A80000E94E9DA1FBF2C960FB6F894DEBF0FBE46
:106A9000CDBFDF91CF911F910895FF920F931F9368
:106AA000CF93DF93F82E162F60E070E080EA91E03C
:106AB0000E948F9DEC0160E082EA91E00E94729D4D
:106AC000282F210F822F6CE30E9441D8092F2D33EC
:106AD00008F021961FB7F894BE016F0D711D80EA72
:106AE00091E00E9409DB602F82EA91E00E94F3DAD4
:106AF0001FBFDF91CF911F910F91FF9008951F93BA
:106B0000CF93DF9300D01F92CDB7DEB70E944C34F5
:106B100019821A821B821FB7F89467E182E090E025
:106B20000E94F3DA61E082E490E00E94F3DA0E94CE
:106B30001D3561E08CE490E00E94F3DA61E088E0CA
:106B400092E00E94F3DA43E050E06AE072E0CE01A6
:106B500001960E94E9DA61E78EE092E00E94F3DAA2
:106B60001FBF0F900F900F90DF91CF911F9108954D
:106B70001F93CF93DF93CDB7DEB727970FB6F89467
:106B8000DEBF0FBECDBF1D821E821F821FB7F894CD
:106B900044E150E060E172E088E093E00E94E9DACD
:106BA00044E150E064EA71E08CE193E00E94E9DAAC
:106BB0004AE050E066E472E080E393E00E94E9DAA4
:106BC0000E9476330E94023461E088E092E00E94E5
:106BD000F3DA43E050E06AE072E0CE0105960E94ED
:106BE000E9DA61E78EE092E00E94F3DA1FBF40E04D
:106BF00050E0BA0182E691E00E94B29D60392CEB30
:106C0000720725E5820728EA9207A8F4A4E6B0E017
:106C10009B01AC010E94CCD828E335E74CE955E054
:106C20000E9475D828513F474F4F5F4F29833A83C1
:106C30004B835C830EC028E335E74CE955E00E94A6
:106C400075D8A4E6B0E00E94CCD869837A838B83A0
:106C50009C830E941D351FB7F89444E050E068E320
:106C600072E0CE0101960E94E9DA1FBF27960FB6A7
:106C7000F894DEBF0FBECDBFDF91CF911F91089575
:106C800040E06DE57AE180E398E00C944CD0CF923F
:106C9000DF92EF92FF920F931F93CF93DF93EC015C
:106CA0008B018881811102C080E048C0DC2ECD2E8E
:106CB00060E0CE010E94A7CF87FFF6CF0E94FD4D76
:106CC000882329F0CE010E94004E61E828C00E946E
:106CD000FA4D811123C00E94E38481111FC02091CD
:106CE00051083091520824303105F1F417C06C2F4F
:106CF0008D2D9C2D0E94A7CF0E945C26219603C05B
:106D0000C0E0D0E07901CE15DF058CF361E801C069
:106D100062E8C8010E94FDCF789404C06AE8C80107
:106D20000E94FDCF81E00AC0F894C8810E942E2302
:106D30002C2F30E08217930718F7EACFDF91CF911D
:106D40001F910F91FF90EF90DF90CF90089586E014
:106D500090E0909352088093510881E08093360828
:106D60000895CF93DF93EB0161E00E94ACCF61E81F
:106D70004A9730F4CE010E94FDCF60E070E005C07C
:106D8000CE010E94FDCF60EC72E0CE01DF91CF9189
:106D90000C94FFCFCF93DF93EB0161E00E94ACCF67
:106DA00061E8CE010E94FDCF60EC72E0CE010E944E
:106DB000FFCF60E070E0CE010E94FFCF61E0CE0126
:106DC0000E94FDCF60E0CE010E94FDCF60E070E048
:106DD000CE01DF91CF910C94FFCFEF92FF920F93F2
:106DE0001F93CF93DF938B0161E8C8010E94FDCF11
:106DF000C3E5D8E07E016991C8010E94FDCFF7018B
:106E00008081882321F0F8E0C237DF0799F7DF910E
:106E1000CF911F910F91FF90EF900895CF93DF9343
:106E2000EB0161E8CE010E94FDCF0E942E23AC0150
:106E300060E070E0CE01DF91CF910C9414D00F93FD
:106E40001F93CF93DF93CDB7DEB764970FB6F89457
:106E5000DEBF0FBECDBF8B01F894CE0101960E941C
:106E6000647B61E8C8010E94FDCF60E070E0CE0164
:106E700001960E94714CFC014081518162817381B5
:106E8000C8010E9414D061E070E0CE0101960E941A
:106E9000714CFC014081518162817381C8010E9463
:106EA00014D062E070E0CE0101960E94714CFC01AA
:106EB0004081518162817381C8010E9414D00E9477
:106EC0006680682FC8010E94FDCF789464960FB643
:106ED000F894DEBF0FBECDBFDF91CF911F910F9110
:106EE00008950F931F93CF93DF93CDB7DEB76497C9
:106EF0000FB6F894DEBF0FBECDBF8B01F894CE0164
:106F000001960E94647B61E8C8010E94FDCF60E0A9
:106F100070E0CE0101960E94714CFC0140815181CC
:106F200062817381C8010E9414D061E070E0CE01DB
:106F300001960E94714CFC014081518162817381F4
:106F4000C8010E9414D062E070E0CE0101960E9458
:106F5000714CFC014081518162817381C8010E94A2
:106F600014D063E070E0CE0101960E94714CFC01E8
:106F70004081518162817381C8010E9414D064E014
:106F800070E0CE0101960E94714CFC01408151815C
:106F900062817381C8010E9414D00E946680682FAC
:106FA00070E0C8010E94FFCF789464960FB6F89401
:106FB000DEBF0FBECDBFDF91CF911F910F9108951E
:106FC0000F931F93CF93DF938C01EB0161E8CE0108
:106FD0000E94FDCFC80103960E94404F682FCE014A
:106FE000DF91CF911F910F910C94FDCFCF93DF9341
:106FF000EB0161E8CE010E94FDCF0E94284EAB015B
:10700000BC01CE010E9414D0DF91CF910C948A4E26
:107010008F929F92AF92BF92CF92DF92EF92FF92A8
:107020000F931F93CF93DF93CDB7DEB77C018B0116
:10703000CDB6DEB69EB6BDB6AEB661E8C8010E945A
:10704000FDCF61E0C7010E94A7CF882379F00E949D
:107050007F4F009759F0682FC8010E94FDCF60E074
:10706000C8010E94FDCF3C2D292D2FC08DB79EB7A2
:107070004F970FB6F8949EBF0FBE8DBFEDB6FEB60C
:10708000EFEFEE1AFE0A40E050E06FE1C7010E9408
:10709000FE4CF7012081222321F0009711F42E32BB
:1070A00091F3682FC8010E94FDCF912CE92DF0E0EB
:1070B0008FE1981629F0EE0DFF1D608161110DC062
:1070C00060E0C8010E94FDCF9501832F922F0FB67B
:1070D000F8949EBF0FBE8DBF05C0C8010E94FDCFB2
:1070E0009394E4CF0FB6F894DEBE0FBECDBEDF9111
:1070F000CF911F910F91FF90EF90DF90CF90BF90B5
:10710000AF909F908F900895CF93DF93EB0161E84C
:10711000CE010E94FDCFF8940E944D63882351F068
:107120000E944923882331F061E0CE010E94FDCF07
:10713000789402C060E0F9CFDF91CF9108957F92FB
:107140008F929F92AF92BF92CF92DF92EF92FF9277
:107150000F931F93CF93DF93CDB7DEB78C015B0105
:107160008DB69EB661E00E94ACCF7C0163E0C801A1
:107170000E94A7CFC82ED12C2DB73EB72C193D09A0
:107180000FB6F8943EBF0FBE2DBF0DB71EB70F5FF1
:107190001F4F7FB6F894482F50E0B701C8010E94F6
:1071A000D3DA7FBE61E8C5010E94FDCF780106C039
:1071B000F80161918F01C5010E94FDCFC8018E19B0
:1071C0009F098C159D05A4F30FB6F8949EBE0FBEC3
:1071D0008DBEDF91CF911F910F91FF90EF90DF90C7
:1071E000CF90BF90AF909F908F907F9008952F92F7
:1071F0003F924F925F926F927F928F929F92AF9247
:10720000BF92CF92DF92EF92FF920F931F93CF9393
:10721000DF931F92CDB7DEB7882E792E6B012DB686
:107220003EB661E00E94ACCF582E692E63E0882DF7
:10723000972D0E94A7CF982EA82EB12C8DB79EB760
:107240008A199B090FB6F8949EBF0FBE8DBF0DB76C
:107250001EB70F5F1F4FFFB6F894402E1983492DBC
:1072600050E0652D762DC8010E94D3DAFFBE78016B
:1072700000E010E00BC0602F6C5F882D972D0E94FE
:10728000A7CFF70181937F010F5F1F4F0A151B05E1
:1072900094F31FB7F894492D50E0652D762D842D79
:1072A00099810E94E9DA1FBF61E8C6010E94FDCF03
:1072B000692DC6010E94FDCF0FB6F8943EBE0FBEE9
:1072C0002DBE0F90DF91CF911F910F91FF90EF9006
:1072D000DF90CF90BF90AF909F908F907F906F90F6
:1072E0005F904F903F902F9008950F931F93CF93EF
:1072F000DF931F92CDB7DEB78B0161E00E94A7CF6D
:1073000080FF04C089830E943281898181FD0E94AF
:10731000522361E8C8010E94FDCF60E0C8010F90D0
:10732000DF91CF911F910F910C94FDCFCF93DF93FD
:10733000EC0161E80E94FDCF60917C0CCE01DF91F1
:10734000CF910C94FDCF0F931F93CF93DF93809138
:107350007208882329F080917208882389F01DC063
:1073600002E718E0C2E2D0E060E0CE010E94729D28
:10737000F80181938F012196C233D105A9F7EBCF94
:10738000E9E9F4E0A2E7B8E084918D93319684E0D6
:10739000E73AF807C9F71092800882E798E0DF9192
:1073A000CF911F910F91089583E598E00895809102
:1073B0005108909152080895CF93DF9381EB9AE0A2
:1073C0000E9458A483E598E00E94024FEC010097C8
:1073D00081F40E9452230E9432810E9442818CECEF
:1073E00098E00E948C4282E090E090935208809353
:1073F0005108CE01DF91CF910895CF92DF92EF92A5
:10740000FF920F931F93CF93DF938C017B0161E871
:10741000C7010E94FDCF83E5C82E88E0D82EC1E0C9
:10742000D0E008C06C2FC8010E94A7CFF60181935D
:107430006F012196F801808190E0C817D90794F375
:10744000109271080E94DC39682FC701DF91CF913B
:107450001F910F91FF90EF90DF90CF900C94FDCF94
:107460000E9417858823B9F085E090E09093520838
:107470008093510881EB9AE00E944FA441E064E0C0
:1074800070E08CEC98E00E948B430E9452230E9493
:1074900032810C9442810895CF93C82F0E944323D8
:1074A000C817C9F08C2F0E943C23CC2341F083E005
:1074B00090E09093500880934F0861E007C081E00E
:1074C00090E09093500880934F0860E089E398E043
:1074D000CF910C9412D3CF910895CF93DF93EB010A
:1074E0000E94432391E089270E944C3A61E8CE0133
:1074F000DF91CF910C94FDCF1F93CF93DF93182F83
:10750000EB010E9446231817E1F0112341F025E01A
:1075100030E03093500820934F0861E007C021E02D
:1075200030E03093500820934F0860E089E398E002
:107530000E9412D3BE01812FDF91CF911F910C9435
:10754000E125DF91CF911F91089540E054EA63E96E
:1075500076ED89E398E00E94BCD210924808089525
:10756000CF92DF92EF92FF920F931F93CF93DF930F
:10757000CDB7DEB76F970FB6F894DEBF0FBECDBFA5
:10758000FC0180915108909152088130910509F4D5
:107590004DC024F4892B09F443C075C08230910595
:1075A00021F0059709F06FC041C09E012F5F3F4F4A
:1075B0006E0180E2C80ED11C41E082819381892B4B
:1075C00019F4418780E01AC084819581E080F180C0
:1075D000B7010E944DD806811781080F191F8481B9
:1075E00095810196B7010E944DD89583848382814D
:1075F0009381019793838283D8018C91D9018D93D4
:107600009D01882309F44AC0AC15BD05B1F646C0FA
:10761000BE016F5F7F4F83E598E00E94A4DA33C01C
:1076200081E090E0909352088093510823E538E080
:1076300041E082819381892B19F4418780E01AC04F
:1076400084819581E080F180B7010E944DD8068148
:107650001781080F191F848195810196B7010E9437
:107660004DD895838483828193810197938382830C
:10767000D8018C91D9018D939D01882321F0B8E028
:1076800022373B07B1F60E94A53A0E94902381E081
:1076900090E09093500880934F0809C06AE373E02C
:1076A000CE0101960E949BDA009769F3B1CF6F96E5
:1076B0000FB6F894DEBF0FBECDBFDF91CF911F9103
:1076C0000F91FF90EF90DF90CF90089589E398E0BD
:1076D0000E94E0D2882369F040E054EA63E976ED45
:1076E00089E398E00E94BCD2809148088F5F809324
:1076F00048080895CF93DF93EB01209139082111B9
:1077000008C020914E08FC01208380914D08888399
:107710000FC020914808FC01208389E398E00E9473
:1077200041D320E037E843E953E00E9475D828832D
:10773000DF91CF910895CF93DF93CDB7DEB72F9729
:107740000FB6F894DEBF0FBECDBF6DE478E08EE4D7
:1077500098E00E947A3B60914D0880914E080E940B
:107760004D35CE0101960E94B8D28FE0FE013196D0
:10777000A9E3B8E001900D928A95E1F710924808CC
:107780002F960FB6F894DEBF0FBECDBFDF91CF911D
:107790000895CF93DF9300D000D000D0CDB7DEB7EF
:1077A00061E070E081EB9AE00E94BFA40E949B3BE5
:1077B0000E9487236093490870934A0880934B087E
:1077C00090934C0882E090E09093500880934F088B
:1077D000109252081092510860E083E00E943080BD
:1077E00060E084E00E94308045E06FE57AE1CE0100
:1077F00001960E944CD060E0CE0101960E949BD081
:1078000026960FB6F894DEBF0FBECDBFDF91CF91A5
:1078100008950F931F93CF93DF93CDB7DEB766978D
:107820000FB6F894DEBF0FBECDBF80915108909186
:1078300052080197029708F073C00E94328160E0FD
:1078400083E00E94308060E084E00E94308041E06C
:1078500060E270E08CEC98E00E948B430E948723EA
:107860006093490870934A0880934B0890934C08A2
:107870000E949B3B62E070E081E00E94E125BE0136
:107880006B5E7F4FCE0146960E947A3B0E942D840C
:10789000182F882309F444C0CE0101960E94D07AA3
:1078A00062E070E0CE010196113059F40E94794CEB
:1078B0008C0182E00E94A07820E030E041E153E4B6
:1078C0000AC00E94794C8C0182E00E94A07820E0DE
:1078D00030E046E153E40E94CED70E9497D6F801EB
:1078E000608371838283938380E00E943C2346E916
:1078F00050E060E070E0CE0101960E94FA7B68EAF9
:1079000074E081EB9AE00E9403A581E08093E50B8F
:1079100040E856E968E970E082E898E00E94BCD24D
:1079200080915108909152080197B9F480914F08C5
:1079300090915008049789F084E090E09093520869
:107940008093510881E08093360840E452E46FE070
:1079500070E081E998E00E94BCD280E00E94B4759A
:1079600040E064E070E08CEC98E00E948B4381E0A2
:107970008093380884E090E09093500880934F08FB
:1079800066960FB6F894DEBF0FBECDBFDF91CF91E4
:107990001F910F9108950F931F93CF93DF9300D002
:1079A000CDB7DEB78C0161E80E94FDCFBE016F5FED
:1079B0007F4FCE0102960E947A3B60914F08C8012A
:1079C0000E94FDCF6A81C8010E94FDCF6981C80174
:1079D0000E94FDCF80914F08909150088130910511
:1079E00029F08330910511F0059729F40E9487232F
:1079F000AB01BC0108C04091490850914A08609110
:107A00004B0870914C08C8010E9414D040E050E02F
:107A1000BA01C8010E9414D00F900F90DF91CF914E
:107A20001F910F910895EF92FF920F931F93CF93A1
:107A3000DF937C01EB01FC018081882309F4F2C013
:107A400061E0C7010E94A7CF082F62E0C7010E9432
:107A5000A7CF803209F446C060F4823001F118F4F7
:107A60008823B1F0DFC0863139F18E3109F0DAC0F8
:107A700030C0833209F44CC020F4813209F0D2C006
:107A80003EC0843209F44EC0853209F0CBC082C0BA
:107A900061E8CE010E94FDCF60EC72E0BEC061E8FB
:107AA000CE010E94FDCF013019F483EA99E002C0B3
:107AB00083EF98E0499613C061E8CE010E94FDCFA4
:107AC000013019F483EA99E002C083EF98E0499607
:107AD00025C061E8CE010E94FDCF8CEF9BE00E94A3
:107AE00075A19AC061E8CE010E94FDCF013019F462
:107AF00083EA99E002C083EF98E0499606C061E806
:107B0000CE010E94FDCF8CEF9BE00E946FA184C04C
:107B100061E8CE010E94FDCF8CEF9BE00E944BA15B
:107B2000682F34C061E8CE010E94FDCF013019F406
:107B300083EA99E002C083EF98E049960E947DA312
:107B4000882311F010E801C010E08CEF9BE00E9448
:107B50007DA3882311F080E401C080E0182B013060
:107B600019F483EA99E002C083EF98E049960E94F5
:107B700082A3182B013019F483EA99E002C083EF45
:107B800098E049960E944BA1612F682BCE010E947C
:107B9000FDCF46C061E8CE010E94FDCF013019F44F
:107BA00083EA99E002C083EF98E049960E947AA1A7
:107BB000BC01CE010E94FFCF013019F483EA99E0A5
:107BC00002C083EF98E049960E947DA1BC01CE01DE
:107BD0000E94FFCF013019F483EA99E002C083EFDD
:107BE00098E049960E9480A1BC01CE010E94FFCF7F
:107BF0008CEF9BE00E947AA1BC01CE010E94FFCFD6
:107C00008CEF9BE00E947DA1BC01CE010E94FFCFC2
:107C10008CEF9BE00E9480A1BC01CE010E94FFCFAF
:107C200081E001C080E0DF91CF911F910F91FF9023
:107C3000EF9008950F931F93CF93DF938C01EB0187
:107C4000FC018081811101C08FC060E0C8010E94E9
:107C5000A7CF87FD89C0E82FF0E0EC31F10508F0EF
:107C600083C0EE58FF4F0C94B3D8BE01C8010E94E8
:107C7000B13678C0BE01C8010E94ED3673C0809154
:107C80005108909152089C01215031092230310550
:107C900010F0059779F484E090E090935008809379
:107CA0004F080E94093C64E070E08CEC98E00E9470
:107CB000204603C081E08093380861E8CE010E942D
:107CC000FDCF50C0BE01C8010E940E374BC0BE019F
:107CD000C8010E941F3746C0BE01C8010E9471370B
:107CE00041C0BE01C8010E94E0373CC0BE01C801CE
:107CF0000E94F63737C0BE01C8010E94FD3932C06C
:107D0000BE01C8010E9408382DC0BE01C8010E94F2
:107D10006D3A28C0BE01C801DF91CF911F910F912C
:107D20000C94133DBE01C8010E9484381BC0BE01E3
:107D3000C8010E949F3816C0BE01C8010E94F738D2
:107D400011C0BE01C8010E9475390CC0CE010E944D
:107D5000963908C0CE010E94CB3C04C0BE01C801C8
:107D60000E94CA3681E001C080E0DF91CF911F916F
:107D70000F910895CF93DF93CDB7DEB72F970FB64E
:107D8000F894DEBF0FBECDBF8091251D9091261DBA
:107D9000892B09F407C18091251D9091261D049718
:107DA00009F01BC1FFC080913608811106C0809187
:107DB0008208882309F4FBC007C081E998E00E948B
:107DC000E0D28111F4CFFCC082E898E00E94E0D2BA
:107DD0008111EDC00E944D638111E9C0F1C0833073
:107DE000910511F0059741F484E090E090935008DC
:107DF00080934F080E94093C109238081092360870
:107E0000CE0101960E94B8D28FE0FE013196A1E921
:107E1000B8E001900D928A95E1F7CE0101960E949B
:107E2000B8D28FE0FE013196A2E8B8E001900D9241
:107E30008A95E1F7809137080E940D40109237082B
:107E4000CE0101960E94B8D28FE0FE013196A0EAE1
:107E5000B8E001900D928A95E1F7109272081092A5
:107E600053081092520810925108B7C08091FF1C1D
:107E70009091001D049709F0ABC016C040E45DE08E
:107E800063E070E080EA98E00E94BCD20DC080EA16
:107E900098E00E94E0D2882339F08CED9CE10E94AA
:107EA00046CF84E08093FE1C8091FE1C882321F045
:107EB0008CED9CE10E9454CF8091FF1C9091001D9D
:107EC000049709F049C080EA98E00E940CD382E050
:107ED0009DE10E94BECF809151089091520820915F
:107EE0003608069761F4222341F069E882E09DE1BB
:107EF0000E94FDCF1092360827C06BE821C02223D4
:107F000071F069E882E09DE10E94FDCF1092360891
:107F100066E070E08CEC98E00E94204615C062E0BC
:107F20007DE18CED9CE10E94473681110DC062E03D
:107F30007DE18CED9CE10E941A3E811105C065E84F
:107F400082E09DE10E94FDCF8CED9CE10E9454CF28
:107F500088ED9CE10E9497D380915108909152083E
:107F6000029741F40E94FA4D811104C01092520808
:107F7000109251088091510890915208059779F418
:107F80000E94E384811104C010925208109251089B
:107F900040E064E070E08CEC98E00E948B430E942B
:107FA000663B1BC0809138088111FDCE09C08091CD
:107FB0004F08909150088130910509F010CF14CFEF
:107FC0008091FF1C9091001D892B09F04FCF6CCF41
:107FD0008091A00881115BCF51CF2F960FB6F894F6
:107FE000DEBF0FBECDBFDF91CF91089540E06DE5BC
:107FF0007AE18FEA98E00E944CD080EA98E00E94F3
:10800000B8D281E998E00E94B8D282E898E00E9454
:10801000B8D289E398E00C94B8D2CF93DF931F9243
:10802000CDB7DEB7F89494B78823A1F098E10FB6E6
:10803000F89490936000109260000FBE14BE99E215
:1080400028E130E00FB6F894A895209360000FBEA9
:108050009093600089830E948A4E0E94844A0E9405
:10806000E6840E9452230E943C9D0E94CF790E9488
:1080700032810E9442818981682F8CEC98E00E94B5
:10808000534878940F90DF91CF9108958CEC98E04D
:108090000E94DF4181E00E940D4078940E94BA3E28
:1080A0000E94D9278CEC98E00E9497460E94CC4B06
:1080B000A895F4CF40E06DE57AE185EB98E00C946B
:1080C0004CD00F931F93CF93DF9300D000D000D0FC
:1080D000CDB7DEB7062F1FB7F89444E06FE57AE11D
:1080E000CE0101960E944CD061E0011101C060E018
:1080F000CE0101960E949BD01FBF26960FB6F89422
:10810000DEBF0FBECDBFDF91CF911F910F910895BC
:10811000CF93DF9300D000D000D0CDB7DEB7109260
:10812000C3081092C20845E06FE67AE1CE010196DD
:108130000E944CD060E0CE0101960E949BD046E0A8
:108140006FE67AE1CE0101960E944CD060E0CE014C
:1081500001960E949BD026960FB6F894DEBF0FBE04
:10816000CDBFDF91CF9108956F927F928F929F92B2
:10817000AF92CF92EF92FF920F931F93CF93DF9323
:10818000CDB7DEB762970FB6F894DEBF0FBECDBF96
:108190004C0104960E94B8D2C40143960E94B8D202
:1081A00043E06BE67AE1CE0101960E944CD044E0B8
:1081B00065E67AE1CE0107960E944CD043E065E681
:1081C0007AE1CE010D960E944CD0E12CFF24F3946D
:1081D0008E010F5F1F4F9E01295F3F4FAE01435F2E
:1081E0005F4F60E0C40187960E943B8744E06BE6E6
:1081F0007AE1C8010E944CD046E061E77AE1CE0105
:1082000007960E944CD045E061E77AE1CE010D96D9
:108210000E944CD09CE1E92EFF24F3948E010F5F65
:108220001F4F9E01295F3F4FAE01435F5F4F61E0EB
:10823000C40189529F4F0E943B87C40189579E4FBA
:108240000E94B8D2C4018A569E4F0E94B8D28401BF
:108250000B551E4FC80102960E94B8D2C801419624
:108260000E94B8D242E06FE67AE1CE0101960E9408
:108270004CD043E06FE67AE1CE0107960E944CD0E5
:1082800044E06FE67AE1CE010D960E944CD03401B5
:1082900087E3681A8EEF780A9E012F5F3F4FAE0189
:1082A000495F5F4FBE01635F7F4FC3010E9403A818
:1082B000A301B801C4018B519E4F0E94DBA334017E
:1082C000E4EE6E1AECEF7E0A40E06FE0C3010E941C
:1082D000E6D1A401425D5C4F8BE493E0FA01918307
:1082E000808322E0A22EC12C30E1E32EFF24F39400
:1082F00000E513EC20E030E0B301C401805D9C4F49
:108300000E945A9F61E08CE490E00E94729DF4010B
:10831000E655FC4F91E0811101C090E09083629698
:108320000FB6F894DEBF0FBECDBFDF91CF911F9186
:108330000F91FF90EF90CF90AF909F908F907F9094
:108340006F9008950E94C94A109220018AE080939C
:1083500021011092220180E090E290932901809304
:10836000280182E0809373008093B00094E09093A2
:10837000B10099E19093B3001092B4008093700023
:1083800091E0909380008BE08093810010928900AF
:108390001092880010928B0010928A0010926F0049
:1083A0009093A0008093A1001092A9001092A800C1
:1083B0001092AB001092AA001092720008950F93D1
:1083C0001F93CF93DF9300D000D000D0CDB7DEB79E
:1083D0008C0180E29DE00E941E500E948EA3F80155
:1083E00086A31082118212821382C8010E94A241C8
:1083F00047E061E77AE1CE0101960E944CD061E04E
:10840000CE0101960E947BD041E06FE67AE1CE0179
:1084100001960E944CD061E0CE0101960E947BD073
:1084200040E06FE67AE1CE0101960E944CD061E017
:10843000CE0101960E947BD041E067E67AE1CE0151
:1084400001960E944CD061E0CE0101960E947BD043
:1084500047E061E77AE1CE0101960E944CD061E0ED
:10846000CE0101960E947BD040E067E67AE1CE0122
:1084700001960E944CD061E0CE0101960E947BD013
:1084800046E061E67AE1CE0101960E944CD061E0BF
:10849000CE0101960E947BD0C80182960E94E88698
:1084A00040E251EA67E070E0C80189579E4F0E94A0
:1084B000BCD2C80187960E94BF87C80189529F4FCE
:1084C0000E94BF8744E06FE57AE1CE0101960E94E9
:1084D0004CD061E0CE0101960E947BD0C801845E41
:1084E0009C4F0E94E0D1C801805D9C4F0E94669E17
:1084F00040E553EC60E070E0C8018A569E4F0E9450
:10850000BCD226960FB6F894DEBF0FBECDBFDF916A
:10851000CF911F910F9108951F93CF93DF93EC019B
:10852000FC01E055FC4F11E010830E94F733682FE7
:10853000CE0180519F4F0E948DA00E94E434682F8D
:108540006127CE01805D9C4F0E948DA0FE01E25408
:10855000FC4F4081518162817381CE0143960E941C
:10856000BCD20E94198AFE01E455FC4F1082FE0124
:10857000EE54FC4F11821082FE01EC54FC4F11822C
:108580001082FE01EA54FC4F11821082FE01EF546A
:10859000FC4F1082FE01E754FC4F1082FE01E654AE
:1085A000FC4F1082FE01E554FC4F1082C454DC4F96
:1085B0001882DF91CF911F9108950F931F934FB7AA
:1085C000F894FC0100811181228133814FBFB801F1
:1085D000C9011F910F9108950E94432381112DC05D
:1085E000809170008D7F80937000809173008D7FEB
:1085F0008093730078940E94F583F89480917000C2
:108600008260809370008091730082608093730019
:108610002091240130912501809128019091290118
:108620002817390750F081E090E09093290180935A
:10863000280110922501109224010895CF93DF9311
:10864000EC01FC01E255FC4F7183608362307105DF
:10865000E1F4805D9C4F0E947DA381111BC00E94AC
:10866000F7338823B9F0CE01805C9F4F0E947DA331
:108670008823A1F0CE0180519F4F0E947DA38111DC
:1086800009C00CC081E08093CB08C555DC4F81E068
:10869000888304C08091CB088823A1F3DF91CF9118
:1086A0000895CF93DF93EC0189E18093C7088FE0B1
:1086B0008093C60881E090E09093C3088093C2083D
:1086C0006FEFCE018B519E4F0E94C1A7C455DC4F66
:1086D00081E08883DF91CF9108950F931F93CF930B
:1086E000DF931F92CDB7DEB78C018B519E4F49832C
:1086F0000E9403A5C8010E94514380E00E94DC4B08
:10870000F801E355FC4F498140830F90DF91CF91F1
:108710001F910F910895FC01E055FC4F442321F077
:108720008081862B80830895609580816823608393
:108730000895CF93DF93EC01805C9F4F0E9483A14B
:1087400081110EC0CE0180519F4F0E9483A18111E3
:1087500007C0CE01805D9C4FDF91CF910C9483A127
:1087600081E0DF91CF910895FC01E754FC4F31E0A7
:108770003083FC01E654FC4F6083FC01E554FC4F60
:108780004083FC01E454FC4F2083FC01E354FC4F84
:1087900010820895EF92FF920F931F93CF93DF9370
:1087A000EC01FC01E754FC4F10828C0107531E4F73
:1087B000FC01E654FC4F7C0185E4E81A8CEFF80AD2
:1087C0004081F7016081C8010E948BAAF701F08007
:1087D000C454DC4F06C065E473E0C8010E9486A95A
:1087E000F3948881F816B8F3DF91CF911F910F9120
:1087F000FF90EF9008959F92AF92BF92CF92DF9239
:10880000EF92FF920F931F93CF93DF93EC01D62E3D
:10881000142FC22E241708F478C030E0241B31092D
:10882000802F90E0281739070CF46FC0FE01EA543E
:10883000FC4F6081718116161706F4F4FE01EC54AA
:10884000FC4FCE018E549C4F0190F081E02DDC0155
:108850008D919C91E81BF90BF7FF03C0F195E19511
:10886000F109E29FC001E39F900DF29F900D11244A
:108870000E9461D8962E01C0912C9016A8F47E011A
:10888000B7E3EB1ABEEFFB0A4D2D612FC7010E9423
:108890008BAA012F06C065E473E0C7010E9486A978
:1088A0000F5F0C11F8CF00E07E0187E3E81A8EEF2E
:1088B000F80A602F610F4D2DC7010E948BAAC12CB1
:1088C000D12C10E0A92CB12C07C06FEFC7010E947A
:1088D000CEAAAFEFCA1ADA0A9601200F311F2A1565
:1088E0003B059CF3C854DC4F888191E0892788833D
:1088F000882331F061ED74E0C7010E949DA906C094
:108900006FEFC7010E94CEAA01C0912C892DDF9183
:10891000CF911F910F91FF90EF90DF90CF90BF907C
:10892000AF909F900895BF92CF92DF92EF92FF9207
:108930000F931F93CF93DF93EC018C010C541C4FCA
:10894000F80111821082FC01EA54FC4F118210825E
:108950007C01FEE4EF1AFCEFFF0AF701118210829E
:108960000E949943882309F4C5C06E01F0EDCF1A27
:10897000FCEFDF0AC6010E9483A18823D9F0C6015B
:108980000E94B9A1880F991FF70120813181280F1A
:10899000391F31832083C6010E946FA1880F991F60
:1089A000F80120813181280F391F3183208306EEA1
:1089B00010E01AC0FE01EA54FF4F8081882331F095
:1089C00060E0CE01805C9F4F0E94CFA1FE01EA597A
:1089D000FE4F8081882331F060E0CE0180519F4FAF
:1089E0000E94CFA100E010E07E01F0E4EF0EF11C48
:1089F000C7010E9483A1882339F0FE01EA54FF4F8A
:108A00008081882309F4A3C07E0180EFE80EF11C69
:108A1000C7010E9483A1882339F0FE01EA59FE4F65
:108A20008081882309F4AEC0FE01EC54FC4F8081A4
:108A30009181FE01EE54FC4F20813181FE01EA5408
:108A4000FC4F821793072CF4081B190B118300832A
:108A500002C09183808380819181892B09F455C064
:108A600061E082E491E00E94729D882309F44DC088
:108A700067E080E491E00E94729D873009F09DC01C
:108A800044C00E94158981E0F8018083FE01EE5404
:108A9000FC4FA081B181FE01EA54FC4FC080D1801F
:108AA000EE24D7FCE094FE2CFE01EC54FC4F008138
:108AB00011810A1B1B0B17FF03C0119501951109AA
:108AC0002FEF30E00E94C5D8A70196010E9497D8E9
:108AD000B22E2FEF30E0D8010E94C5D8A701960131
:108AE0000E9497D8E22F20E04B2D60E08E2F0E944D
:108AF00026890BC08E010F541C4FF80180818823FA
:108B000021F00E94198AF8011082FE01E754FC4FFF
:108B10008081882309F459C07E01F3E4EF1AFCEF49
:108B2000FF0ACE0184549C4FDE01A554BC4FBE0108
:108B300066547C4FF7010081FC0120814C91FB01C0
:108B40006081CE010E94FB43F70180833EC0C701D4
:108B50000E94B9A1FE01EE54FC4F20813181280F03
:108B6000391F31832083C7010E946FA1FE01EC549D
:108B7000FC4F20813181280F391F318320830A5116
:108B80001F4F42CFC7010E94B9A1FE01EE54FC4F16
:108B900020813181280F391F31832083C7010E9432
:108BA0006FA1FE01EC54FC4F20813181280F391F49
:108BB0003183208302591F4F37CF8E010F541C4F32
:108BC000F8018081811162CF5CCFDF91CF911F913D
:108BD0000F91FF90EF90DF90CF90BF90089540E00D
:108BE00052ED69E47BE643960C94BCD21F920F923F
:108BF0000FB60F9211240BB60F922F933F934F9302
:108C00005F936F937F938F939F93AF93BF93EF93F4
:108C1000FF938CEC98E00E94EC42FF91EF91BF91A2
:108C2000AF919F918F917F916F915F914F913F9104
:108C30002F910F900BBE0F900FBE0F901F901895A5
:108C40000F931F93CF93DF9300D000D000D0CDB708
:108C5000DEB78B016115710589F41092C508109279
:108C6000C40847E061E77AE1CE0101960E944CD04A
:108C700060E0CE0101960E949BD00CC08091C80894
:108C800090E08617970731F082E090E09093C50856
:108C90008093C4080093C80826960FB6F894DEBFE8
:108CA0000FBECDBFDF91CF911F910F910895CF934C
:108CB000DF9300D000D000D0CDB7DEB7411551050D
:108CC000E9F41092C3081092C20845E06FE67AE119
:108CD000CE0101960E944CD061E0CE0101960E9427
:108CE0009BD046E06FE67AE1CE0101960E944CD01F
:108CF00061E0CE0101960E949BD010C06115710504
:108D000019F40E9488400AC06093C7084093C608BF
:108D100081E090E09093C3088093C20826960FB636
:108D2000F894DEBF0FBECDBFDF91CF910895DF92E3
:108D3000EF92FF920F931F93CF93DF93EC018EA1DD
:108D4000811102C0D12C1CC08E010B511E4FC801D5
:108D50000E9431A47E0124E0E20EF11CC7010E94B2
:108D6000E0D2882379F3C8010E9418A6C8010E94A6
:108D700036A4AB01BC01C7010E94BCD2DD24D39450
:108D8000FE01E655FC4F8081882341F08E010A5692
:108D90001E4FC8010E94E0D281110EC17E0184E500
:108DA000E81A8CEFF80AF70180818823F9F08E0128
:108DB0000B511E4FC8010E94C6A78823B9F040E09E
:108DC00050E060E070E0CE010E9457460E94198A90
:108DD000F7011082C8010E94DFA5FE01E355FC4F98
:108DE000808181110E94093C1092C9088E010D5E9C
:108DF0001F4FC8010E94E0D2882309F44FC0FE0132
:108E0000E555FC4F8081811149C00E94D7390297F6
:108E100009F444C00E94D739019709F0DAC03EC076
:108E2000CE0180519F4F0E946FA11816190674F44D
:108E3000FE01E254FC4F80819181A281B381803494
:108E40009244AF40B10509F0D7C009C0CE01805DA2
:108E50009C4F0E946FA11816190654F309C0C8014F
:108E60000E9441D36115724D89449B4608F0C4C0ED
:108E700060E070E0C7010E9499A060E070E0CE0160
:108E800080519F4F0E9499A060E070E0CE01805D0C
:108E90009C4F0E9499A0C8010E940FD3FE01E55586
:108EA000FC4F8081882309F473C08091C908811127
:108EB0006FC00E94C94B81116BC0AFC06CEF74E0F2
:108EC00002C06DE475E0CE018B519E4F0E9403A558
:108ED00037C06EE975E0F7CF6FEE75E0F4CF40E094
:108EE00060E476E0CE010E946D438E01005C1F4F6E
:108EF000C8010E947DA3882329F060E070E0C801CA
:108F00000E9499A08E0100511F4FC8010E947DA3AD
:108F1000882329F060E070E0C8010E9499A08E01CA
:108F2000005D1C4FC8010E947DA3882329F060E0EA
:108F300070E0C8010E9499A0C555DC4F1882ABC0F3
:108F400060E070E0CE01805C9F4F0E9499A060E0DD
:108F500070E0CE0180519F4F0E9499A060E070E0C8
:108F6000CE01805D9C4F0E9499A080E00E94DC4B66
:108F70000E941A890E94A7360E943F230E943281D4
:108F800010E060E0812F0E9430801F5F1530C9F72C
:108F90008E0109571E4FC8010E94E0D2882309F4B0
:108FA00076C0D11074C061C0CE0189529F4F0E941B
:108FB000DF871092CA086FC0CE01805D9C4F0E946F
:108FC00058A240E553EC60E070E0C8010E94BCD2BA
:108FD000E5CEFE01E055FC4F80818E7F806480836A
:108FE0007E0180E4E80EF11CC7010E946FA11816F3
:108FF00019060CF41DCF14CF63ED74E0CE018B5134
:109000009E4F0E9403A5CE010E94514321E04FEFE5
:1090100060E080E00E9426892BCF81E08093C90820
:109020008AE08093C7088093C60881E090E090931F
:10903000C3088093C208FE01E255FC4F80819181F4
:109040008830910509F43DCF44F48230910509F44C
:1090500046CF049709F074CF31CF8031910509F4E0
:1090600038CF809709F06CCF37CFCE0187960E941A
:10907000DF87CE010E94934440E251EA67E070E04E
:10908000C8010E94BCD281E08093CA0804C08091CC
:10909000CA08811189CFDF91CF911F910F91FF9065
:1090A000EF90DF900895DF92EF92FF920F931F935E
:1090B000CF93DF9300D000D000D0CDB7DEB78C01C6
:1090C000D62E60E070E00E94204660E082E090E0F2
:1090D0000E94729D8095881F8827881F0E94F77BB9
:1090E00061E088ED9CE10E94B9D38CED9CE10E9487
:1090F00054CFF801108211821282138260E084E45E
:1091000092E00E94729DF801E254FC4FA82FB0E05B
:1091100020E037E843E953E00E94CCD8605C7D4B07
:10912000804F9F4F6083718382839383F80186A170
:10913000882309F45EC07801FBE1EF1AFEEFFF0A15
:10914000C7010E9453A545E06FE67AE1CE01019682
:109150000E944CD061E0CE0101960E947BD046E097
:109160006FE67AE1CE0101960E944CD061E0CE011B
:1091700001960E947BD045E06FE67AE1CE01019630
:109180000E944CD061E0CE0101960E949BD046E047
:109190006FE67AE1CE0101960E944CD061E0CE01EB
:1091A00001960E949BD060E086E591E00E94729D4E
:1091B000811103C065E070E002C064E070E0C701A7
:1091C0000E94BFA4DD2049F02FEF8BE792E92150E8
:1091D00080409040E1F700C00000C7010E94BAA3A0
:1091E000C7010E9436A4AB01BC01C80104960E94CD
:1091F000BCD240E050E060E070E0C8010E945746F9
:10920000DD2071F00E94BB8A83E00E94DC4BF801F4
:10921000E555FC4F1082F801E255FC4F1182108297
:10922000C8010E948C42F80186A1882341F060E0C9
:1092300086E591E00E94729D81110E94C6A3269648
:109240000FB6F894DEBF0FBECDBFDF91CF911F9157
:109250000F91FF90EF90DF9008951F920F920FB63D
:109260000F9211240BB60F922F933F934F935F935E
:109270006F937F938F939F93AF93BF93EF93FF93DE
:10928000CF93DF93CDB7DEB72697DEBFCDBF8091FA
:10929000CC089091CD08A091CE08B091CF088C5900
:1092A0009F4FAF4FBF4F8093CC089093CD08A093B2
:1092B000CE08B093CF080E942B848091BB08982FD2
:1092C0009F5F9093BB08853A08F4C3C01092BB0817
:1092D0008091C0089091C1081816190614F40197DE
:1092E0003AC08091C4089091C50881309105F1F48D
:1092F0008091BE089091BF0801969093BF0880931B
:10930000BE0882E090E09093C5088093C40882E193
:1093100090E09093C1088093C00847E061E77AE14C
:10932000CE0101960E944CD060E034C0823091059D
:10933000B9F48091C80890E02091BE083091BF0830
:10934000281739079CF083E090E09093C50880933C
:10935000C40880E590E09093C1088093C0081EC0C7
:109360000397E1F41092BF081092BE0881E090E0EC
:109370009093C5088093C40882E190E09093C1085F
:109380008093C00847E061E77AE1CE0101960E9430
:109390004CD061E0CE0101960E949BD08091BC0828
:1093A0009091BD081816190634F401979093BD08E2
:1093B0008093BC084EC08091C2089091C308813050
:1093C000910509F582E090E09093C3088093C2086C
:1093D0008091C7088093BC081092BD0845E06FE6F5
:1093E0007AE1CE0101960E944CD061E0CE01019657
:1093F0000E949BD046E06FE67AE1CE0101960E9482
:109400004CD061E022C0029721F581E090E090937A
:10941000C3088093C2088091C6088093BC0810924C
:10942000BD0845E06FE67AE1CE0101960E944CD07E
:1094300060E0CE0101960E949BD046E06FE67AE1A3
:10944000CE0101960E944CD060E0CE0101960E94B0
:109450009BD026960FB6F894DEBF0FBECDBFDF912E
:10946000CF91FF91EF91BF91AF919F918F917F919C
:109470006F915F914F913F912F910F900BBE0F9085
:109480000FBE0F901F90189586559C4FFC0160836E
:1094900008950F931F93CF93DF9300D000D000D097
:1094A000CDB7DEB7062F1FB7F89445E06FE57AE138
:1094B000CE0101960E944CD061E0CE0101960E943F
:1094C0007BD045E06FE57AE1CE0101960E944CD059
:1094D000602FCE0101960E949BD01FBF26960FB62B
:1094E000F894DEBF0FBECDBFDF91CF911F910F91DA
:1094F000089540E06DE57AE18EE89CE00E944CD052
:109500008CEC98E00C94B440CF93DF9300D000D063
:1095100000D0CDB7DEB761E08AE491E00E94729D91
:1095200091E0811101C090E09093EE0C1092970CA5
:109530001092960C1092990C1092980C10929C0C10
:1095400010929D0C8FEE9CE00E940FD31092FE0CA7
:1095500045E067E67AE1CE0101960E944CD061E0D9
:10956000CE0101960E947BD045E067E67AE1CE010C
:1095700001960E944CD060E0CE0101960E949BD0E3
:1095800026960FB6F894DEBF0FBECDBFDF91CF9108
:10959000089514BC15BC17BC18BC16BC10926E0004
:1095A0000895CF92DF92EF92FF92CF938091960C25
:1095B0009091970C892B39F48FEE9CE00E940FD389
:1095C0001092FE0C4BC021E02093FE0C8091960C73
:1095D0009091970C892B31F420939D0CC12CD12CA8
:1095E00076012EC08091980C9091990C2091940C4A
:1095F0003091950CB9010E944DD8880F991F880FA2
:10960000991FE0919A0CF0919B0CE80FF91F809143
:10961000980C9091990C0196B9010E944DD89093A5
:10962000990C8093980C8091960C9091970C0197CF
:109630009093970C8093960CC080D180E280F38049
:109640009701A8EEB3E00E94B9D8AB01BC018FEE40
:109650009CE00E94BCD2C601009739F4CF91FF90E4
:10966000EF90DF90CF900C94C94AA0E0B0E0823434
:109670002FE09207A105B10570F4883E21E0920722
:10968000A105B10558F48A379105A105B10548F047
:10969000C4E068E008C0C2E063E005C0C3E066E083
:1096A00002C0C5E06AE09C01AD01220F331F441FD8
:1096B000551F04C0220F331F441F551F6A95D2F750
:1096C00060E074E284EF90E00E9475D8215082E15E
:1096D00084BDC5BD27BD18BC16BC10926E00CF91CD
:1096E000FF90EF90DF90CF9008950F931F93CF934B
:1096F000DF938C01D62FC72F8091EE0C882309F4BD
:1097000043C06091940C7091950C4091960C5091CF
:10971000970C6417750771F14091960C5091970C56
:109720004617570720F54091960C5091970C809161
:10973000980C9091990C840F951F0E944DD8880F1A
:10974000991F880F991FE0919A0CF0919B0CE80FDC
:10975000F91F00831183D283C3838091960C90916B
:10976000970C01969093970C8093960C03C081E020
:1097700080939C0C8091FE0C811106C0DF91CF91EB
:109780001F910F910C94D14ADF91CF911F910F91AE
:1097900008958091FE0C08958091EE0C882359F075
:1097A0008091FE0C882339F08FEE9CE00E94E0D27D
:1097B00081110C94D14A0895FF920F931F93CF9378
:1097C000DF93883028F5E82FF0E0EE0FFF1FE35B12
:1097D000FC4F0081118101151105D1F0F12C24E01D
:1097E000F29EC0011124F801E80FF91F2591349170
:1097F000FC013296E00FF11FC591D491209721F022
:10980000BE01C9010E94754BF394CD2B41F70BC0EB
:1098100064EF71E08BE790E0DF91CF911F910F91A2
:10982000FF900C94754BDF91CF911F910F91FF909A
:10983000089540E06DE57AE18FEF9CE00E944CD006
:1098400084E190E09093950C8093940C1092970C87
:109850001092960C1092990C1092980C8EE99CE044
:1098600090939B0C80939A0C10929C0C10929D0CE0
:109870008FEE9CE00C94B8D208958F929F92AF9295
:10988000BF92CF92DF92EF92FF920F931F93CF93ED
:10989000DF93CDB7DEB7FC014083518362837383CE
:1098A0000483158326833783C086D186E286F386B8
:1098B00084869586A686B7864F85588969897A8970
:1098C000408B518B628B738BDF91CF911F910F91E6
:1098D000FF90EF90DF90CF90BF90AF909F908F90D0
:1098E0000895660F771F660F771F680F791FCB01EA
:1098F0000895660F771F660F771F680F791FCB01DA
:1099000008950F9300E029EA3AE940EE59E962ED43
:1099100078E98DE298E90E947E969093190D8093E4
:10992000180D892B79F40FEF29EA3AE940EE59E94D
:1099300062ED78E98DE298E90E947E969093190D88
:109940008093180D81E02091180D3091190D232B73
:1099500009F480E00F9108958091180D9091190DF0
:109960000E94F98F9093170D8093160D21E0892B9B
:1099700009F420E0822F0895CF93DF93CDB7DEB7AF
:10998000AB970FB6F894DEBF0FBECDBFAE014F5FF1
:109990005F4F6DE573E08091160D9091170D0E9459
:1099A000F994BE016F5F7F4F8091160D9091170D56
:1099B0000E94F2939093150D8093140D21E0892B52
:1099C00009F420E0822FAB960FB6F894DEBF0FBEED
:1099D000CDBFDF91CF9108958091160D9091170D15
:1099E0000E9457966095709580959095662797FD93
:1099F0006395772788279927862F0895BF92CF925E
:109A0000DF92EF92FF920F931F93CF93DF93CDB727
:109A1000DEB7AB970FB6F894DEBF0FBECDBF8C019B
:109A20006A0135E0B32EE62EF12C81E0E81AF10848
:109A3000BE016F5F7F4F8091140D9091150D0E94B4
:109A40003994F8018823E1F0DE01119620E030E03E
:109A50002E153F0544F0F801E20FF31F1082211587
:109A6000310559F004C08D9181110CC0F4CFC1149F
:109A7000D10461F0F601208309C0BA94C9F606C08A
:109A8000108204C081932F5F3F4FE2CF80E090E0CF
:109A9000AB960FB6F894DEBF0FBECDBFDF91CF916E
:109AA0001F910F91FF90EF90DF90CF90BF9008959E
:109AB0000F931F93CF93DF938C01EB010EC0B8017E
:109AC000CE010E949BDA009741F48091140D909191
:109AD000150D0E942C9481E009C0BE018091140DE7
:109AE0009091150D0E9439948111E9CFDF91CF91AA
:109AF0001F910F9108950F931F93CF93DF93CDB7CD
:109B0000DEB7AB970FB6F894DEBF0FBECDBF8B01AB
:109B1000BE016F5F7F4F0E94584D882371F0BE01D8
:109B20006F5F7F4F8091160D9091170D0E94749179
:109B3000F8019183808381E001C080E0AB960FB68D
:109B4000F894DEBF0FBECDBFDF91CF911F910F9173
:109B5000089560910E0D70910F0D8091100D9091F0
:109B6000110D0895CF93DF93CDB7DEB7AB970FB646
:109B7000F894DEBF0FBECDBFBE016F5F7F4F0E9466
:109B8000584D882359F0BE016F5F7F4F8091160DAD
:109B90009091170D0E94DB9581E001C080E0AB96AB
:109BA0000FB6F894DEBF0FBECDBFDF91CF91089501
:109BB000CF93DF93CDB7DEB7AB970FB6F894DEBF88
:109BC0000FBECDBFAE014F5F5F4FBC018091140D42
:109BD0009091150D0E94859591E0811101C090E052
:109BE000892FAB960FB6F894DEBF0FBECDBFDF91C5
:109BF000CF91089580910C0D089580910D0D0895D9
:109C0000CF93DF93EC018091120D9091130D00978B
:109C1000E1F04881BE016E5F7F4F50E00E94C39229
:109C200028818091080D9091090DA0910A0DB091A5
:109C30000B0D820F911DA11DB11D8093080D9093F6
:109C4000090DA0930A0DB0930B0DDF91CF910895EC
:109C500080910D0D882381F08091120D9091130D4C
:109C6000009721F00E94A8910E94C5971092130DB1
:109C70001092120D10920D0D6091080D7091090D4A
:109C800080910A0D90910B0D08950E948D97882365
:109C900091F041E050E067E07DE08091120D9091FD
:109CA000130D0E94BC9121E0181619060CF020E05B
:109CB0002093060D089541E06DE078E08CEC98E08B
:109CC0000E946D431092060D1092050D089580912B
:109CD000060D0895CF93DF931F92CDB7DEB7809125
:109CE000070D89830E94454E89810F90DF91CF91A6
:109CF000089510920C0D8091120D9091130D009704
:109D000021F00E94A8910E94C5971092130D109205
:109D1000120D089580910C0D81110E94794E809151
:109D20000D0D81110E94284E8091140D9091150DFA
:109D3000009731F00E9426941092150D1092140D88
:109D40008091160D9091170D009731F00E946E9141
:109D50001092170D1092160D8091180D9091190DFB
:109D6000009731F00E941E971092190D1092180D55
:109D700010920E0D10920F0D1092100D1092110DE9
:109D800008950E94329981110EC00E948D97811111
:109D900005C00E948A4E21E030E032C00E948A4E07
:109DA00022E030E02DC00E94814C811105C00E944C
:109DB0008A4E23E030E024C00E94AC4C811105C0E3
:109DC0000E948A4E24E030E01BC00E94BC4C8111EE
:109DD00005C00E948A4E25E030E012C00E94EC4C83
:109DE000811105C00E948A4E2AE030E009C00E941D
:109DF000AA97882319F026E030E002C020E030E086
:109E0000C9010895CF93DF93EC010E948A4E0E940E
:109E1000C14E9C01009719F08630910569F51092AA
:109E2000080D1092090D10920A0D10920B0D109250
:109E3000130D1092120D62E17DE0CE010E947B4D68
:109E4000882331F08091120D9091130D009719F431
:109E500027E030E011C00E94519660930E0D709380
:109E60000F0D8093100D9093110D81E080930C0DD8
:109E70000E94454E20E030E0C901DF91CF91089566
:109E80000F931F93CF93DF938C010E948A4E0E9401
:109E9000C14EEC01009769F51092080D1092090D62
:109EA00010920A0D10920B0D1092130D1092120DBC
:109EB000C8010E94B24DC8010E94D84D882389F084
:109EC00062E17DE0C8010E947B4D882369F08091AA
:109ED000120D9091130D892B51F081E080930D0D9F
:109EE00008C0C7E0D0E005C0C3E0D0E002C0C8E0D1
:109EF000D0E0CE01DF91CF911F910F9108950E9484
:109F00008A4E0E94C14E9C01009719F0863091053F
:109F100041F48091140D9091150D0E942C9420E035
:109F200030E0C901089540E06DE57AE18AE19DE005
:109F30000C944CD0CF92DF92EF92FF920F931F932D
:109F4000CF93DF9300D000D000D0CDB7DEB78C0127
:109F50007C016C018EE1C80ED11CC7010E943ED06D
:109F6000E6E0EE0EF11CEC14FD04B9F745E063E603
:109F70007AE1C8014E960E944CD085E0F80184A396
:109F800043E069E67AE1CE0101960E944CD086E07A
:109F9000FE013196D80101900D928A95E1F747E0D4
:109FA00069E67AE1CE0101960E944CD086E0FE017E
:109FB0003196D801169601900D928A95E1F743E00B
:109FC00061E67AE1CE0101960E944CD086E0FE0166
:109FD0003196D8011C9601900D928A95E1F745E0E3
:109FE00063E77AE1CE0101960E944CD086E0FE0143
:109FF0003196D801529601900D928A95E1F746E08C
:10A0000063E67AE1CE0101960E944CD086E0FE0123
:10A010003196D801589601900D928A95E1F72696CF
:10A020000FB6F894DEBF0FBECDBFDF91CF911F9169
:10A030000F91FF90EF90DF90CF900895EF92FF92F5
:10A040000F931F93CF93DF93EC01F12C86E0E82E62
:10A050000EC08E01EF9C000D111D112461E0C8019E
:10A060000E947BD061E0C8010E949BD0F3948CA138
:10A07000F81678F36E9661E0CE010E947BD061E025
:10A08000CE01DF91CF911F910F91FF90EF900C9433
:10A090009BD00F931F93CF93DF93EC0185E18A95BB
:10A0A000F1F7000061E0CE014E960E949BD085E161
:10A0B0008A95F1F7000010E006E009C061E0CE01EA
:10A0C000019F800D911D11240E949BD01F5F8CA1C8
:10A0D0001817A0F385E18A95F1F70000DF91CF9181
:10A0E0001F910F910895CF92DF92EF92FF920F93FD
:10A0F0001F93CF93DF93C62EEA0128E0E22EF12CC6
:10A1000030E8D32E8C01025E1F4F9D2D9C2161E013
:10A1100009F460E0CE010E949BD061E0C8010E947A
:10A120009BD085E18A95F1F7000060E0C8010E94AC
:10A130009BD0D69481E0E81AF10839F761E0CE01AE
:10A140000E949BD060E0CE010E947BD061E0C801FC
:10A150000E949BD0CE010E948ED0F82E60E0C801F4
:10A160000E949BD061E0CE010E947BD081E08F25D0
:10A17000DF91CF911F910F91FF90EF90DF90CF90E3
:10A180000895DF92EF92FF920F931F93CF93DF9387
:10A19000EC01E62E8A01F12C46E0D42E09C060E0E5
:10A1A000CE01DF9C800D911D11240E949BD0F39461
:10A1B0008CA1F816A0F385E18A95F1F7000060E024
:10A1C000CE014E960E949BD0A8016E2DCE01DF914C
:10A1D000CF911F910F91FF90EF90DF900C947350EF
:10A1E00040E06DE57AE185E49DE00E944CD080E29C
:10A1F0009DE00C949A4F4F925F926F927F928F9254
:10A200009F92AF92BF92CF92DF92EF92FF920F9305
:10A210001F93CF93DF9380915D0D90915E0D892BFD
:10A2200009F021C49091870D8091860D981771F0E7
:10A23000C091860D17E7C19FE0011124C857D24F86
:10A24000FE01EC58FF4F81E0808302C0C0E0D0E007
:10A25000D0935E0DC0935D0D209709F4B4C3888D33
:10A26000998DAA8DBB8D8093EB159093EC15A093DF
:10A27000ED15B093EE158C8D9D8DAE8DBF8D8093B9
:10A28000EF159093F015A093F115B093F21588A1F6
:10A2900099A1AAA1BBA18093F3159093F415A09363
:10A2A000F515B093F6158CA19DA1AEA1BFA1809329
:10A2B000F7159093F815A093F915B093FA1588A5A2
:10A2C00099A5AAA5BBA58093FB159093FC15A09317
:10A2D000FD15B093FE158AAD80935F0D8091600DE2
:10A2E000811111C01092630D1092640D1092650DD2
:10A2F0001092660DFE01E25AFF4F208131813F34FA
:10A3000008F046C051C0BE01E1E6FDE049E55DE070
:10A3100020E030E0DB011C96CD90DD90ED90FC90CC
:10A320001F97CD28CE28CF2839F18081882321F1AD
:10A33000D901A95AB24F8C91D901AA0FBB1F12EEB5
:10A34000E12E15E1F12EEA0EFB1ED701882341F024
:10A350008D919C91DA010D911C91801B910B07C08E
:10A360008D919C91DA010D911C91800F911FD70165
:10A3700011969C938E9310822F5F3F4F6C5F7F4F9F
:10A3800031964E5F5F4F2230310509F4ABCFC2CF1B
:10A390003D3930F403E0369527950A95E1F702C080
:10A3A00028E833E188E014C0383230F0369527953C
:10A3B0003695279584E00CC0343120F036952795EA
:10A3C00082E006C02032310510F420E230E081E066
:10A3D0008093670D205231092115B8E03B07D8F072
:10A3E000E32FFF27EE0FFF1FEE0FFF1FEF5DF74F6D
:10A3F00085919591A591B491AC01BD01AA27279FA4
:10A40000C001269F810D9A1F06948A1F9A1F11244E
:10A41000481B590B1BC0F901F695E795EC7FEF5DE2
:10A42000F34F4591559165917491DB012770332766
:10A430002A9FB0012B9F700D3A9F700D1124E3E00D
:10A4400076956795EA95E1F7461B570B5093690D92
:10A450004093680D8091670D80936A0DFE01EE5860
:10A46000FF4F8081882309F474C0CA59DF4F888167
:10A47000998190936C0D80936B0D9F3460F09D39A2
:10A4800030F443E0969587954A95E1F702C088E855
:10A4900093E128E014C0983230F096958795969510
:10A4A000879524E00CC0943120F09695879522E0A2
:10A4B00006C08032910510F480E290E021E0209304
:10A4C000670D9C01205231092115C8E03C07D8F0E6
:10A4D000E32FFF27EE0FFF1FEE0FFF1FEF5DF74F7C
:10A4E00085919591A591B491AC01BD01AA27279FB3
:10A4F000C001269F810D9A1F06948A1F9A1F11245E
:10A50000481B590B1BC0F901F695E795EC7FEF5DF1
:10A51000F34F4591559165917491DB012770332775
:10A520002A9FB0012B9F700D3A9F700D112403E0FC
:10A53000769567950A95E1F7461B570BCA01A0E08F
:10A54000B0E080936D0D90936E0DA0936F0DB0935E
:10A55000700D5093290140932801E0915D0DF09119
:10A560005E0D20AD2093710DEA58FF4F3081809130
:10A57000E2159091E315892B09F033608091E41581
:10A580009091E515892B09F034608091E01538131E
:10A590001CC0E0915D0DF0915E0D408151816281A2
:10A5A0007381F48805891689D789DF01AB58BF4FBD
:10A5B0003C9181E0411551056105710509F480E088
:10A5C00080931B16811144C087C0A5E1B2E0E9E188
:10A5D000F2E080E090E041E050E0BA01082E01C0D6
:10A5E000660F0A94EAF7D62FC091E015C327C62359
:10A5F00041F1D3237091E015DD2391F0762B709318
:10A60000E015CD91DC9111971881BA01008002C04C
:10A61000660F771F0A94E2F760956123688311C083
:10A62000609567236093E015CD91DC9111971881B7
:10A63000BA01008002C0660F771F0A94E2F7162B5A
:10A64000188301969396B3968530910531F6A1CF84
:10A65000C22FC1708F2D902FA12FBD2F6C017D01B6
:10A66000F594E794D794C794F094E094D094C09470
:10A67000C11CD11CE11CF11CC0921C16D0921D16ED
:10A68000E0921E16F0921F16D1E03111D0E0D09367
:10A6900013168093141690931516A0931616B09364
:10A6A0001716409324165093251660932616709320
:10A6B0002716CC2311F08FEF01C081E0809319168B
:10A6C00081E08C2780931A16109220161092211682
:10A6D000109222161092231644815581668177814B
:10A6E000F48805891689D78981E0411551056105EE
:10A6F000710509F480E080934416882309F446C06C
:10A7000021FBCC27C0F98F2D902FA12FBD2F6C01DD
:10A710007D01F594E794D794C794F094E094D09495
:10A72000C094C11CD11CE11CF11CC0924516D092F2
:10A730004616E0924716F0924816D1E0313009F003
:10A74000D0E0D0933C1680933D1690933E16A09394
:10A750003F16B093401640934D1650934E1660939B
:10A760004F1670935016CC2311F08FEF01C081E08B
:10A770008093421681E08C278093431610924916ED
:10A7800010924A1610924B1610924C164085518525
:10A7900062857385F48805891689D78981E041151A
:10A7A00051056105710509F480E080936D168823D9
:10A7B00009F446C022FBCC27C0F98F2D902FA12F82
:10A7C000BD2F6C017D01F594E794D794C794F09464
:10A7D000E094D094C094C11CD11CE11CF11CC09227
:10A7E0006E16D0926F16E0927016F0927116D1E04C
:10A7F000323009F0D0E0D0936516809366169093BE
:10A800006716A0936816B093691640937616509316
:10A8100077166093781670937916CC2311F08FEF2A
:10A8200001C081E080936B1681E08C2780936C16C9
:10A83000109272161092731610927416109275166A
:10A840004485558566857785F48805891689D78975
:10A8500081E0411551056105710509F480E080939F
:10A860009616882309F446C023FBCC27C0F98F2D08
:10A87000902FA12FBD2F6C017D01F594E794D79403
:10A88000C794F094E094D094C094C11CD11CE11CF6
:10A89000F11CC0929716D0929816E0929916F092F9
:10A8A0009A16D1E0333009F0D0E0D0938E16809321
:10A8B0008F1690939016A0939116B0939216409392
:10A8C0009F165093A0166093A1167093A216CC23E6
:10A8D00011F08FEF01C081E08093941681E08C2706
:10A8E0008093951610929B1610929C1610929D16AE
:10A8F00010929E1640895189628973891489D5897D
:10A90000C6893789EB58FF4FF08181E04115510529
:10A910006105710509F480E08093BF16882309F46E
:10A9200045C024FBEE27E0F9812F9D2FAC2FB32FDC
:10A930008C019D01359527951795079530952095A4
:10A94000109501951F4F2F4F3F4F0093C016109346
:10A95000C1162093C2163093C31621E0F43009F0DB
:10A9600020E02093B7168093B8169093B916A09361
:10A97000BA16B093BB164093C8165093C91660938D
:10A98000CA167093CB16EE2311F08FEF01C081E051
:10A990008093BD1681E08E278093BE161092C41658
:10A9A0001092C5161092C6161092C7161092730D0B
:10A9B0001092720D10924B0D10924C0D10924D0D85
:10A9C00010924E0D50C080ED97E090932901809336
:10A9D00028018091E2159091E315892B09F043C07D
:10A9E0008091E4159091E515892B11F40C94E160A8
:10A9F0003AC0A901082E01C0440F0A94EAF7C42FF7
:10AA00006091E0156727642341F1C7235091E01559
:10AA1000CC2391F0542B5093E015CD91DC911197FC
:10AA20006881A901008002C0440F551F0A94E2F713
:10AA300040954623488311C0409545234093E01537
:10AA4000CD91DC9111976881A901008002C0440F6B
:10AA5000551F0A94E2F7642B688301969396B39688
:10AA60008530910531F68091600D811108C080918B
:10AA70005D0D90915E0D892B09F04BC047C0409150
:10AA80005D0D50915E0DE1E6FDE0A9E5BDE080E0E1
:10AA900090E0FF24F394BA016A587F4F41155105A5
:10AAA00069F0EB01288130E0EC0123960C2E02C006
:10AAB000359527950A94E2F720FD20C020812111C9
:10AAC0001DC0EC01C95AD24F2881EC01CC0FDD1F0B
:10AAD000CE51DA4E222341F0288139810D911C910B
:10AAE0001197200F311F07C0288139810D911C91CA
:10AAF0001197201B310B39832883F0820196319600
:10AB000012968230910509F4B2CFC8CF80E00C9440
:10AB10005A61E091670D4091720D5091730DC09094
:10AB2000740DD090750DE090760DF090770DF09447
:10AB3000E094D094C094C11CD11CE11CF11CCD2C1C
:10AB4000DE2CEF2CFF24E7FCFA9470E021E030E0EB
:10AB500061E05EC5C0915D0DD0915E0DDE01AE5825
:10AB6000BF4F8C91811105C080911B16811177C058
:10AB70005EC141155105E9F042305105A1F58EAD98
:10AB80009FAD919581959109AA2797FDA095BA2F20
:10AB90008090971690909816A0909916B0909A165B
:10ABA000880D991DAA1DBB1D8C0D9D1DAE1DBF1DC1
:10ABB00012C08CAC9DACAA2497FCA094BA2C8091B6
:10ABC000971690919816A0919916B0919A16880DA3
:10ABD000991DAA1DBB1D8093971690939816A0935C
:10ABE0009916B0939A164115510599F48CAC9DAC09
:10ABF000AA2497FCA094BA2C8091C0169091C116FB
:10AC0000A091C216B091C316880D991DAA1DBB1D37
:10AC10001DC04230510509F0A7CF8EAD9FAD919573
:10AC200081959109AA2797FDA095BA2F8090C0160B
:10AC30009090C116A090C216B090C316880D991DB1
:10AC4000AA1DBB1D8C0D9D1DAE1DBF1D8093C01682
:10AC50009093C116A093C216B093C31685CF80906F
:10AC6000241690902516A0902616B0902716809155
:10AC70001C1690911D16A0911E16B0911F16880DDE
:10AC8000991DAA1DBB1D80931C1690931D16A093A1
:10AC90001E16B0931F16181619061A061B060CF07E
:10ACA000C6C04090201650902116609022167090D9
:10ACB0002316481459046A047B040CF0B8C0809031
:10ACC000141690901516A0901616B09017168819A5
:10ACD0009909AA09BB0980931C1690931D16A0938D
:10ACE0001E16B0931F1680911816882379F0809154
:10ACF000DC159091DD15F09119168F0F911DF7FD60
:10AD00009A959093DD158093DC1563C090911A1687
:10AD10008091001681119627A0910E02B0910F022A
:10AD200080911202FC91E90102C0CC0FDD1F8A95CF
:10AD3000E2F7992319F0FC2BFC9304C0CE01809517
:10AD40008F238C9380911A168823B1F0809123026F
:10AD500090912402892B11F40C94F360A0912502A8
:10AD6000B09126028C9190E00090270202C0959548
:10AD700087950A94E2F715C080911C0290911D02FC
:10AD8000892B11F40C94F360A0911E02B0911F0264
:10AD90008C9190E00090200202C0959587950A94CE
:10ADA000E2F781709091FF1589130C9404610C9463
:10ADB000F360A0910702B0910802FC91C9010090D4
:10ADC0000B0202C0880F991F0A94E2F780958F2327
:10ADD0008C938091EB159091EC15A091ED15B091AD
:10ADE000EE1580901916992487FC9094A92CB92C03
:10ADF000880D991DAA1DBB1D8093EB159093EC1532
:10AE0000A093ED15B093EE15809120169091211628
:10AE1000A0912216B09123160196A11DB11D809319
:10AE2000201690932116A0932216B093231680919A
:10AE30004416882309F4E8C080904D1690904E1671
:10AE4000A0904F16B09050168091451690914616DE
:10AE5000A0914716B0914816880D991DAA1DBB1DDB
:10AE60008093451690934616A0934716B0934816C4
:10AE7000181619061A061B060CF0C6C04090491693
:10AE800050904A1660904B1670904C164814590416
:10AE90006A047B040CF0B8C080903D1690903E167A
:10AEA000A0903F16B090401688199909AA09BB09CD
:10AEB0008093451690934616A0934716B093481674
:10AEC00080914116882379F08091DE159091DF15ED
:10AED000F09142168F0F911DF7FD9A959093DF1513
:10AEE0008093DE1563C090914316809129168111DD
:10AEF0009627A0913102B091320280913502FC91E7
:10AF0000E90102C0CC0FDD1F8A95E2F7992319F001
:10AF1000FC2BFC9304C0CE0180958F238C938091F1
:10AF200043168823B1F08091460290914702892B05
:10AF300011F40C940861A0914802B09149028C91DF
:10AF400090E000904A0202C0959587950A94E2F736
:10AF500015C080913F0290914002892B11F40C940E
:10AF60000861A0914102B09142028C9190E0009062
:10AF7000430202C0959587950A94E2F781709091FB
:10AF8000281689130C9419610C940861A0912A0267
:10AF9000B0912B02FC91C90100902E0202C0880FD3
:10AFA000991F0A94E2F780958F238C938091EF1577
:10AFB0009091F015A091F115B091F2158090421684
:10AFC000992487FC9094A92CB92C880D991DAA1D51
:10AFD000BB1D8093EF159093F015A093F115B093DE
:10AFE000F2158091491690914A16A0914B16B09196
:10AFF0004C160196A11DB11D8093491690934A16D7
:10B00000A0934B16B0934C1680916D16882309F4CB
:10B01000E8C08090761690907716A0907816B09041
:10B02000791680916E1690916F16A0917016B0915E
:10B030007116880D991DAA1DBB1D80936E169093E5
:10B040006F16A0937016B0937116181619061A068B
:10B050001B060CF0C6C0409072165090731660909C
:10B06000741670907516481459046A047B040CF029
:10B07000B8C08090661690906716A0906816B09041
:10B08000691688199909AA09BB0980936E169093CD
:10B090006F16A0937016B093711680916A1688236C
:10B0A00079F08091E0159091E115F0916B168F0F7A
:10B0B000911DF7FD9A959093E1158093E01563C07B
:10B0C00090916C168091521681119627A09154028E
:10B0D000B091550280915802FC91E90102C0CC0F59
:10B0E000DD1F8A95E2F7992319F0FC2BFC9304C02D
:10B0F000CE0180958F238C9380916C168823B1F0BC
:10B100008091690290916A02892B11F40C941D615F
:10B11000A0916B02B0916C028C9190E000906D0256
:10B1200002C0959587950A94E2F715C08091620256
:10B1300090916302892B11F40C941D61A09164021B
:10B14000B09165028C9190E00090660202C09595E6
:10B1500087950A94E2F781709091511689130C94A7
:10B160002E610C941D61A0914D02B0914E02FC9194
:10B17000C9010090510202C0880F991F0A94E2F79A
:10B1800080958F238C938091F3159091F415A09165
:10B19000F515B091F61580906B16992487FC909464
:10B1A000A92CB92C880D991DAA1DBB1D8093F315E0
:10B1B0009093F415A093F515B093F615809172163F
:10B1C00090917316A0917416B09175160196A11DF9
:10B1D000B11D8093721690937316A0937416B0935A
:10B1E000751680919616882309F4E8C080909F1602
:10B1F0009090A016A090A116B090A21680919716DC
:10B2000090919816A0919916B0919A16880D991D53
:10B21000AA1DBB1D8093971690939816A09399161C
:10B22000B0939A16181619061A061B060CF0C6C01B
:10B2300040909B1650909C1660909D1670909E16A4
:10B24000481459046A047B040CF0B8C080908F162F
:10B2500090909016A0909116B09092168819990926
:10B26000AA09BB098093971690939816A0939916F4
:10B27000B0939A1680919316882379F08091E21505
:10B280009091E315F09194168F0F911DF7FD9A950B
:10B290009093E3158093E21563C090919516809189
:10B2A0007B1681119627A0917702B0917802809148
:10B2B0007B02FC91E90102C0CC0FDD1F8A95E2F709
:10B2C000992319F0FC2BFC9304C0CE0180958F23A9
:10B2D0008C93809195168823B1F080918C02909187
:10B2E0008D02892B11F40C943261A0918E02B091E1
:10B2F0008F028C9190E00090900202C09595879506
:10B300000A94E2F715C08091850290918602892BFC
:10B3100011F40C943261A0918702B09188028C9153
:10B3200090E00090890202C0959587950A94E2F713
:10B33000817090917A1689130C9443610C94326158
:10B34000A0917002B0917102FC91C9010090740249
:10B3500002C0880F991F0A94E2F780958F238C937F
:10B360008091F7159091F815A091F915B091FA1503
:10B3700080909416992487FC9094A92CB92C880D60
:10B38000991DAA1DBB1D8093F7159093F815A093E6
:10B39000F915B093FA1580919B1690919C16A09187
:10B3A0009D16B0919E160196A11DB11D80939B160E
:10B3B00090939C16A0939D16B0939E168091BF16F5
:10B3C000882309F4E4C08090C8169090C916A09014
:10B3D000CA16B090CB168091C0169091C116A0915C
:10B3E000C216B091C316880D991DAA1DBB1D80936E
:10B3F000C0169093C116A093C216B093C316181628
:10B4000019061A061B060CF0C2C04090C4165090D4
:10B41000C5166090C6167090C716481459046A0481
:10B420007B040CF0B4C08090B8169090B916A09030
:10B43000BA16B090BB1688199909AA09BB0980935E
:10B44000C0169093C116A093C216B093C3168091F4
:10B45000BC16882379F08091E4159091E515F09160
:10B46000BD168F0F911DF7FD9A959093E51580936A
:10B47000E4155FC09091BE168091A41681119627A5
:10B48000A0919A02B0919B0280919E02FC91E901E9
:10B4900002C0CC0FDD1F8A95E2F7992319F0FC2B2F
:10B4A000FC9304C0CE0180958F238C938091BE16AF
:10B4B0008823A9F08091AF029091B002892B09F402
:10B4C000E9C6A091B102B091B2028C9190E00090D7
:10B4D000B30202C0959587950A94E2F714C0809153
:10B4E000A8029091A902892B09F4D4C6A091AA02BE
:10B4F000B091AB028C9190E00090AC0202C09595A7
:10B5000087950A94E2F781709091A3168913BFC6BC
:10B51000C1C6A0919302B0919402FC91C901009020
:10B52000970202C0880F991F0A94E2F780958F2333
:10B530008C938091FB159091FC15A091FD15B09115
:10B54000FE158090BD16992487FC9094A92CB92CE7
:10B55000880D991DAA1DBB1D8093FB159093FC15AA
:10B56000A093FD15B093FE158091C4169091C51659
:10B57000A091C616B091C7160196A11DB11D80936A
:10B58000C4169093C516A093C616B093C7168091A3
:10B590004B0D90914C0DA0914D0DB0914E0D01961B
:10B5A000A11DB11D80934B0D90934C0DA0934D0D9B
:10B5B000B0934E0D80904B0D90904C0DA0904D0D82
:10B5C000B0904E0DA0915D0DB0915E0D54968D9191
:10B5D0009D910D90BC91A02D88169906AA06BB06D8
:10B5E000B0F040914B0D50914C0D60914D0D70910C
:10B5F0004E0DE0915D0DF0915E0D84A595A5A6A57B
:10B60000B7A584179507A607B70730F4BDC07F5FBD
:10B610007E170CF49FCAE5CF00916D0D10916E0D51
:10B6200020916F0D3091700D44A955A966A977A995
:10B63000AA27059FB12D169FC001269F900D259F1B
:10B64000800D911D069FB00D811D9A1F159FB00D95
:10B65000811D9A1F249FB00D811D9A1F149FB10D4B
:10B660008A1F9A1FB6958A1F9A1F1124DF01AA59B3
:10B67000BF4F4D915C91480F591F50936C0D4093F3
:10B680006B0DE25AFF4F80819181A281B38160E00E
:10B6900070E084179507A607B70720F490936C0D08
:10B6A00080936B0D80916B0D90916C0D9F3460F0C9
:10B6B0009D3930F4D3E096958795DA95E1F702C08D
:10B6C00088E893E148E014C0983230F09695879569
:10B6D0009695879544E00CC0943120F09695879517
:10B6E00042E006C08032910510F480E290E041E033
:10B6F0004093670D80978115D8E09D07C8F0E92F2A
:10B70000FF27EE0FFF1FEE0FFF1FEF5DF74FC590F6
:10B71000D590E590F490A601B701AA27879FF00184
:10B72000869FE10DFA1F0694EA1FFA1F112419C023
:10B73000FC01F695E795EC7FEF5DF34FC590D59052
:10B74000E590F490A601877099278E9DF0018F9D5A
:10B75000F00D9E9DF00D112463E0F695E7956A9536
:10B76000E1F74E1B5F0B5093290140932801040F12
:10B77000151F211D311D00936D0D10936E0D20932B
:10B780006F0D3093700D2AC140914B0D50914C0DAF
:10B7900060914D0D70914E0D80A991A9A2A9B3A9F8
:10B7A0002091720D3091730D84179507A607B70786
:10B7B00008F000C1232B31F481E090E09093730DE9
:10B7C0008093720D8091720D9091730D019771F4B9
:10B7D00082E090E09093730D8093720D1092740D3F
:10B7E0001092750D1092760D1092770DEF01C05CDE
:10B7F000DF4F8091740D9091750DA091760DB091F1
:10B80000770D488159816A817B81840F951FA61F1E
:10B81000B71F8093740D9093750DA093760DB09320
:10B82000770D0091630D1091640D2091650D30919D
:10B83000660D44A955A966A977A9AA27059FB12D28
:10B84000169FC001269F900D259F800D911D069F7C
:10B85000B00D811D9A1F159FB00D811D9A1F249F49
:10B86000B00D811D9A1F149FB10D8A1F9A1FB695A6
:10B870008A1F9A1F11249093790D8093780D40911F
:10B880006B0D50916C0D60915D0D70915E0D4817C0
:10B89000590730F4FB01E659FF4F8081918114C0B4
:10B8A000481B590B5093790D4093780DFB01E659D5
:10B8B000FF4F80819181A281B38160E070E04817E1
:10B8C00059076A077B0720F49093790D8093780DD0
:10B8D0008091780D9091790D9F3460F09D3930F40E
:10B8E000D3E096958795DA95E1F702C088E893E171
:10B8F00048E014C0983230F09695879596958795D4
:10B9000044E00CC0943120F09695879542E006C043
:10B910008032910510F480E290E041E04093670DA1
:10B920008097811548E09407C8F0E92FFF27EE0FB4
:10B93000FF1FEE0FFF1FEF5DF74FC590D590E5900D
:10B94000F490A601B701AA27879FF001869FE10D19
:10B95000FA1F0694EA1FFA1F112419C0FC01F6957C
:10B96000E795EC7FEF5DF34FC590D590E590F490AF
:10B97000A601877099278E9DF0018F9DF00D9E9DE9
:10B98000F00D112463E0F695E7956A95E1F74E1BFB
:10B990005F0B5093290140932801040F151F211DAF
:10B9A000311D0093630D1093640D2093650D30934A
:10B9B000660D14C0232B31F481E090E09093730D59
:10B9C0008093720D8091680D9091690D909329017B
:10B9D0008093280180916A0D8093670D40914B0DF3
:10B9E00050914C0D60914D0D70914E0DE0915D0D9B
:10B9F000F0915E0D84899589A689B7894817590702
:10BA00006A077B0708F482C810925E0D10925D0DE4
:10BA10009091870D8091860D981731F08091860D59
:10BA20008F5F8F708093860D9091870D8091860D2A
:10BA3000981771F0C091860D87E7C89FE001112427
:10BA4000C857D24FFE01EC58FF4F81E0808302C0FF
:10BA5000C0E0D0E0D0935E0DC0935D0D209709F457
:10BA6000AEC3888D998DAA8DBB8D8093EB15909375
:10BA7000EC15A093ED15B093EE158C8D9D8DAE8DCC
:10BA8000BF8D8093EF159093F015A093F115B093AF
:10BA9000F21588A199A1AAA1BBA18093F315909357
:10BAA000F415A093F515B093F6158CA19DA1AEA148
:10BAB000BFA18093F7159093F815A093F915B09353
:10BAC000FA1588A599A5AAA5BBA58093FB15909307
:10BAD000FC15A093FD15B093FE158AAD80935F0D04
:10BAE0008091600D811111C01092630D1092640D50
:10BAF0001092650D1092660DFE01E25AFF4F2081F3
:10BB000031813F3408F041C04CC0BE0141E65DE0E8
:10BB1000E9E5FDE020E030E0DB011C96CD90DD9012
:10BB2000ED90FC901F97CD28CE28CF2819F1DA018F
:10BB30008C918823F9F0D901A95AB24F8C91D9017F
:10BB4000AA0FBB1FAE51BA4E882341F08D919C9134
:10BB5000119700811181801B910B07C08D919C91E1
:10BB6000119700811181800F911F11969C938E93E4
:10BB7000DA011C922F5F3F4F6C5F7F4F4F5F5F4F2B
:10BB800032962230310541F6AFCF3D3930F403E033
:10BB9000369527950A95E1F702C028E833E188E059
:10BBA00014C0383230F0369527953695279584E0C5
:10BBB0000CC0343120F03695279582E006C0203243
:10BBC000310510F420E230E081E08093670D2052CF
:10BBD00031092115B8E03B07D8F0E32FFF27EE0F1E
:10BBE000FF1FEE0FFF1FEF5DF74F85919591A59118
:10BBF000B491AC01BD01AA27279FC001269F810DEA
:10BC00009A1F06948A1F9A1F1124481B590B1BC0A8
:10BC1000F901F695E795EC7FEF5DF34F459155916E
:10BC200065917491DB01277033272A9FB0012B9F08
:10BC3000700D3A9F700D1124E3E076956795EA95B3
:10BC4000E1F7461B570B5093690D4093680D8091A7
:10BC5000670D80936A0DFE01EE58FF4F80818823A7
:10BC600009F474C0CA59DF4F8881998190936C0D93
:10BC700080936B0D9F3460F09D3930F443E09695CE
:10BC800087954A95E1F702C088E893E128E014C05F
:10BC9000983230F0969587959695879524E00CC05C
:10BCA000943120F09695879522E006C08032910568
:10BCB00010F480E290E021E02093670D9C01205277
:10BCC00031092115C8E03C07D8F0E32FFF27EE0F1C
:10BCD000FF1FEE0FFF1FEF5DF74F85919591A59127
:10BCE000B491AC01BD01AA27279FC001269F810DF9
:10BCF0009A1F06948A1F9A1F1124481B590B1BC0B8
:10BD0000F901F695E795EC7FEF5DF34F459155917D
:10BD100065917491DB01277033272A9FB0012B9F17
:10BD2000700D3A9F700D112403E0769567950A9582
:10BD3000E1F7461B570BCA01A0E0B0E080936D0D00
:10BD400090936E0DA0936F0DB093700D50932901D9
:10BD500040932801E0915D0DF0915E0D20AD2093A0
:10BD6000710DEA58FF4F30818091E2159091E315F3
:10BD7000892B09F033608091E4159091E515892BAA
:10BD800009F034608091E01538131CC0E0915D0D1E
:10BD9000F0915E0D4081518162817381F488058943
:10BDA0001689D789DF01AB58BF4F3C9181E041151F
:10BDB00051056105710509F480E080931B1681111E
:10BDC00044C087C0A5E1B2E0E9E1F2E080E090E0A4
:10BDD00041E050E0BA01082E01C0660F0A94EAF76C
:10BDE000D62FC091E015C327C62341F1D32370910C
:10BDF000E015DD2391F0762B7093E015CD91DC9169
:10BE000011971881BA01008002C0660F771F0A944B
:10BE1000E2F760956123688311C0609567236093A2
:10BE2000E015CD91DC9111971881BA01008002C014
:10BE3000660F771F0A94E2F7162B188301969396E4
:10BE4000B3968530910531F6A1CFC22FC1708F2DE9
:10BE5000902FA12FBD2F6C017D01F594E794D7940D
:10BE6000C794F094E094D094C094C11CD11CE11C00
:10BE7000F11CC0921C16D0921D16E0921E16F09274
:10BE80001F16D1E03111D0E0D09313168093141611
:10BE900090931516A0931616B09317164093241678
:10BEA000509325166093261670932716CC2311F015
:10BEB0008FEF01C081E08093191681E08C27809379
:10BEC0001A16109220161092211610922216109215
:10BED00023164481558166817781F4880589168906
:10BEE000D78981E0411551056105710509F480E0AC
:10BEF00080934416882309F446C021FBCC27C0F95F
:10BF00008F2D902FA12FBD2F6C017D01F594E7940B
:10BF1000D794C794F094E094D094C094C11CD11CE1
:10BF2000E11CF11CC0924516D0924616E0924716CD
:10BF3000F0924816D1E0313009F0D0E0D0933C16B1
:10BF400080933D1690933E16A0933F16B0934016F3
:10BF500040934D1650934E1660934F1670935016A3
:10BF6000CC2311F08FEF01C081E08093421681E075
:10BF70008C27809343161092491610924A161092FD
:10BF80004B1610924C164085518562857385F48856
:10BF900005891689D78981E041155105610571052B
:10BFA00009F480E080936D16882309F446C022FBD3
:10BFB000CC27C0F98F2D902FA12FBD2F6C017D01B3
:10BFC000F594E794D794C794F094E094D094C094F7
:10BFD000C11CD11CE11CF11CC0926E16D0926F16D0
:10BFE000E0927016F0927116D1E0323009F0D0E094
:10BFF000D09365168093661690936716A093681683
:10C00000B09369164093761650937716609378161E
:10C0100070937916CC2311F08FEF01C081E08093EB
:10C020006B1681E08C2780936C161092721610921A
:10C030007316109274161092751644855585668590
:10C040007785F48805891689D78981E041155105DE
:10C050006105710509F480E080939616882309F440
:10C0600046C023FBCC27C0F98F2D902FA12FBD2FC9
:10C070006C017D01F594E794D794C794F094E09413
:10C08000D094C094C11CD11CE11CF11CC092971625
:10C09000D0929816E0929916F0929A16D1E0333029
:10C0A00009F0D0E0D0938E1680938F16909390165F
:10C0B000A0939116B093921640939F165093A0169A
:10C0C0006093A1167093A216CC2311F08FEF01C0DC
:10C0D00081E08093941681E08C27809395161092CE
:10C0E0009B1610929C1610929D1610929E164089D7
:10C0F0005189628973891489D589C6893789EB5832
:10C10000FF4FF08181E0411551056105710509F48A
:10C1100080E08093BF16882309F445C024FBEE27F6
:10C12000E0F9812F9D2FAC2FB32F8C019D01359508
:10C1300027951795079530952095109501951F4FD8
:10C140002F4F3F4F0093C0161093C1162093C21675
:10C150003093C31621E0F43009F020E02093B716A5
:10C160008093B8169093B916A093BA16B093BB16E5
:10C170004093C8165093C9166093CA167093CB1695
:10C18000EE2311F08FEF01C081E08093BD1681E0B6
:10C190008E278093BE161092C4161092C516109268
:10C1A000C6161092C7161092730D1092720D10924F
:10C1B0004B0D10924C0D10924D0D10924E0D81E0D2
:10C1C00079C07091E1158091E015781711F40C9405
:10C1D0003355A5E1B2E0E9E1F2E080E090E021E052
:10C1E00030E00C94F954A0910702B0910802FC9140
:10C1F000C90100900B0202C0880F991F0A94E2F750
:10C20000F82BFC930C94D9561092E6150C94D95641
:10C21000A0912A02B0912B02FC91C90100902E023C
:10C2200002C0880F991F0A94E2F7F82BFC930C9434
:10C23000C6571092E7150C94C657A0914D02B091C5
:10C240004E02FC91C9010090510202C0880F991F53
:10C250000A94E2F7F82BFC930C94B3581092E8156B
:10C260000C94B358A0917002B0917102FC91C90175
:10C270000090740202C0880F991F0A94E2F7F82B0D
:10C28000FC930C94A0591092E9150C94A0591092AB
:10C29000EA153FC9A0919302B0919402FC91C901A3
:10C2A0000090970202C0880F991F0A94E2F7F82BBA
:10C2B000FC932FC9DF91CF911F910F91FF90EF90C9
:10C2C000DF90CF90BF90AF909F908F907F906F90B6
:10C2D0005F904F90089570917A0D7F5F70937A0D03
:10C2E00080917B0D8F5F80937B0D50917C0D6091D1
:10C2F0007E0D40E081E090E03FC030917B16E09100
:10C300007702F091780220917B02311199C0A2C08E
:10C310002091E2153091E3152F5F3F4F18C0209117
:10C32000E2153091E3151216130624F530917B16B1
:10C33000E0917702F091780220917B023111A0C048
:10C3400095C02091E2153091E315215031093093C9
:10C35000E3152093E215E0917002F0917102708173
:10C360009C010090740202C0220F331F0A94E2F76E
:10C37000722B70834F5F70E02091E2153091E315CE
:10C38000232B61F470937A0D50917D0D60917F0D98
:10C3900070917B0D40E081E090E045C0751708F496
:10C3A000F1CF461379C0EECF3091A416E0919A02F6
:10C3B000F0919B0220919E02311191C084C0209186
:10C3C000E4153091E5152F5F3F4F18C02091E4151B
:10C3D0003091E5151216130624F53091A416E0915C
:10C3E0009A02F0919B0220919E02311182C08DC071
:10C3F0002091E4153091E515215031093093E51570
:10C400002093E415E0919302F091940270819C01D5
:10C410000090970202C0220F331F0A94E2F7722B9A
:10C4200070834F5F70E02091E4153091E515232B68
:10C4300009F475C0751708F472C0461373C06FC055
:10C440007081DC0102C0AA0FBB1F2A95E2F77A2B8C
:10C4500070835ECF7081DC0102C0AA0FBB1F2A95DA
:10C46000E2F79D0120952723208352CF7081DC01C4
:10C4700002C0AA0FBB1F2A95E2F77A2B708361CF07
:10C480007081DC0102C0AA0FBB1F2A95E2F79D0153
:10C4900020952723208355CFE0917002F0917102FF
:10C4A00070819C010090740202C0220F331F0A9415
:10C4B000E2F72095272320832091E2153091E315A0
:10C4C00037FF2DCF1ACF7081DC0102C0AA0FBB1F2E
:10C4D0002A95E2F79D0120952723208370CF708154
:10C4E000DC0102C0AA0FBB1F2A95E2F77A2B7083EA
:10C4F00066CF7081DC0102C0AA0FBB1F2A95E2F74C
:10C500009D0120952723208373CF7081DC0102C019
:10C51000AA0FBB1F2A95E2F77A2B708369CF70931D
:10C520007B0D0895E0919302F091940270819C013B
:10C530000090970202C0220F331F0A94E2F7209561
:10C54000272320832091E4153091E51537FF3ECF56
:10C550002BCF4F925F926F927F928F929F92AF926A
:10C56000BF92CF92DF92EF92FF920F931F93CF93E0
:10C57000DF9310925F0D9FE4C92E9DE0D92E2AE72C
:10C58000E22E2DE0F22ECEE7DDE03CE7A32E3DE0EB
:10C59000B32E00E010E055245394F60161907190A1
:10C5A000819091906F01802F8D5F0E94A0789B01F8
:10C5B000AC01C401B3010E94CED79B01AC0160E085
:10C5C00070E48CE196E40E94F5D53B014C0120E03B
:10C5D00030E040E85FE3772D992D0E94CAD7181606
:10C5E0004CF4662D772D882D992D0E94DED53B01C8
:10C5F0004C0110C020E030E040E85FE3662D772D6D
:10C60000882D992D0E94F1D587FF04C0612C712CD3
:10C61000812C912C662D772D882D992D0E949CD6EA
:10C62000462EF50161935F01662311F018820FC059
:10C63000262D372D482D592D60E070E080E89FE3CE
:10C640000E94F5D50E94DED50E949CD66883888121
:10C65000811101C05882F801EE0FFF1FEE51FA4E12
:10C6600011821082F70141927F010F5F1F4F2196C7
:10C670000230110509F091CFDF91CF911F910F91F9
:10C68000FF90EF90DF90CF90BF90AF909F908F90F2
:10C690007F906F905F904F9008952091870D9091BB
:10C6A000860D81E0291380E008950F931F93CF93A7
:10C6B000DF93FB017FB7F894EC0188819981AA810F
:10C6C000BB818093EB159093EC15A093ED15B0937F
:10C6D000EE1580819181A281B3818093EF159093B3
:10C6E000F015A093F115B093F215FA0180819181B4
:10C6F000A281B3818093F3159093F415A093F5155F
:10C70000B093F615E90188819981AA81BB81809354
:10C71000F7159093F815A093F915B093FA15F80151
:10C7200080819181A281B3818093FB159093FC1548
:10C73000A093FD15B093FE157FBFDF91CF911F91A0
:10C740000F9108958F929F92AF92BF92EF92FF92B6
:10C750000F931F93CF93DF93EFB7F8948090EB156F
:10C760009090EC15A090ED15B090EE15DC018D9237
:10C770009D92AD92BC9213978091EF159091F01518
:10C78000A091F115B091F215EB0188839983AA83EA
:10C79000BB838091F3159091F415A091F515B0919C
:10C7A000F615EA0188839983AA83BB838091F715E4
:10C7B0009091F815A091F915B091FA15E9018883C7
:10C7C0009983AA83BB838091FB159091FC15A0915E
:10C7D000FD15B091FE15E80188839983AA83BB8378
:10C7E00080915F0DD7018C93EFBFDF91CF911F91A7
:10C7F0000F91FF90EF90BF90AF909F908F90089512
:10C80000809173008D7F8093730006C08091860DA8
:10C810008F5F8F708093860D9091870D8091860D2C
:10C8200098135DC010925E0D10925D0D2FB7F894B5
:10C830008091EB159091EC15A091ED15B091EE154E
:10C8400080930D1590930E15A0930F15B0931015AE
:10C850008091EF159091F015A091F115B091F2151E
:10C860008093111590931215A0931315B09314157E
:10C870008091F3159091F415A091F515B091F615EE
:10C880008093151590931615A0931715B09318154E
:10C890008091F7159091F815A091F915B091FA15BE
:10C8A0008093191590931A15A0931B15B0931C151E
:10C8B0008091FB159091FC15A091FD15B091FE158E
:10C8C00080931D1590931E15A0931F15B0932015EE
:10C8D0002FBF8091730082608093730008959091C0
:10C8E000870D8091860D981709F496CF8FCF80938E
:10C8F000600D81E08093610D8093620D089540E0AA
:10C900006DE57AE180E89DE00C944CD030EC20E4B9
:10C91000889410F0921710F0921B232B3695880FF5
:10C92000991F23273E7FA9F710F0880F2907231F9F
:10C93000C90108952F923F924F925F926F927F921A
:10C940008F929F92AF92BF92CF92DF92EF92FF921F
:10C950000F931F93CF93DF93CDB7DEB768970FB6D2
:10C96000F894DEBF0FBECDBF1C0148015901F10193
:10C97000EE58FF4F80818823A1F0242F352FAB0183
:10C980002130310561E04607510524F020E030E018
:10C9900041E050E071E087169104A706B1042CF441
:10C9A00008C020E030E041E050E0812C912C54019F
:10C9B000A39471018EE5E80EF11CD7014D905D90B6
:10C9C0006D907C90C201772766270E9462D47058D0
:10C9D0008F4F9F4F9C01552737FD5095452F2D8335
:10C9E0003E834F835887F70180819181A281B38173
:10C9F00077276627A50194010E9462D470588F4F53
:10CA00009F4F9C01552737FD5095452F29873A8721
:10CA10004B875C874D815E816F81788548375105F2
:10CA20006105710540F468E770E080E090E06D8397
:10CA30007E838F83988789859A85AB85BC85883767
:10CA40009105A105B10540F428E730E040E050E051
:10CA500029873A874B875C872D813E814F81588596
:10CA6000CA01B9010E9431D82B013C0129853A85C0
:10CA70004B855C85CA01B9010E9431D86D8B7E8BD4
:10CA80008F8B988F910122593F4FD9014D915D9124
:10CA90006D917C91498B5A8B6B8B7C8B6A017B01EE
:10CAA000CC0CDD1CEE1CFF1CF101EE58FF4F808109
:10CAB000882309F447C091012E593F4FD9014D9168
:10CAC0005D916D917C9149835A836B837C83C11402
:10CAD000D104E104F10469F0CB01BA0164197509CC
:10CAE00086099709A70196010E9497D849015A0122
:10CAF00003C0812C912C540122273327A9012C1922
:10CB00003D094E095F092D873E874F87588B232BA0
:10CB1000242B252BF9F06D897E898F89988D2981A9
:10CB20003A814B815C81621B730B840B950B2D85C5
:10CB30003E854F8558890E9497D829833A834B8335
:10CB40005C830CC019821A821B821C82812C912C5E
:10CB5000540104C019821A821B821C82D10154968E
:10CB60004D915D916D917C9157974D875E876F8751
:10CB7000788BDB01CA0188199909AA09BB092981A7
:10CB80003A814B815C81821B930BA40BB50BB7FFE1
:10CB90003CC08D849E84AF84B888C114D104E10464
:10CBA000F104D9F0A7019601C501B4010E9431D862
:10CBB00064197509860997092D893E894F89588D11
:10CBC000620F731F841F951FA7019601220F331F49
:10CBD000441F551F0E9497D803C020E030E0A901F0
:10CBE000DA01C90157FF03C080E090E0DC014D8508
:10CBF0005E856F85788984179507A607B70714F4B3
:10CC00004C015D0180E090E0DC01A5019401280F5A
:10CC1000391F4A1F5B1F2D873E874F87588BF101B5
:10CC200023AD222309F412C1892B8A2B8B2B09F007
:10CC300073C0A50194012F5F3F4F4F4F5F4F57FFC8
:10CC400020C050954095309521953F4F4F4F5F4FF5
:10CC500069897A898B899C890E9431D8660F771FF0
:10CC6000881F991F641575058605970508F04BC048
:10CC7000A3019201261B370B480B590BDA01C9019E
:10CC800010C069897A898B899C890E9431D8DC011E
:10CC9000CB01880F991FAA1FBB1F840D951DA61DD0
:10CCA000B71D811530E89307A105B10558F40E941E
:10CCB00086642C01662457FC6094762C320155243E
:10CCC000442424C0F12C22E0B695A795979587952A
:10CCD0002A95D1F7F394811540E89407A105B10591
:10CCE00090F70E9486642C01662457FC6094762C91
:10CCF00032015524442404C0440C551C661C771C86
:10CD0000FA94D2F703C0412C512C3201230177242D
:10CD100057FC7094672C07C0F101E25AFF4F408026
:10CD2000518062807380181419041A041B04F4F4EF
:10CD3000D301C2012D813E814F815885821B930B07
:10CD4000A40BB50BAC0133272227609174157091A9
:10CD5000751580917615909177150E9462D4BB2746
:10CD600097FDB095AB2F6C0197FF02C0C12CD12C61
:10CD70004D855E856F8578894F5F5F4F6F4F7F4F21
:10CD8000F10184899589A689B789481759076A07E7
:10CD90007B070CF063C029853A854B855C85421A78
:10CDA000530A640A750AA201332722276091741579
:10CDB0007091751580917615909177150E9462D4C7
:10CDC0007C018091701590917115A0917215B091B0
:10CDD0007315892B8A2B8B2B99F169817A818B8131
:10CDE0009C81AB0133272227F101E259FF4F80815B
:10CDF0009181A281B38165E0B595A79597958795B7
:10CE00006A95D1F7772766270E94CCD42B013C0185
:10CE100060917015709171158091721590917315D4
:10CE200020E030E044E650E00E9462D4A301920189
:10CE30000E9462D4BB2797FDB095AB2FB7FF03C00C
:10CE400080E090E0DC01F7FE0EC00BC080E090E0D7
:10CE5000DC01E12CF12CC12CD12C05C080E090E04C
:10CE6000DC01E12CF12C2FB7F894F101EC58FF4FC5
:10CE70003081311142C0F101EE58FF4F3081332330
:10CE800069F0F10184A695A6A6A6B7A64D855E8594
:10CE90006F85788940AB51AB62AB73AB5101F6E65D
:10CEA000AF0EB11C4D815E816F817885F5014083A5
:10CEB0005183628373835101FAE6AF0EB11C498539
:10CEC0005A856B857C85F50140835183628373832A
:10CED000F101D5AEC4AEF7AEE6AEEC5BFF4F11820A
:10CEE0001082F101EA5BFF4F11821082F101E05CD8
:10CEF000FF4F80839183A283B3832FBF68960FB6C1
:10CF0000F894DEBF0FBECDBFDF91CF911F910F917F
:10CF1000FF90EF90DF90CF90BF90AF909F908F9059
:10CF20007F906F905F904F903F902F9008952F9239
:10CF30003F924F925F926F927F928F929F92AF92A9
:10CF4000BF92CF92DF92EF92FF920F931F93CF93F6
:10CF5000DF9300D000D0CDB7DEB71C018B01009766
:10CF600009F497C16115710509F493C19C01205B17
:10CF70003F4FD9018D919D910D90BC91A02D89833A
:10CF80009A83AB83BC83F101E45BFF4F8081918185
:10CF9000A281B38129813A814B815C8182179307F9
:10CFA000A407B50709F475C1F101E35AFF4F808169
:10CFB000811147C1FB01ED58FF4F8081882309F49F
:10CFC00040C1FB01E45BFF4F80819181A281B3816D
:10CFD00082179307A407B5070CF033C1BC01CD013C
:10CFE0005CE095958795779567955A95D1F7F1010E
:10CFF000E85AFF4F80809180A280B380B094A094C3
:10D0000090948094811C911CA11CB11CE6E0B59405
:10D01000A79497948794EA95D1F7F101EC5AFF4FC2
:10D02000C080D180E280F380F5E0F594E794D79456
:10D03000C794FA95D1F79B01AC010E9462D42B01F1
:10D040003C01A5019401C701B6010E9462D4461AB1
:10D05000570A680A790AF12C4114510461047104D9
:10D0600009F442C0D301C20188279927AA27B07EBC
:10D07000892B8A2B8B2B09F4FAC01414150416047F
:10D08000170494F5C301BB2797FDB095AB2F36E08D
:10D090003F15A8F40E948664AA2797FDA095BA2F91
:10D0A000DC01992788272F2D30E02650310904C054
:10D0B000B595A795979587952A95D2F718C00E94A0
:10D0C0008664AA2797FDA095BA2FDC0199278827A7
:10D0D00026E030E02F19310904C0880F991FAA1FDC
:10D0E000BB1F2A95D2F703C080E090E0DC012981C4
:10D0F0003A814B815C81281739074A075B0744F462
:10D10000F101E05BFF4F80819181A281B38191C0E9
:10D11000F801E45BFF4F6081718182819381FCE0C3
:10D120009595879577956795FA95D1F7F101E85A26
:10D13000FF4F80809180A280B380B094A09490949F
:10D140008094811C911CA11CB11CA6E0B594A794ED
:10D1500097948794AA95D1F7F101EC5AFF4FC080BC
:10D16000D180E280F380B5E0F594E794D794C7943A
:10D17000BA95D1F79B01AC010E9462D42B013C010E
:10D18000A5019401C701B6010E9462D493018201F6
:10D19000061B170B280B390BB901A80110E041152C
:10D1A00051056105710509F441C0DB01CA018827F9
:10D1B0009927AA27B07E892B8A2B8B2B09F460C074
:10D1C00014161506160617068CF5CB01BB2797FD1E
:10D1D000B095AB2F1730A8F00E948664AA2797FD60
:10D1E000A095BA2FDC0199278827212F30E02650FF
:10D1F000310904C0B595A795979587952A95D2F7DB
:10D2000018C00E948664AA2797FDA095BA2FDC015A
:10D210009927882726E030E0211B310904C0880FB8
:10D22000991FAA1FBB1F2A95D2F703C080E090E088
:10D23000DC01F101E45BFF4F80839183A283B38320
:10D2400010C0F101E45BFF4F29813A814B815C8181
:10D250002083318342835383F101ED58FF4F81E0F6
:10D260008083F101E45AFF4F81E0808312C022E005
:10D27000440C551C661C771C2A95D1F7F394ECCE10
:10D2800092E0440F551F661F771F9A95D1F71F5FD5
:10D2900086CF0F900F900F900F90DF91CF911F913D
:10D2A0000F91FF90EF90DF90CF90BF90AF909F9045
:10D2B0008F907F906F905F904F903F902F90089548
:10D2C000FF920F931F93CF93DF931091870D8FB72A
:10D2D000F8940091860D8FBF60E070E0A7E7FA2E0A
:10D2E0000DC0111101C010E11150F19EE001112497
:10D2F000C857D24FCE010E949767BE011013F1CFDD
:10D30000DF91CF911F910F91FF9008952F923F923F
:10D310004F925F926F927F928F929F92AF92BF9245
:10D32000CF92DF92EF92FF920F931F93CF93DF93F1
:10D3300000D000D0CDB7DEB71C018B01009709F4F7
:10D3400072C1FB01EE58FF4F8081882309F46BC145
:10D35000F101E35AFF4F8081811165C1F101ED5860
:10D36000FF4F8081882309F45EC1F101E45BFF4F28
:10D3700080819181A281B381FB01E45BFF4F4080FA
:10D3800051806280738084159505A605B7050CF061
:10D390004AC1BC01CD01ECE09595879577956795DD
:10D3A000EA95D1F7F101E85AFF4F80809180A28081
:10D3B000B380F6E0B594A79497948794FA95D1F743
:10D3C000F101EC5AFF4FC080D180E280F380A5E0EC
:10D3D000F594E794D794C794AA95D1F79B01AC0133
:10D3E0000E9462D469837A838B839C83A501940114
:10D3F000C701B6010E9462D429813A814B815C81C8
:10D40000620F731F841F951FF12C61157105810533
:10D41000910509F444C0812C912CA12C50EEB52E1D
:10D4200086229722A822B92289288A288B2809F4E3
:10D43000E8C016161706180619068CF5BB2797FDC7
:10D44000B095AB2F36E03F15A8F40E948664AA275A
:10D4500097FDA095BA2FDC01992788272F2D30E062
:10D460002650310904C0B595A795979587952A95BB
:10D47000D2F718C00E948664AA2797FDA095BA2FFC
:10D48000DC019927882726E030E02F19310904C0F4
:10D49000880F991FAA1FBB1F2A95D2F703C080E0EF
:10D4A00090E0DC01481659066A067B0644F4F80150
:10D4B000E45BFF4F80819181A281B38188C0F1013B
:10D4C000E45BFF4F6081718182819381FCE09595DF
:10D4D000879577956795FA95D1F7F101E85AFF4F4F
:10D4E0004080518062807380A6E075946794579461
:10D4F0004794AA95D1F7F101EC5AFF4FC080D18033
:10D50000E280F380B5E0F594E794D794C794BA9598
:10D51000D1F79B01AC010E9462D44B015C01A301D5
:10D520009201C701B6010E9462D4680D791D8A1D5F
:10D530009B1DB12C611571058105910509F444C04D
:10D54000C12CD12CE12CE0EEFE2EC622D722E822FF
:10D55000F922CD28CE28CF2809F45CC0161617066C
:10D56000180619068CF5BB2797FDB095AB2F46E042
:10D570004B15A8F40E948664AA2797FDA095BA2FA0
:10D58000DC01992788274B2D50E04650510904C0F3
:10D59000B595A795979587954A95D2F718C00E949B
:10D5A0008664AA2797FDA095BA2FDC0199278827C2
:10D5B00026E030E02B19310904C0880F991FAA1FFB
:10D5C000BB1F2A95D2F703C080E090E0DC01F80190
:10D5D000E45BFF4F40815181628173814817590795
:10D5E0006A077B0701F180839183A283B383F801EB
:10D5F000E45AFF4F81E08083F801ED58FF4F8083AC
:10D6000012C022E0660F771F881F991F2A95D1F755
:10D61000F394FBCEB2E0660F771F881F991FBA956F
:10D62000D1F7B39487CF0F900F900F900F90DF91A9
:10D63000CF911F910F91FF90EF90DF90CF90BF900F
:10D64000AF909F908F907F906F905F904F903F90A2
:10D650002F9008950F931F93CF93DF931091860D12
:10D6600080E090E007E70DC0019FE0011124C8575A
:10D67000D24FBE010E9486691F5F103109F410E08D
:10D68000CE012091870D1213EFCFDF91CF911F9123
:10D690000F9108958F929F92AF92BF92CF92DF9297
:10D6A000EF92FF920F931F93CF93DF939090860D8D
:10D6B000C0E0D0E0B7E78B2E53C0899C5001112405
:10D6C00088E89DE0A80EB91E209709F443C0FE012A
:10D6D000EE58FF4F80818823E9F1F501EE58FF4FA6
:10D6E00080818823B9F1FE01E45AFF4F80818111C6
:10D6F00006C0F501E45AFF4F8081882359F18E015D
:10D70000085B1F4FF8012081318142815381F5016F
:10D71000E45BFF4F60817181828193810E94CCD450
:10D720006B017C01F8012081318142815381FE012E
:10D73000E45BFF4F60817181828193810E94CCD430
:10D74000AB01BC0197018601CE010E949A64C45AC4
:10D75000DF4F18829394F0E19F1201C0912CE501F4
:10D760008091870D9812A9CF2097D1F0FE01E85B38
:10D77000FF4F2081318142815381FE01E45BFF4FE5
:10D7800060817181828193810E94CCD4AB01BC0104
:10D790008A019B01CE010E949A64C45ADF4F18820D
:10D7A000DF91CF911F910F91FF90EF90DF90CF907D
:10D7B000BF90AF909F908F9008950E9460690E94E3
:10D7C0002A6B0C944A6B0F931092870D1092860D62
:10D7D00010920D1510920E1510920F151092101533
:10D7E0001092111510921215109213151092141513
:10D7F00010921515109216151092171510921815F3
:10D800001092191510921A1510921B1510921C15D2
:10D8100010921D1510921E1510921F1510922015B2
:10D8200060937415709375158093761590937715A2
:10D8300020937015309371154093721550937315A2
:10D840000093F81481E0809306020F9108952F92BF
:10D850003F924F925F926F927F928F929F92AF9280
:10D86000BF92CF92DF92EF92FF920F931F93CF93CD
:10D87000DF93CDB7DEB7C154D1090FB6F894DEBF40
:10D880000FBECDBF4B015C015CA34BA33DA72CA7F2
:10D8900080918C1590918D15892B41F09091870D79
:10D8A0008091860D981711F40C9419754090870D8E
:10D8B000142D1F5F1EA7103109F41EA68091870D3D
:10D8C00027E7829F1001112448E85DE0240E351EF1
:10D8D000F101EC58FF4F1082F101EE58FF4F008329
:10D8E000D101DA96EC92DA978FB7F894C0900D15C3
:10D8F000D0900E15E0900F15F0901015F101C08E2C
:10D90000D18EE28EF38E0091111510911215209197
:10D910001315309114155C960D931D932D933C9324
:10D920005F974090151550901615609017157090E0
:10D9300018154FA658AA69AA7AAA90964D925D9298
:10D940006D927C9293974090191550901A156090A3
:10D950001B1570901C154BAA5CAA6DAA7EAA949602
:10D960004D925D926D927C92979740901D155090CC
:10D970001E1560901F15709020154FAA58AE69AE05
:10D980007AAE98964D925D926D927C929B978FBFE6
:10D9900040903F1550904015609041157090421591
:10D9A0004F8A588E698E7A8E4D925D926D927C92DE
:10D9B0001397409043155090441560904515709012
:10D9C00046154F8E58A269A27AA214964D925D9286
:10D9D0006D927C9217974090471550904815609033
:10D9E000491570904A154FA258A669A67AA61896AE
:10D9F0004D925D926D927C921B9740914B15509188
:10DA00004C1560914D1570914E154487558766876A
:10DA1000778780914F1590915015A0915115B09135
:10DA20005215808B918BA28BB38B409054155090E4
:10DA300055156090561570905715448A558A668A18
:10DA4000778AEB58FF4F7090531570824F88588C2F
:10DA5000698C7A8C452846284728D9F44F8C58A0E1
:10DA600069A07AA045284628472899F44FA058A4D1
:10DA700069A47AA445284628472859F44115510538
:10DA80006105710541F4E1E0EBA70097A105B1053F
:10DA900021F41BA602C0F1E0FBA7F10110AE4090FB
:10DAA000F9145090FA146090FB147090FC144C140C
:10DAB0005D046E047F041CF4FF24F394F0AEC09068
:10DAC000FD14D090FE14E090FF14F0900015C016E5
:10DAD000D106E206F30624F4F10120AD226020AF66
:10DAE0000091011510910215209103153091041534
:10DAF0004FA458A869A87AA8041515052605370566
:10DB000024F4F10120AD246020AF0091051510919F
:10DB1000061520910715309108154BA85CA86DA833
:10DB20007EA8041515052605370524F4F10120AD5E
:10DB3000286020AF0091091510910A1520910B154E
:10DB400030910C154FA858AC69AC7AAC041515058A
:10DB50002605370524F4F10120AD206120AF4115E1
:10DB600051056105710541F00097A105B10509F066
:10DB700009C0F10111AE0BC00097A105B10511F06C
:10DB800021E003C0ECA5FDA52081F10121AF4F8864
:10DB9000588C698C7A8C45284628472829F0209192
:10DBA000E11521602093E115CF8CD8A0E9A0FAA05F
:10DBB000CD28CE28CF2829F02091E115226020938E
:10DBC000E115EFA0F8A409A51AA5EF28E02AE12A9B
:10DBD00029F02091E11524602093E115452B462B77
:10DBE000472B29F02091E11528602093E115892B1E
:10DBF0008A2B8B2B29F08091E11580618093E115B0
:10DC00008091E115F101EA58FF4F80839091F8145B
:10DC1000992311F0846080836091870D8091860D37
:10DC2000681B6F70462E512C58A24F8E452841F527
:10DC30001092C6151092C7151092C8151092C915EA
:10DC40001092CA151092CB151092CC151092CD15CA
:10DC50001092CE151092CF151092D0151092D115AA
:10DC60001092D2151092D3151092D4151092D5158A
:10DC70001092D6151092D7151092D8151092D9156A
:10DC8000EBA1FCA180819181A281B3818101025A23
:10DC90001F4FF80180839183A283B38320918C1559
:10DCA00030918D152115310509F443C0809106028C
:10DCB000882341F04F8C58A042165306D4F110929D
:10DCC000060237C06F8C78A06216730694F5A30124
:10DCD0004230510574F1C901AA2797FDA095BA2FCA
:10DCE000AC0133272227862F90E0A0E0B0E0772711
:10DCF00066270E94CCD46B017C019B01AC01C5015D
:10DD0000B4010E9462D44B015C01F80180819181D1
:10DD1000A281B38177276627A70196010E9462D46A
:10DD2000BB2797FDB095AB2FF80180839183A28329
:10DD3000B38381149104A104B10409F45FC0F1011B
:10DD4000EC5AFF4F4BA44420C1F0D101D9969C91CD
:10DD500004E0909FD0011124A859BA4E8D919D9155
:10DD60000D90BC91A02DB7FF10C0B095A0959095D7
:10DD700081959F4FAF4FBF4F08C08091581590912C
:10DD80005915A0915A15B0915B1580839183A28398
:10DD9000B383F101EC5AFF4F2081318142815381DD
:10DDA00060E070E081E090E00E94CCD46B017C01E7
:10DDB0009B01AC01C501B4010E9462D42B013C015E
:10DDC0000CE515E19E012F5F3F4F388F2F8BD80157
:10DDD0006D917D918D919D918D01A30192010E9484
:10DDE00062D4EF89F88D6193719381939193F88F49
:10DDF000EF8BF5E100371F0751F703C0C12CD12C81
:10DE00007601F101EE58FF4F8081811120C1EBA115
:10DE1000FCA180819181A281B381F101E25AFF4F7F
:10DE200080839183A283B38389288A288B2809F46D
:10DE300091C08E010F5F1F4F62E9A62E65E1B62EDD
:10DE40004E01F5E18F0E911C412C512C320163944F
:10DE5000D8013C9111962C91119712969C91129792
:10DE600013968C910C5F1F4FC32ED22EE92EF82EE5
:10DE7000F7FE08C0F094E094D094C094C11CD11C6B
:10DE8000E11CF11CF50160817181828193816C1527
:10DE90007D058E059F05A4F4A70196010E94CCD4B0
:10DEA00046165706680679065CF0D5016D917D919E
:10DEB0008D919C91A70196010E94CCD42B013C012D
:10DEC000B4E0AB0EB11C0815190511F6EBA1FCA1CD
:10DED00080819181A281B3818101025A1F4F8115F6
:10DEE0009048A105B10510F1F80180819181A281CE
:10DEF000B38124E0B695A795979587952A95D1F794
:10DF000080839183A283B38377276627A30192013D
:10DF10000E9462D4BB2797FDB095AB2F54E0880FC9
:10DF2000991FAA1FBB1F5A95D1F70FC0F801808116
:10DF30009181A281B38177276627A30192010E9474
:10DF400062D4BB2797FDB095AB2FF80180839183F6
:10DF5000A283B383D1019C961D921D921D921C92A7
:10DF60009F9754968D919D910D90BC91A02D0196F7
:10DF7000A11DB11DF10180AB91ABA2ABB3ABE25AD5
:10DF8000FF4F6081718182819381F101EE59FF4FD2
:10DF90009B01AC010E9431D860837183828393839B
:10DFA0004EA44092870D2FB7F8948091F914909168
:10DFB000FA14A091FB14B091FC1480930D1590936A
:10DFC0000E15A0930F15B09310158091FD1490912C
:10DFD000FE14A091FF14B091001580931115909339
:10DFE0001215A0931315B0931415809101159091FB
:10DFF0000215A0910315B091041580931515909307
:10E000001615A0931715B0931815809105159091CA
:10E010000615A0910715B0910815809319159093D6
:10E020001A15A0931B15B0931C158091091590919A
:10E030000A15A0910B15B0910C1580931D159093A6
:10E040001E15A0931F15B09320152FBF66C55BA4A6
:10E05000511035C06F8C78A0672889F58091211503
:10E0600090912215A0912315B09124151816190628
:10E070001A061B0624F581010C5A1F4FD8016D9119
:10E080007D918D919C911616170618061906BCF401
:10E09000181419041A041B0494F4A50194010E9495
:10E0A000CCD4209121153091221540912315509107
:10E0B000241562177307840795070CF4BFC4F10198
:10E0C000E25AFF4F6081718182819381F101EE59A3
:10E0D000FF4F9B01AC010E9431D860837183828322
:10E0E0009383F101E85BFF4F80829182A282B38229
:10E0F000F10184899589A689B7898115F0E89F0780
:10E10000A105B10568F0A7019601220F331F441F36
:10E11000551FB595A795979587957727662704C0CE
:10E1200077276627A70196010E9462D42B013C0144
:10E13000F101E259FF4F9301552737FD5095452FC7
:10E14000CBA4CC2079F06091AA157091AB15809189
:10E15000AC159091AD150E9431D860837183828394
:10E160009383F0C06091AE157091AF158091B0159A
:10E170009091B1150E9431D860837183828393831B
:10E180003CAE2BAE08E715E118A70FA327E235E157
:10E190003CAB2BABFDA7ECA7ABADBCAD6D917D91BE
:10E1A0008D919D91BCAFABAF6F8B788F898F9A8F1C
:10E1B000672B682B692B09F4B6C0D1015496CD901A
:10E1C000DD90ED90FC905797CFA6D8AAE9AAFAAABD
:10E1D000EBA9FCA94081518162817381AFA1B8A5EF
:10E1E0004C155D056E057F0510F1CD90DD90ED902D
:10E1F000FC90ECA5FDA560817181828193812F89BE
:10E20000388D498D5A8D0E9431D84B015C01A70190
:10E2100096016FA578A989A99AA90E9431D8681595
:10E2200079058A059B0508F07EC0DF0177C0CD9097
:10E23000DD90ED90FC90CFAAD8AEE9AEFAAECF88D3
:10E24000D88CE98CFA8CFF0CCC08DC2C7601CBA2A4
:10E25000DCA2EDA2FEA2ACA5BDA50D911D912D9154
:10E260003C9158016901E12CF12C00E010E02F896C
:10E27000388D498D5A8D6BA1762F862F962F0E944F
:10E2800016D9922E832E4BA35DAF6EAF7FAF219632
:10E290008FAF219722969FAF2297EFA8F8AC09ADD8
:10E2A0001AAD6701780100E010E09801CF8AD88E9E
:10E2B000E98EFA8E0B8F1C8F2D8F3E8F8FA598A91C
:10E2C000A9A9BAA98C019D015C016901E12CF12C7D
:10E2D00000E010E02F89388D498D5A8D60E070E0A4
:10E2E00080E090E00E9416D959016A017B018C01FF
:10E2F000292D382D4BA15DAD6EAD7FAD21968FAD33
:10E30000219722969FAD22970E9418DA61F058F06B
:10E31000CFA8D8ACE9ACFAACACA5BDA5CD92DD9246
:10E32000ED92FC921397EFA1F8A53496F8A7EFA30E
:10E330000BA91CA90C5F1F4F1CAB0BABEC58F54194
:10E3400009F02ACFF101E259FF4F80819181A2812A
:10E35000B381811520E89207A105B10528F477273C
:10E360006627A301920117C0009732E0A307B10509
:10E37000C0F4A3019201E2E05595479537952795A2
:10E38000EA95D1F7F2E0B595A79597958795FA9517
:10E39000D1F7772766270E94CCD4F101E85AFF4FC6
:10E3A00038C08101085A1F4F009748E0A407B10503
:10E3B000D8F4A3019201F4E0559547953795279538
:10E3C000FA95D1F764E0B595A795979587956A95E5
:10E3D000D1F7772766270E94CCD4D8016D937D931F
:10E3E0008D939C93139719C0A301920165E05595F5
:10E3F0004795379527956A95D1F775E0B595A79517
:10E40000979587957A95D1F7772766270E94CCD480
:10E41000F8016083718382839383F101E259FF4F96
:10E4200080819181A281B3816C017D0100E010E0C7
:10E4300098018F8BD88EE98EFA8E0B8F1C8F2D8FC3
:10E440003E8FAFEDAA2EB8E1BB2E12E0C12ED12C2B
:10E45000E12CF12C00E010E02F89388D498D5A8D88
:10E4600060E070E080E090E00E9416D90EE00E942B
:10E4700009DAD101D4962C93D497D5963C93D597AD
:10E48000D6964C93D697D7965C93F101E85BFF4FF5
:10E490004F8C58A04528B9F460918E1570918F1556
:10E4A000809190159091911560933B1570933C1558
:10E4B00080933D1590933E15208131814281538197
:10E4C0000E94CCD4E2C280819181A281B38140912B
:10E4D000A6155091A7156091A8157091A915481718
:10E4E00059076A077B076CF080933B1590933C15A6
:10E4F000A0933D15B0933E1560E070E081E090E0A0
:10E50000C4C28E010F5F1F4F26EC35E138A72FA341
:10E5100042E955E158A34F8FBE016B5E7F4F7E8B62
:10E520006D8B3CA32BA3188F0F8B412C512C3201E8
:10E530006394AF89B88D2D913D914D915D91B88FC8
:10E54000AF8BEBA1FCA181919191A191B191FCA321
:10E55000EBA32115310541055105D9F1EF8DF8A146
:10E56000C080D180E280F38049015A01881A990A5B
:10E57000AA0ABB0AB7FE08C0B094A09490948094F5
:10E58000811C911CA11CB11CC814D904EA04FB0411
:10E5900004F582179307A407B5073CF4BC01CD012D
:10E5A0006C0D7D1D8E1D9F1D06C0BC01CD016C191B
:10E5B0007D098E099F090E94CCD4161617061806ED
:10E5C0001906F4F4641575058605970514F42B01F6
:10E5D0003C012F8D38A12C5F3F4F38A32F8FCF8860
:10E5E000D88CED88FE88CE14DF0409F0A2CFC301D9
:10E5F000B2014114510421E06206710479F103C0B3
:10E60000412C512C3201F101E85BFF4F6081718197
:10E6100082819381A30192010E9462D460933B1591
:10E6200070933C1580933D1590933E15D8016D91E4
:10E630007D918D919D918D01A30192010E9462D4E3
:10E64000EFA1F8A56193719381939193F8A7EFA33C
:10E65000CD88DE880C151D0549F710C0F101E85B77
:10E66000FF4F008111812281338100933B1510936C
:10E670003C1520933D1530933E1507C260918E15D1
:10E6800070918F1580919015909191154CE0959512
:10E690008795779567954A95D1F7F101E85AFF4F2D
:10E6A00080809180A280B38056E0B594A79497941F
:10E6B00087945A95D1F7F101EC5AFF4FC080D18071
:10E6C000E280F380E5E0F594E794D794C794EA9567
:10E6D000D1F79B01AC010E9462D46F8B788F898F38
:10E6E0009A8FA5019401C701B6010E9462D4EF88F8
:10E6F000F88C098D1A8D6E0D7F1D801F911F10E003
:10E70000611571058105910509F443C0C12CD12C17
:10E71000E12C30EEF32EC622D722E822F922CD28B2
:10E72000CE28CF2809F4F0C11616170618061906C8
:10E7300084F5BB2797FDB095AB2F1730A8F00E944A
:10E740008664AA2797FDA095BA2FDC019927882710
:10E75000212F30E02650310904C0B595A795979533
:10E7600087952A95D2F718C00E948664AA2797FD3C
:10E77000A095BA2FDC019927882726E030E0211BDD
:10E78000310904C0880F991FAA1FBB1F2A95D2F711
:10E7900003C080E090E0DC0140913B1550913C15B6
:10E7A00060913D1570913E15C0908E15D0908F15DB
:10E7B000E0909015F09091159101245B3F4F8101FD
:10E7C000005B1F4FF9014C155D056E057F0554F484
:10E7D000C082D182E282F382F801C082D182E282D9
:10E7E000F38209C04083518362837383F8014083BD
:10E7F000518362837383F101E85BFF4F4081518154
:10E8000062817381F101E35AFF4F84179507A607D0
:10E81000B7071CF081E0808301C01082F101E45A47
:10E82000FF4F81E08083F101ED58FF4F1082F1012D
:10E83000E05CFF4F1082118212821382F101848505
:10E840009585A685B785892B8A2B8B2B41F48089EA
:10E850009189A289B389892B8A2B8B2BD9F0FBA5AF
:10E86000F11118C08091741590917515A0917615CD
:10E87000B0917715892B8A2B8B2B19F58091701508
:10E8800090917115A0917215B0917315892B8A2BF7
:10E890008B2BB9F4D101DB961C92DB97DD961C9291
:10E8A0001E92DC97DF961C921E92DE97F101EC5BC4
:10E8B000FF4F11821082F101EA5BFF4F118210823B
:10E8C00003C081E0F10183AF93018201B301A20192
:10E8D000C1010E949A644EA44092870D2FB7F8940C
:10E8E0008091F9149091FA14A091FB14B091FC144A
:10E8F00080930D1590930E15A0930F15B0931015DE
:10E900008091FD149091FE14A091FF14B091001518
:10E910008093111590931215A0931315B0931415AD
:10E920008091011590910215A0910315B0910415E5
:10E930008093151590931615A0931715B09318157D
:10E940008091051590910615A0910715B0910815B5
:10E950008093191590931A15A0931B15B0931C154D
:10E960008091091590910A15A0910B15B0910C1585
:10E9700080931D1590931E15A0931F15B09320151D
:10E980002FBF0E94DD6BF10180859185A285B38543
:10E99000892B8A2B8B2B09F4C0C0809126158823E4
:10E9A00009F4BBC02091251580E991E0289FA001C2
:10E9B000299F500D1124662757FD6095762F809171
:10E9C000011590910215A0910315B09104158417BB
:10E9D0009507A607B7070CF4A0C01092261587E08C
:10E9E00090E00E94CCA381EB9AE00E944FA489E0C2
:10E9F00090E00E94CCA361E070E081E0CF5BDF4F4C
:10EA00000FB6F894DEBF0FBECDBFDF91CF911F913F
:10EA10000F91FF90EF90DF90CF90BF90AF909F90BD
:10EA20008F907F906F905F904F903F902F900C94BD
:10EA30007C3A81E0809306020C94566CD8016D916B
:10EA40007D918D919C910E94CCD42B013C01A5011C
:10EA500094010E94CCD49B01AC018101025A1F4F4A
:10EA6000F80180819181A281B381772766270E9476
:10EA700062D4BB2797FDB095AB2FF80180839183BB
:10EA8000A283B383420153011ACB09811A812B81DE
:10EA90003C810093C6151093C7152093C815309379
:10EAA000C9150D811E812F8138850093CA151093D9
:10EAB000CB152093CC153093CD1509851A852B8560
:10EAC0003C850093CE151093CF152093D01530932D
:10EAD000D1150D851E852F8538890093D215109389
:10EAE000D3152093D4153093D51509891A892B890C
:10EAF0003C890093D6151093D7152093D8153093E1
:10EB0000D9152B013C01BACD02E0660F771F881F93
:10EB1000991F0A95D1F71F5FF3CDCF5BDF4F0FB67B
:10EB2000F894DEBF0FBECDBFDF91CF911F910F9143
:10EB3000FF90EF90DF90CF90BF90AF909F908F901D
:10EB40007F906F905F904F903F902F9008958093AB
:10EB5000261560E080E592E00E94729D8093251565
:10EB600008958091261508958093261508950F9392
:10EB70001F93CF93CFB7F894FC0180819181A2813C
:10EB8000B38180930D1590930E15A0930F15B0933C
:10EB90001015FB0180819181A281B38180931115B1
:10EBA00090931215A0931315B0931415FA01808158
:10EBB0009181A281B3818093151590931615A0932E
:10EBC0001715B0931815F90180819181A281B38145
:10EBD0008093191590931A15A0931B15B0931C15CB
:10EBE000F80180819181A281B38180931D1590935A
:10EBF0001E15A0931F15B09320158091870D90913D
:10EC0000860D891B8F7061F40DE115E129E135E175
:10EC100045E155E161E175E18DE095E10E945563C3
:10EC2000CFBFCF911F910F91089540E06DE57AE13C
:10EC30008AED95E10C944CD02F923F924F925F92C7
:10EC40006F927F928F929F92AF92BF92CF92DF92FC
:10EC5000EF92FF920F931F93CF93DF93CDB7DEB761
:10EC600067970FB6F894DEBF0FBECDBF898B8823A0
:10EC7000B1F060E082E090E00E94729DF82E60E0CA
:10EC800084E090E00E94729D8E8360E08EE092E0CE
:10EC90000E94729D813729F00E94B83502C01E8201
:10ECA000F12C8FEF95E19F8B8E8B07E012E090E2C5
:10ECB000892E92E0992EA2E1B2E0B887AF83EBE013
:10ECC000F2E0FA87E98789E192E09D838C8327E26D
:10ECD000222E22E0322EA3E7B3E0BC87AB87E6E426
:10ECE000F2E0FE87ED87A12CB12C1B821A82C12C89
:10ECF000D12C8F2D90E09B8B8A8BEE24E394F12C0A
:10ED0000BE81AB2FB0E0BD8BAC8BC982E989EE230D
:10ED100009F491C1FE81F7FF0AC08C899D890C2CF2
:10ED200002C0959587950A94E2F7817001C081E051
:10ED3000AE89BF898C93EA81FB81E150FA4EF88B52
:10ED4000EF878A899B890C2C02C0959587950A9438
:10ED5000E2F781708183F501E15AFC4F40815181D6
:10ED600062817381C5018C559E4F0E94B29D0E94A5
:10ED7000C8D620E034E244E759E40E94F5D5AE89D4
:10ED8000BF8912966D937D938D939C931597EB8518
:10ED9000FC85608171818D859E850E948F9DBC015F
:10EDA00080E090E00E94C8D6AE89BF8916966D9328
:10EDB0007D938D939C931997F501E358FC4F408107
:10EDC000518162817381C501805F9D4F0E94B29D18
:10EDD0000E94CAD6EE89FF89228133814481558100
:10EDE0000E94CED720E030E04AE754E40E94CED71C
:10EDF0000E9497D628EE33E040E050E00E9497D87A
:10EE000029013A01F981F23011F118F0F53008F4D6
:10EE100043C0C301B20122E030E040E050E00E9474
:10EE200097D8AE89BF8950962D933D934D935C93AF
:10EE3000539788279927DC01821B930BA40BB50BF2
:10EE4000EE89FF8984879587A687B78737C040E01A
:10EE500050E0BA01C5018C5D9D4F0E94B29D0E9499
:10EE6000C8D6AE89BF8912962D913D914D915C9186
:10EE700015970E94CED70E9497D6461A570A680A5D
:10EE8000790AEE89FF89408A518A628A738A1486D8
:10EE900015861686178612C0EE89FF89208B318B66
:10EEA000428B538B7094609450944094411C511C3D
:10EEB000611C711C4486558666867786D8011C962F
:10EEC000ED91FC911D972081C701AF81B8850C9011
:10EED00002C0880F991F0A94E2F7282B2083D801DB
:10EEE0001596ED91FC9116972081C701A985BA85E9
:10EEF0000C9002C0880F991F0A94E2F7282B2083F8
:10EF0000D8011E96ED91FC911F972081C701AC811D
:10EF1000BD810C9002C0880F991F0A94E2F7282B3C
:10EF20002083D8015396ED91FC9154972081C7011D
:10EF3000AC81BD810C9002C0880F991F0A94E2F742
:10EF4000282B2083F801848D958D892B81F101A0D8
:10EF5000F2A1E02D2081C701D1010C9002C0880FE1
:10EF6000991F0A94E2F7809582238083EE89FF89B6
:10EF70008081D8015C96ED91FC915D97208188237A
:10EF800059F0C701D1010C9002C0880F991F0A9453
:10EF9000E2F7282B20830BC0C701D1010C9002C0DF
:10EFA000880F991F0A94E2F7809582238083F801E5
:10EFB00085899689892B81F1028CF38DE02D208142
:10EFC000C701D4010C9002C0880F991F0A94E2F780
:10EFD000809582238083EE89FF898081D8015596B0
:10EFE000ED91FC9156972081882359F0C701D401F7
:10EFF0000C9002C0880F991F0A94E2F7282B2083F7
:10F000000BC0C701D4010C9002C0880F991F0A944D
:10F01000E2F7809582238083F601EE0FFF1FEE0F4B
:10F02000FF1FE551FA4E1082118212821382EF8582
:10F03000F88912861386F601EA51FA4E1082EA81A7
:10F04000FB81E150FA4E81E09981933008F480E031
:10F05000818FAE89BF895D961D921D921D921C9273
:10F060009097B1E0B28F138E148AEE89FF89158ACA
:10F07000168A178A108EDF0111A212A213A214A2FF
:10F0800015A216A217A210A6FFEFCF1ADF0A8A81D7
:10F090009B8189969B838A839996BF8BAE8B0D5DEE
:10F0A0001F4FB3E28B0E911CEF81F885B396F88762
:10F0B000EF8389859A8583969A878987AC81BD81FC
:10F0C0009396BD83AC83B3E22B0E311CE4E0AE0E0D
:10F0D000B11C8B859C8502969C878B87AD85BE85F0
:10F0E0001296BE87AD87B5E0CB16D10409F00DCEE0
:10F0F000E989EE2321F01092E1151092E0151092AB
:10F10000E3151092E2151092E5151092E41567963A
:10F110000FB6F894DEBF0FBECDBFDF91CF911F9128
:10F120000F91FF90EF90DF90CF90BF90AF909F90A6
:10F130008F907F906F905F904F903F902F900895A9
:10F1400099E2899FF0011124E150FA4EDF011296F5
:10F15000528111964C91119712963C9112971396E9
:10F160002C91652F742F832F922F0895CF93DF93C7
:10F170001F92CDB7DEB749830E94CAD6498129E2E2
:10F18000429FF0011124E150FA4E228133814481E3
:10F1900055810E94F5D50F90DF91CF9108954F9240
:10F1A0005F926F927F928F929F92AF92BF92CF9217
:10F1B000DF92EF92FF920F931F93CF93DF93142F61
:10F1C00020E030E04AE754E40E94CED70E945DD6AA
:10F1D00029013A014B01D82FC92F89E2189FF0016C
:10F1E0001124E150FA4E62817381848195810E94DD
:10F1F0005DD659016A017B018C019201A301B40122
:10F200008D2F9C2F0E9416D9E8EEAE2EF3E0BF2E74
:10F21000C12CD12CE12CF12C00E010E00E94D9D8B7
:10F22000952FB901842FDF91CF911F910F91FF90FE
:10F23000EF90DF90CF90BF90AF909F908F907F9096
:10F240006F905F904F90089540E06DE57AE18CEC0F
:10F2500096E10C944CD01F93CF93DF93C0E0D0E0A5
:10F260001BE01C9FC0011D9F900D11246C2F895E17
:10F27000984E0E94F39C2196C530D10591F7DF91FD
:10F28000CF911F91089580911617811103C080912D
:10F290001517089581E008956F927F929F92AF9223
:10F2A000BF92CF92DF92EF92FF920F931F93CF9373
:10F2B000DF9300D000D0CDB7DEB79FB6F89408E357
:10F2C00012E0612C712C40E050E0BA01C8010E94AC
:10F2D000B29D6B017C01862D0E94A0789B01AC0140
:10F2E000B30185ED96E129833A834B835C830E94C9
:10F2F000794C5C01C701B6010E94CAD629813A81C6
:10F300004B815C810E94CED720E030E04AE754E494
:10F310000E94F5D50E9497D6F501608371838283A0
:10F320009383FFEF6F1A7F0A0C5F1F4F83E068160D
:10F33000710449F602E010E0B80185ED96E10E9403
:10F34000794CFC0110821182128213820F5F1F4FD1
:10F350000530110589F700E010E0B80189EE96E16B
:10F360000E94794CFC0110821182128213820F5F7D
:10F370001F4F0530110589F79FBE0F900F900F901A
:10F380000F90DF91CF911F910F91FF90EF90DF9041
:10F39000CF90BF90AF909F907F906F900895109204
:10F3A00016171092151781E00E941C760E942B7987
:10F3B0004FEF5FEFBA0188E392E00E94B29D6F3F8A
:10F3C0007F4F8F4F9F4F11F40C941D3508957F92FE
:10F3D0008F929F92AF92BF92CF92DF92EF92FF9265
:10F3E0000F931F93CF93DF93CDB7DEB764970FB61C
:10F3F000F894DEBF0FBECDBF44E1FC019E012F5F3C
:10F400003F4FD90101900D924A95E1F78AE0E82E2D
:10F4100086E1F82E00E010E077247394D22EC32EFC
:10F42000F7017082B8018091D3169091D4160E9492
:10F43000794CFC0180809180A280B380B8018D2D31
:10F440009C2D0E94794CFC01408151816281738125
:10F45000480D591D6A1D7B1D408351836283738350
:10F460000F5F1F4FF9E2EF0EF11C05301105C1F6D9
:10F4700064E070E08D2D9C2D0E94794C8C0163E03E
:10F4800070E08D2D9C2D0E94794C4C0162E070E063
:10F490008D2D9C2D0E94794C5C0161E070E08D2DDA
:10F4A0009C2D0E94794C7C0160E070E08D2D9C2D9C
:10F4B0000E94794C9401A501B7010E94B77564962A
:10F4C0000FB6F894DEBF0FBECDBFDF91CF911F9175
:10F4D0000F91FF90EF90DF90CF90BF90AF909F90F3
:10F4E0008F907F900895AF92BF92CF92DF92EF926C
:10F4F000FF920F931F93CF93DF93CDB7DEB764973F
:10F500000FB6F894DEBF0FBECDBF24E1FC01DE01D3
:10F51000119601900D922A95E1F781E080930A16E9
:10F520008093331680935C16809385168093AE1675
:10F5300064E070E0CE0101960E94794C8C0163E09A
:10F5400070E0CE0101960E94794C5C0162E070E0AF
:10F55000CE0101960E94794C6C0161E070E0CE0111
:10F5600001960E94794C7C0160E070E0CE0101962A
:10F570000E94794C9501A601B7010E94B775649667
:10F580000FB6F894DEBF0FBECDBFDF91CF911F91B4
:10F590000F91FF90EF90DF90CF90BF90AF900895C4
:10F5A0005F926F927F928F929F92AF92BF92CF9213
:10F5B000DF92EF92FF920F931F93CF93DF93CDB71C
:10F5C000DEB764970FB6F894DEBF0FBECDBF3C0127
:10F5D0000E943C4C5FB6F8948090191590901A15D3
:10F5E000A0901B15B0901C15C0901515D090161545
:10F5F000E0901715F0901815009111151091121543
:10F60000209113153091141540910D1550910E1540
:10F6100060910F1570911015809120158F93809136
:10F620001F158F9380911E158F9380911D158F93B9
:10F63000CE0101960E943D4C84E1FE013196D3013A
:10F6400001900D928A95E1F70F900F900F900F9017
:10F6500000E010E0B8018091D3169091D4160E947A
:10F66000794CFC01C080D180E280F380B801C301F5
:10F670000E94794CFC0140815181628173814C1957
:10F680005D096E097F0940835183628373830F5F35
:10F690001F4F05301105F1F65FBEC30164960FB62A
:10F6A000F894DEBF0FBECDBFDF91CF911F910F91B8
:10F6B000FF90EF90DF90CF90BF90AF909F908F9092
:10F6C0007F906F905F9008956F927F928F929F923C
:10F6D000AF92BF92CF92DF92EF92FF920F931F9360
:10F6E000CF93DF93CDB7DEB765970FB6F894DEBF43
:10F6F0000FBECDBF3C0145E1E42EF12CEC0EFD1E0A
:10F700008E010F5E1F4F9E01235F3F4FAE01475F8B
:10F710005F4FBE016B5F7F4FCE0101960E94A263D7
:10F720008D8981708D8B813029F435EDC32E36E1C2
:10F73000D32E04C029EEC22E26E1D22EEE24E3946D
:10F74000F12CEC0EFD1E00E010E0B801C6010E9495
:10F75000794CF7014081518162817381FC01808184
:10F760009181A281B381481B590B6A0B7B0BF70176
:10F7700041935193619371937F010F5F1F4F053048
:10F78000110519F78D849E84AF84B888C984DA8402
:10F79000EB84FC840D811E812F81388549815A813B
:10F7A0006B817C818C898F938B898F938A898F93CE
:10F7B00089898F93C3010E943D4C0F900F900F9049
:10F7C0000F90C30165960FB6F894DEBF0FBECDBF94
:10F7D000DF91CF911F910F91FF90EF90DF90CF902D
:10F7E000BF90AF909F908F907F906F90089580937F
:10F7F000FF1608954F925F926F927F928F929F9221
:10F80000AF92BF92CF92DF92EF92FF920F931F932E
:10F81000CF93DF93CDB7DEB728970FB6F894DEBF4E
:10F820000FBECDBF6C019A01AB0109EF14E1780165
:10F83000A12CB12CB501C6012D833E834F8358877F
:10F840000E94714CFC014080518062807380B50140
:10F850008091D3169091D4160E94794CFC0180813E
:10F860009181A281B381840D951DA61DB71DF7015D
:10F8700081939193A193B1937F01FFEFAF1ABF0AD8
:10F880002D813E814F81588585E0A816B10491F6FF
:10F89000C0900115D0900215E0900315F09004156A
:10F8A0008091611690916216A0916316B0916416D2
:10F8B000C816D906EA06FB0614F4D701C6018093E0
:10F8C000011590930215A0930315B09304156DE0F4
:10F8D000862E65E1962E6FE375E1B12CA12CC12C2B
:10F8E000D12C7601F80181919191A191B1918F0173
:10F8F000F40141905190619071904F0184199509E4
:10F90000A609B709B7FF07C0B095A0959095819556
:10F910009F4FAF4FBF4FFB0181939193A193B19341
:10F92000BF01C816D906EA06FB061CF4AB2C6C0115
:10F930007D01B394F5E0BF12D5CFA0925315C092CC
:10F940005415D0925515E0925615F0925715CD28C2
:10F95000CE28CF2839F160E472E48FE090E00E9475
:10F9600097D829833A834B835C83E090D21600E0DA
:10F9700022ED36E1AE014F5F5F4F60E070E0CB01FA
:10F980000E94276C8091870D9091860D891B8F7046
:10F9900090911417891720F081E08093161702C008
:10F9A0001092161728960FB6F894DEBF0FBECDBF83
:10F9B000DF91CF911F910F91FF90EF90DF90CF904B
:10F9C000BF90AF909F908F907F906F905F904F907F
:10F9D00008952F923F924F925F926F927F928F92F3
:10F9E0009F92AF92BF92CF92DF92EF92FF920F93CE
:10F9F0001F93CF93DF93CDB7DEB72A970FB6F89456
:10FA0000DEBF0FBECDBF5C014F83588769877A8701
:10FA10007DE0272E75E1372E89EF94E19E838D835B
:10FA20007C01610100E010E0822E912CC401002EC7
:10FA300002C0959587950A94E2F780FF0AC0F60107
:10FA40004080518062807380B801C5010E94714C72
:10FA500010C0B801C5010E94714CFC01408051806A
:10FA600062807380B8018091D3169091D4160E9461
:10FA7000794CFC0180819181A281B381840D951D17
:10FA8000A61DB71DF70180839183A283B3830F5F07
:10FA90001F4FF4E0CF0ED11C84E0E80EF11C0530BE
:10FAA000110521F640910115509102156091031541
:10FAB000709104158091611690916216A091631661
:10FAC000B0916416481759076A077B0714F4DB01E5
:10FAD000CA018093011590930215A0930315B0936A
:10FAE00004150FE315E160E070E020E030E0A901CB
:10FAF000ED81FE8181919191A191B191FE83ED8380
:10FB0000F101C190D190E190F1901F018C199D09F4
:10FB1000AE09BF09B7FF07C0B095A0959095819534
:10FB20009F4FAF4FBF4FF80181939193A193B19332
:10FB30008F01281739074A075B071CF4762F9C01B1
:10FB4000AD016F5F6530A1F6709353152093541586
:10FB5000309355154093561550935715211531057F
:10FB60004105510569F16F81788589859A850E94E3
:10FB700097D860E472E48FE090E00E9497D82983E0
:10FB80003A834B835C83E090D21600E022ED36E1AD
:10FB9000AE014F5F5F4F60E070E0CB010E94276CC9
:10FBA0008091870D9091860D891B8F70909114170D
:10FBB000891720F081E08093161702C01092161763
:10FBC0002A960FB6F894DEBF0FBECDBFDF91CF915E
:10FBD0001F910F91FF90EF90DF90CF90BF90AF906B
:10FBE0009F908F907F906F905F904F903F902F905D
:10FBF00008952F923F924F925F926F927F928F92D1
:10FC00009F92AF92BF92CF92DF92EF92FF920F93AB
:10FC10001F93CF93DF93CDB7DEB766970FB6F894F7
:10FC2000DEBF0FBECDBF1C014D875E876F87788B0F
:10FC300047015801DA8AC98A4DE055E15C874B8754
:10FC400089EF94E19A8789873C012A0100E010E05E
:10FC5000422F50E05E834D838D819E81002E02C035
:10FC6000959587950A94E2F780FF0AC0F201C0805B
:10FC7000D180E280F380B801C1010E94714C10C0B4
:10FC8000B801C1010E94714CFC01C080D180E280AA
:10FC9000F380B8018091D3169091D4160E94794CCC
:10FCA000FC0180819181A281B3818C0D9D1DAE1DCF
:10FCB000BF1DF30180839183A283B3830F5F1F4F26
:10FCC000F4E04F0E511C24E0620E711C053011054A
:10FCD00019F640910115509102156091031570912C
:10FCE00004158091611690916216A0916316B091EF
:10FCF0006416481759076A077B0714F4DB01CA0129
:10FD00008093011590930215A0930315B0930415E9
:10FD100010925315AFE32A2EA5E13A2E40E057E1A9
:10FD200058874F830CE515E11D82412C512C32017F
:10FD3000E985FA856191719181919191FA87E987BD
:10FD4000EB85FC85C190D190E190F190FC87EB8729
:10FD50006C197D098E099F09F1016083718382838B
:10FD600093836B017C0197FF07C0CC24DD247601CF
:10FD7000C61AD70AE80AF90AC114F0E8DF06E10456
:10FD8000F10464F4EF81F88520813181428153814F
:10FD9000CB01772766270E9462D424C00E94CAD66E
:10FDA0006B8B7C8B8D8B9E8BEF81F8856081718155
:10FDB000828193810E94CAD620E030E040E857E378
:10FDC0000E94CED79B01AC016B897C898D899E896D
:10FDD0000E94CED720E030E040E857E40E94CED722
:10FDE0000E9497D6F8016083718382839383F10127
:10FDF000C082D182E282F3824C145D046E047F04DF
:10FE00002CF4FD81F09353152601370124E0220ED6
:10FE1000311C3D813F5F3D834F8158854C5F5F4F73
:10FE200058874F830C5F1F4F353009F081CF4092C8
:10FE300054155092551560925615709257154528D5
:10FE40004628472809F459C020E030E0A901C5013F
:10FE5000B4010E94F1D5882309F44FC020E030E0BE
:10FE600040E857E4C501B4010E94CED70E9497D65E
:10FE7000609358157093591580935A1590935B159C
:10FE80002091B602222379F0E989FA89BF018827F7
:10FE900077FD8095982FEAE0660F771F881F991FDE
:10FEA000EA95D1F703C060E070E0CB01E090D21694
:10FEB000222319F00091B70201C000E02D853E8594
:10FEC0004F85588929833A834B835C8322ED36E141
:10FED000AE014F5F5F4F0E94276C8091870D90911C
:10FEE000860D891B8F7090911417891720F081E07F
:10FEF0008093161702C01092161766960FB6F894E4
:10FF0000DEBF0FBECDBFDF91CF911F910F91FF904C
:10FF1000EF90DF90CF90BF90AF909F908F907F90A9
:10FF20006F905F904F903F902F9008952F923F9247
:10FF30004F925F926F927F929F92AF92BF92CF92B9
:10FF4000DF92EF92FF920F931F93CF93DF93CDB782
:10FF5000DEB768970FB6F894DEBF0FBECDBF982E00
:10FF6000A62E1092B7028E010F5F1F4FC8012D8B76
:10FF70003E8B4F8B588F0E94647B89E0C82E86E1B0
:10FF8000D82EE12CF12CB12C302E212E11E0588DE1
:10FF90004F893E892D89C5010E2C02C09595879504
:10FFA0000A94E2F780FD05C0F701EA51FA4E10828B
:10FFB0002BC0B701832D922D2D8B3E8B4F8B588FED
:10FFC0000E94794C2D893E894F89588D992039F0AE
:10FFD00044244A94542C642C0FE3702E05C0412C09
:10FFE000512C612CB0EC7B2EFC014082518262824C
:10FFF0007382F701EA51FA4E1083F2E0EF1202C069
:020000021000EC
:100000001093FE16F6011083FFEFEF1AFF0A89E244
:10001000C80ED11CE5E0EE16F10409F0BCCFBA0120
:10002000A901CE0101960E94FA7B81E08093151709
:1000300068960FB6F894DEBF0FBECDBFDF91CF91AB
:100040001F910F91FF90EF90DF90CF90BF90AF90F6
:100050009F907F906F905F904F903F902F9008956A
:10006000853098F49091E11521E030E0082E01C030
:10007000220F0A94EAF7662321F0922B9093E11560
:100080000895209529232093E11508958091E11585
:100090000895853040F42BE0829FC0011124895ED1
:1000A000984E0C94F89C08958093B702089581703F
:1000B0008093D216813019F485ED96E102C089EE65
:1000C00096E19093D4168093D31608958091690297
:1000D00090916A02892B99F0E0916B02F0916C0289
:1000E000808190E000906D0202C0959587950A94FA
:1000F000E2F7817091E020915116821301C090E0E7
:10010000892F90E0E5E0880F991FEA95E1F72091AB
:10011000620230916302232B99F0E0916402F09126
:100120006502208130E00090660202C03595279577
:100130000A94E2F7217031E040915116241301C076
:1001400030E0232F30E074E0220F331F7A95E1F77F
:10015000282B392B8091460290914702892B99F0E8
:10016000E0914802F0914902808190E000904A02BB
:1001700002C0959587950A94E2F7817091E04091CD
:100180002816841301C090E0892F90E063E0880F67
:10019000991F6A95E1F7822B932B20913F023091B2
:1001A0004002232B99F0E0914102F091420220811C
:1001B00030E00090430202C0359527950A94E2F79B
:1001C000217031E040912816241301C030E0232F24
:1001D00030E0220F331F220F331F282B392B809141
:1001E000230290912402892B99F0E0912502F0914D
:1001F0002602808190E00090270202C095958795A5
:100200000A94E2F7817091E04091FF15841301C0D8
:1002100090E0892F90E0880F991F822B932B2091DB
:100220001C0230911D02232B99F0E0911E02F091E7
:100230001F02208130E00090200202C035952795F2
:100240000A94E2F7217031E04091FF15241301C0B8
:1002500030E0832B08959091B602911101C080E0A7
:100260000C9477640E940064109216171092151770
:1002700080E00E941C768091B6028093B70281E0F4
:100280000C942B812F923F924F925F927F928F928C
:100290009F92AF92BF92CF92DF92EF92FF920F9315
:1002A0001F93CF93DF9380E00E941C760E942B79EE
:1002B0001092FD161092FE160E944C7980E00E946A
:1002C00057806FEF88E891E00E94729D803811F0AE
:1002D0000E94763360E08EE691E00E94729D81700C
:1002E0008093B6028093B70281E00E942B81C0E028
:1002F000D7E110E0812F0E94A0789B01AC0160E063
:1003000070E080E89FE30E94F5D520E030E040E80F
:1003100057E40E94CED70E9497D669937993899328
:1003200099931F5F153031F768EE73E082E791E033
:100330000E948F9DA0E0B0E08093B2159093B3151A
:10034000A093B415B093B51568EE73E084E791E01F
:100350000E948F9DA0E0B0E08093B6159093B715F2
:10036000A093B815B093B91566E970E086E791E0FF
:100370000E948F9DA0E0B0E08093BA159093BB15CA
:10038000A093BC15B093BD1560EA7FE088E791E0CB
:100390000E948F9DA0E0B0E08093BE159093BF15A2
:1003A000A093C015B093C11560EA7FE08AE791E0A1
:1003B0000E948F9DA0E0B0E08093C2159093C3157A
:1003C000A093C415B093C515C2EBD5E1A8E7EA2EFA
:1003D000A5E1FA2E07E215E1712C88248A94982C65
:1003E00054016E01288039804A805B80872D0E94ED
:1003F000A0789B01AC0160EF7FEF8FE799E40E944A
:10040000F5D50E949CD6621573058405950588F480
:10041000872D0E94A0789B01AC0160EF7FEF8FE7F2
:1004200099E40E94F5D50E949CD6688379838A83DB
:100430009B832496F60160817181828193810E9461
:10044000C8D61B012C01872D0E94A0789B01AC010E
:10045000C201B1010E94CED70E949CD69B01AC0183
:10046000F70161937193819391937F01C501B40169
:100470000E9475D8F80121933193419351938F01D4
:100480007394F5E07F12ADCF60ED77E080E791E007
:100490000E948F9DA0E0B0E0813127E29207A10584
:1004A000B10508F404C080E197E2A0E0B0E08093D9
:1004B000AE159093AF15A093B015B093B11560EA47
:1004C0007FE086E891E00E948F9DA0E0B0E081315E
:1004D000E7E29E07A105B10508F404C080E197E2B8
:1004E000A0E0B0E08093AA159093AB15A093AC1553
:1004F000B093AD1560E070E080EE91E00E948F9DBA
:1005000090935A0D8093590D60E070E082EE91E077
:100510000E948F9D90935C0D80935B0D6AE070E06C
:100520008CE791E00E948F9DBC0180E090E00E94EA
:10053000C8D620E030E040E857E40E94CED70E94C1
:1005400097D660939215709393158093941590931A
:1005500095156AE070E08EE791E00E948F9DBC01E6
:1005600080E090E00E94C8D620E030E040E857E408
:100570000E94CED70E9497D66093961570939715D8
:1005800080939815909399156AE070E080E891E067
:100590000E948F9DBC0180E090E00E94C8D620E0C0
:1005A00030E040E857E40E94CED70E9497D660938F
:1005B0009A1570939B1580939C1590939D156EE1F1
:1005C00070E082E891E00E948F9DBC0180E090E0A5
:1005D0000E94C8D620E030E040E857E40E94CED721
:1005E0000E9497D660939E1570939F158093A015D7
:1005F0009093A1156EE170E084E891E00E948F9DD8
:10060000BC0180E090E00E94C8D620E030E040E8E5
:1006100057E40E94CED70E9497D66093A21570939C
:10062000A3158093A4159093A51580919A15909188
:100630009B15A0919C15B0919D15E2E9F5E14191C2
:10064000519161917191481759076A077B0714F41A
:10065000DB01CA0125E1E63AF20789F78093A61586
:100660009093A715A093A815B093A91542E553E060
:1006700060E070E088ED91E00E94B29D0E94C8D6D3
:1006800020E030E543EC57E40E94F5D520E030E06F
:1006900040E857E40E94CED70E9497D67B01D82F1E
:1006A000C92F44E853E060E070E08CED91E00E94D7
:1006B000B29D0E94C8D620E030E543EC57E40E948A
:1006C000F5D520E030E040E857E40E94CED70E9404
:1006D00097D6B62EA72E6C018EE195E0A0E0B0E093
:1006E0008093211590932215A0932315B093241580
:1006F00080E090E0A2E0B0E080938E1590938F159B
:10070000A0939015B093911561E084EE91E00E9462
:10071000729D882309F184E090E090938D15809379
:100720008C150E94FA4D81110AC080918C15909110
:100730008D15880F991F90938D1580938C1580913E
:100740008C1590918D1509975CF088E090E090935E
:100750008D1580938C1504C010928D1510928C15F8
:1007600081E08093570D8093580D00918016109171
:100770008116209182163091831600934F0D1093AD
:10078000500D2093510D3093520D0091A9161091E8
:10079000AA162091AB163091AC160093530D10930E
:1007A000540D2093550D3093560D8FE08093141700
:1007B0000091FF162B2D3A2DA601B7018D2F9C2FEE
:1007C0000E94E36BDF91CF911F910F91FF90EF900B
:1007D000DF90CF90BF90AF909F908F907F905F9071
:1007E0004F903F902F900C94A9620E94FB50811172
:1007F0001092161780911517882361F11092151722
:100800008091E61590911517892B8093151780918B
:10081000E71590911517892B809315178091E8158E
:1008200090911517892B80931517809115178111B9
:1008300011C00E9400648091FE16882339F08091D7
:10084000FD168F5F8093FD161092FE168091B60202
:100850008093B70208950C946B618091FD16089502
:10086000CF93DF9300D000D000D0CDB7DEB740E00B
:100870006DE57AE18EE497E10E944CD043E069E6B1
:100880007AE1CE0101960E944CD041E953E0BE01CD
:100890006F5F7F4F87E197E10E947F9C47E069E6A9
:1008A0007AE1CE0101960E944CD041E953E0BE01AD
:1008B0006F5F7F4F82E297E10E947F9C43E061E699
:1008C0007AE1CE0101960E944CD041E953E0BE018D
:1008D0006F5F7F4F8DE297E10E947F9C45E063E769
:1008E0007AE1CE0101960E944CD041E953E0BE016D
:1008F0006F5F7F4F88E397E10E947F9C46E063E64D
:100900007AE1CE0101960E944CD041E953E0BE014C
:100910006F5F7F4F83E497E10E947F9C89EE96E1B1
:100920000E943C4C85ED96E10E943C4C26960FB609
:10093000F894DEBF0FBECDBFDF91CF91089594EA4A
:100940009093BC009091BC0097FFFCCF9091B900B0
:10095000987F983061F58093BB0084E88093BC0059
:100960008091BC0087FFFCCF8091B900887F8831DF
:1009700001F5CB01FB0150E064E80EC0219120930A
:10098000BB006093BC002091BC0027FFFCCF2091EE
:10099000B900287F283279F49F01281B390B2417CE
:1009A000350764F384E98093BC0080E0089581E01A
:1009B000089582E0089583E008951092B90080E2DE
:1009C0008093B800089580915B17089510925B178B
:1009D00081E080935417089581E040915917509118
:1009E0005A172091571730915817421753070CF098
:1009F00080E008958091591790915A1720915717C8
:100A000030915817821793076CF4E0915517F091C5
:100A10005617E80FF91F019690935A1780935917AC
:100A20008491089580E00895809154170895CF939C
:100A3000C82F81E080935B1710925A1710925917B4
:100A400010925417C13039F018F0C23009F516C0B1
:100A500021E230E106C00E94F733882339F020E814
:100A600030E1309356172093551716C08AEA96E165
:100A70009093561780935517C2E00EC08093541779
:100A800084ED9CE19093561780935517C3E004C002
:100A900010925B1780E00EC0EC2FF0E0EE0FFF1F0E
:100AA000ED52F24D8591949180935717909358177A
:100AB00080915B17CF91089510925B1781E080932E
:100AC0005417089540E06DE57AE18CE597E10C94C8
:100AD0004CD01092631740E251EA67E070E0FC01ED
:100AE00040A351A362A373A3E4E0F1E08081807E80
:100AF0008083E5E0F1E08081807E808308958F929D
:100B00009F92AF92BF92CF92DF92EF92FF920F939C
:100B10001F93CF93DF93CDB7DEB72F970FB6F8941F
:100B2000DEBF0FBECDBF8C01FC01818181118EC063
:100B30009090030180916317981649F080E291EA42
:100B4000A7E0B0E080A391A3A2A3B3A30CC0F801D7
:100B50008281882309F470C0C80102960E94E0D205
:100B600081116AC073C06801F2E0CF0ED11CC601CA
:100B70000E940FD391FC10C08091621781111BC09D
:100B800040E856E968E970E0C80141960E94BCD28D
:100B900081E0809362170FC0CE0101960E94B8D207
:100BA0008FE0FE013196D801519601900D928A9501
:100BB000E1F710926217780181E1E80EF11CC7019C
:100BC0000E94E0D2882391F086E0F801808381E0E2
:100BD0008183CE0101960E94B8D28FE0FE0131964A
:100BE000D70101900D928A95E1F730C0E12CF12CEC
:100BF000A92CB12C88248394C5010E2C02C0959594
:100C000087950A94E2F780FD0DC0F801818181117A
:100C100009C0E082818240A151A162A173A1C601F5
:100C20000E94BCD2FFEFEF1AFF0A85E0E816F1043C
:100C300019F7909263170AC040EA56E861E070E045
:100C4000F80140A351A362A373A38DCF2F960FB6D3
:100C5000F894DEBF0FBECDBFDF91CF911F910F91F2
:100C6000FF90EF90DF90CF90BF90AF909F908F90CC
:100C70000895FC01F89481819081118278948823F1
:100C800019F0FB01908311820895FC0140A351A348
:100C900062A373A3089540E06DE57AE184E697E1ED
:100CA0000C944CD00F931F93CF93DF9300D000D0C0
:100CB00000D0CDB7DEB78C0140E065E67AE1CE0129
:100CC00001960E944CD0CE0101960E948ED08111D7
:100CD00029C041E065E67AE1CE0101960E944CD040
:100CE00061E0CE0101960E949BD044E067E67AE184
:100CF000CE0101960E944CD0CE0101960E948ED06A
:100D0000882321F0C8010E949D860CC041E065E661
:100D10007AE1CE0101960E944CD060E0CE010196AE
:100D20000E949BD026960FB6F894DEBF0FBECDBFB3
:100D3000DF91CF911F910F9108950F931F93CF9340
:100D4000DF9300D000D000D0CDB7DEB78C0140E0FB
:100D500065E67AE1CE0101960E944CD060E0CE01BA
:100D600001960E949BD040E065E67AE1CE010196B3
:100D70000E944CD061E0CE0101960E947BD0F80128
:100D8000108244E067E67AE1CE0101960E944CD0E1
:100D9000CE0101960E948ED0882319F0C8010E94CE
:100DA000528641E065E67AE1CE0101960E944CD080
:100DB00060E0CE0101960E949BD026960FB6F89473
:100DC000DEBF0FBECDBFDF91CF911F910F91089570
:100DD0000F931F93CF93DF9300D000D000D0CDB7F7
:100DE000DEB78C0141E065E67AE1CE0101960E9412
:100DF0004CD060E0CE0101960E949BD041E065E6B8
:100E00007AE1CE0101960E944CD061E0CE010196BC
:100E10000E947BD044E067E67AE1CE0101960E9411
:100E20004CD060E0CE0101960E949BD044E067E682
:100E30007AE1CE0101960E944CD060E0CE0101968D
:100E40000E947BD0C8010E949D86F8011182128207
:100E5000138226960FB6F894DEBF0FBECDBFDF918A
:100E6000CF911F910F91089540E06DE57AE18AE6F8
:100E700097E10C944CD02F923F924F925F926F92D9
:100E80007F928F929F92AF92CF92DF92EF92FF92DA
:100E90000F931F93CF93DF93CDB7DEB72E970FB687
:100EA000F894DEBF0FBECDBF4C01D62E5E874D87B6
:100EB0002901370145E06BE67AE1CE0101960E94F7
:100EC0004CD042E06BE67AE1CE0107960E944CD00E
:100ED0009E012F5F3F4FAE01495F5F4FB801C401D4
:100EE0000E9490D287E993E0F401978B868BD08E95
:100EF0001401F9E12F0E311C8AE0E80EF11CA40167
:100F00004A5E5F4FAD2CCC24C39400E211EA27E087
:100F100030E0B401C1010E945A9F6D857E85C401F5
:100F20008D569F4F0E9463D0F401E756FF4FD08249
:100F3000A301465E5F4F9201B101C40186569F4FE7
:100F40000E94629CF401E255FF4F718260822E96EE
:100F50000FB6F894DEBF0FBECDBFDF91CF911F91CA
:100F60000F91FF90EF90DF90CF90AF909F908F9078
:100F70007F906F905F904F903F902F9008950F93C8
:100F80001F93CF93DF93EC018C010D561F4F60E050
:100F9000C8010E949BD061E0C8010E947BD0CE01B5
:100FA00049960E94669ECE010E94F8D1CE018656D7
:100FB0009F4FDF91CF911F910F910C94359CCF9350
:100FC000DF93EC0149960E9458A2CE0186569F4FAE
:100FD000DF91CF910C94F29B86569F4F61110C9438
:100FE000E69B0C94319C882321F0809180008068DE
:100FF00003C0809180008F738093800008958823C0
:1010000021F08091A000806803C08091A0008F73C0
:101010008093A00008950F931F93CF93DF9300D088
:1010200000D000D0CDB7DEB7162F0FB7F894FC0173
:101030008281811116C0862F81508E3F38F080E06A
:101040000E94FF8743E065E67AE117C070E0709385
:10105000A9006093A8008091A00080688093A00000
:1010600023C0813009F5862F81508E3F98F080E0B3
:101070000E94F38745E061E77AE1CE0101960E9484
:101080004CD061E01F3F09F060E0CE0101960E9464
:101090009BD00AC070E070938900609388008091B3
:1010A00080008068809380000FBF26960FB6F8946A
:1010B000DEBF0FBECDBFDF91CF911F910F9108957D
:1010C00040E06DE57AE180E797E10C944CD0CF9356
:1010D000DF9300D000D0CDB7DEB795E09B836A8365
:1010E000811109C081E08983842F809590917717C1
:1010F00089234A7A09C0813011F583E08983842FDE
:101100008095909177178923842B8C8342E0BE01D0
:101110006D5F7F4F84EC0E949F8485E08A95F1F794
:10112000000042E0BE016F5F7F4F84EC0E949F840D
:1011300085E08A95F1F700008C81809377170F90F6
:101140000F900F900F90DF91CF910895CF93DF9381
:1011500000D0CDB7DEB795E09983262F20959091EA
:101160007717882331F0822F89236575862B8A8330
:1011700002C092239A8342E0BE016F5F7F4F84ECEE
:101180000E949F848A81809377170F900F90DF9140
:10119000CF910895CF93DF9300D000D0CDB7DEB7C5
:1011A00095E09B831C821A8219826A83811109C08F
:1011B00082E08983842F80959091771789234A7ADA
:1011C00009C0813051F484E08983842F8095909107
:1011D00077178923842B8C8308C081E0611101C0BB
:1011E00080E0642F0E94A68819C042E0BE016D5FB6
:1011F0007F4F84EC0E949F8485E08A95F1F7000080
:1012000042E0BE016F5F7F4F84EC0E949F8485E0C7
:101210008A95F1F700008C81809377170F900F90DB
:101220000F900F90DF91CF9108954FE360E083E03E
:101230000C94CA880E94158943E068EC81E00E9402
:10124000CA8843E062E881E00C946788CF92DF921D
:10125000EF92FF920F931F93CF93DF931F92CDB71F
:10126000DEB7F82E162F042F222321F099830E9437
:10127000158999814FEFF41201C093E01F3F09F4E3
:101280009C600F3F09F49063492F61E083E00E9466
:10129000CA889F2D915081E09E3F08F080E0282F62
:1012A00030E0912F91509E3F10F42F5F3F4FE02E82
:1012B000EA94EDEFEE1518F022303105A1F1882304
:1012C00089F043E06091761780E099830E946788F7
:1012D00043E06F2D80E00E94CA88CC24C394D12CB7
:1012E000998102C0C12CD12C9E3F78F4FC2C4CE09B
:1012F000609176178C2D0E946788FFEFCF1ADF0A66
:101300004CE0612F8F2D0E94CA884DEF4E1508F4D6
:1013100075C040E3609176178C2D0E94678840E38A
:10132000602F8C2D60C0EF2DF0E0202F30E0DF012A
:10133000A21BB30BB7FF03C0B195A195B109812FD3
:1013400090E0E81BF90BF7FF03C0F195E195F10977
:10135000281B390B37FF03C0319521953109AE1792
:10136000BF07BCF4A217B30754F54CE060917617A1
:1013700080E00E9467884CE0612F80E00E94CA886C
:1013800043E36091761781E00E94678843E36F2D05
:1013900029C0E217F3079CF440E36091761780E0E0
:1013A0000E94678840E3602F80E00E94CA884FE077
:1013B0006091761781E00E9467884FE012C043E099
:1013C0006091761780E00E94678843E06F2D80E08F
:1013D0000E94CA884CE36091761781E00E9467887A
:1013E0004CE3612F81E00F90DF91CF911F910F911E
:1013F000FF90EF90DF90CF900C94CA880F90DF9110
:10140000CF911F910F91FF90EF90DF90CF900895B3
:101410001F93CF93DF93C82FD62F142F0E942F3303
:1014200021E0412F6D2F8C2FDF91CF911F910C94D4
:1014300026898F929F92AF92BF92CF92DF92EF92C6
:10144000FF92CF930E94158961E080E491E00E94B1
:10145000729DC82F4FEF5FEFBA0184E491E00E94C4
:10146000B29D6B017C01C33009F450C020F4C1303F
:1014700041F1B8F50AC0C53081F058F1C63009F421
:101480004EC0C83009F069C053C04FE36091761771
:1014900081E00E9467884FE307C040E360917617C0
:1014A00081E00E94678840E364E681E0CF91FF908D
:1014B000EF90DF90CF90BF90AF909F908F900C9463
:1014C000CA8843E06091761781E00E94678843E014
:1014D000EBCF4CE06091761781E00E9467884CE08A
:1014E000E3CF4CE06091761781E00E9467884CE082
:1014F00062E381E00E94CA8843E06091761780E051
:101500000E94678843E068EC80E0D0CF43E36091BD
:10151000761781E00E94678843E366E4C6CF43E321
:101520006091761781E00E94678843E368ECBDCF45
:101530008D2C9E2CAF2CBB24B7018827992721E046
:10154000482D8F2DCF91FF90EF90DF90CF90BF90DF
:10155000AF909F908F900C942689CF91FF90EF9041
:10156000DF90CF90BF90AF909F908F900895809321
:1015700076170C94198A0E94DD840C94198A40E035
:101580006DE57AE188E797E10C944CD04F925F9239
:101590006F927F92AF92BF92CF92DF92EF92FF92C3
:1015A0000F931F93CF93DF9300D0CDB7DEB75C01CD
:1015B000009709F448C06230710508F444C0DC01AA
:1015C00016964D905D906D907C901997660F771FE1
:1015D00073016201C60ED71EE11CF11CD501ED910D
:1015E000FC910190F081E02D22E030E0AE014F5FF0
:1015F0005F4FC701B6010995882329F109811A8136
:1016000001151105F1F0C80140960897E0F0083F78
:10161000BFEF1B0710F000E010E01A821982D5011D
:10162000ED91FC910480F581E02D22E030E0AE01E7
:101630004F5F5F4FC701B6010995B801011511054C
:1016400029F681E001C080E00F900F90DF91CF91EB
:101650001F910F91FF90EF90DF90CF90BF90AF90D0
:101660007F906F905F904F9008952F923F924F928E
:101670005F926F927F928F929F92AF92BF92CF9222
:10168000DF92EF92FF920F931F93CF93DF93CDB72B
:10169000DEB72C970FB6F894DEBF0FBECDBF4C015E
:1016A0007A876987009709F476C0DC01ED91FC9197
:1016B0001197208131813C872B87848195819E837E
:1016C0008D831696CD90DD90ED90FC9019975A96EB
:1016D000AD90BC905B971A968D919D910D90BC91A9
:1016E000A02DB695A7959795879598878F83D40158
:1016F0005B961C921E925A971A011C821B8200E074
:1017000010E059C0B2E0AB16B10430F0EF81F885BB
:10171000AE16BF0608F403C042E0A42EB12CC501EA
:10172000880F991F26013701480E591E611C711C34
:1017300022E030E0AE014F5F5F4FC301B201EB85A5
:10174000FC850995882339F189819A81892B51F586
:101750002114310431F4D4015B96BC92AE925A97B5
:1017600034C00115110529F4EFEFFFEFFA83E98387
:1017700002C01A83098322E030E0AE014F5F5F4F61
:10178000C301B201ED81FE810995811107C0B80145
:10179000C4010E94C68A00E010E033C0F1E02F1AB5
:1017A000310885012FEFA21AB20A4B815C814F5F8D
:1017B0005F4F5C834B838F819885AB81BC818A1797
:1017C0009B0709F09FCF232811F7E985FA85E230BE
:1017D000F105B8F009831A83CF01880F991FA7017B
:1017E0009601280F391F411D511DCA01B90122E080
:1017F00030E0AE014F5F5F4FED81FE810995882398
:1018000031F2C8012C960FB6F894DEBF0FBECDBFE3
:10181000DF91CF911F910F91FF90EF90DF90CF90CC
:10182000BF90AF909F908F907F906F905F904F9000
:101830003F902F90089580E190E008950F931F93BB
:10184000FC010097A9F06230710590F09B012250D5
:101850003109A089B1890E94B9D88B019C01828984
:101860009389A489B589080F191F2A1F3B1F03C03C
:1018700000E010E09801B801C9011F910F9108958F
:10188000FC01819191E0219180FB879587F9820F7E
:101890009F5F9B30C1F70895CF92DF92EF92FF9246
:1018A0000F931F93CF93DF93CDB7DEB761970FB63A
:1018B000F894DEBF0FBECDBF6C017901D9010D9147
:1018C0001C91119712968D919C9113978096139667
:1018D0009C938E931297F6018081853E11F08111C1
:1018E00004C0D70114961C92B3C0F60183858F30D3
:1018F000B9F5D90114968C91882319F0958589172B
:1019000089F08BE2F80111928A95E9F7D6011D96CC
:101910008C91F7018483D80197964D935D936D93D5
:101920007C939A97F60120812F7330E02150310982
:101930004DE0429FC001439F900D1124E4EDF2E081
:10194000DE01119601900D924A95E1F7FE01319664
:101950009E01225F3F4F8F31910508F47BC078C014
:10196000D8018C91882309F485C0C6014E875F8712
:10197000688B798B0E94408CF70194814E855F853E
:1019800068897989981376C048C09C919032A1F0FB
:10199000FA019083F601248523FF08C02C9121349D
:1019A00028F02B3518F4905EFA0190838F5F119622
:1019B0004F5F5F4F883049F7D8019C91953011F403
:1019C00095EE9C93F6019085903219F1F801E80F9D
:1019D000F11D9EE29083F6013896382F3C5F8F5FB1
:1019E00090819032B1F0A801480F511DDA019C930B
:1019F000D6011C962C9124FF08C02081213428F0A8
:101A00002B3518F4905EDA019C938F5F3196831327
:101A1000E7CFF801E80FF11D1082F6018385D801A8
:101A200090968C939097828D938D92969C938E93A3
:101A30009197848D958DA68DB78DF80183A394A37E
:101A4000A5A3B6A381E0D70115968C9380E022C0B0
:101A500081E020C041917801E80EF91EB601640FC3
:101A6000711DDB014C91D7014C930196E217F307EE
:101A700079F371CF8BE2F80111928A95E9F7D801D9
:101A800097964D935D936D937C939A97D601A80199
:101A900080E07BCF61960FB6F894DEBF0FBECDBF5E
:101AA000DF91CF911F910F91FF90EF90DF90CF903A
:101AB00008953F924F925F926F927F928F929F9282
:101AC000AF92BF92CF92DF92EF92FF920F931F934C
:101AD000CF93DF93CDB7DEB7A0970FB6F894DEBFF4
:101AE0000FBECDBF8B01009711F480E00CC16115D2
:101AF0007105D9F3DC01ED91FC9184809580FB01A7
:101B0000C7A0D0A4E1A4F2A4B62EA12EFB0101909F
:101B10000020E9F73197E61BF70B6E2ECF019927CE
:101B20000C966DE070E00E9461D8762E4BE050E09C
:101B300060E270E0CE0101960E9489DA6EE270E008
:101B4000C8010E94C8DA009729F0DC0111962C9197
:101B50002111C0C0B8E0B61598F0462D50E06B2DAD
:101B60007A2DCE0101960E9480DAF80180818E32B2
:101B700059F581818E3209F48281882321F124C0B4
:101B800088E0EB2DFA2DDE01119601900D928A95D9
:101B9000E1F7D80191968D919C9192979C01332702
:101BA000A4E035952795AA95E1F7803A10F4205DD9
:101BB00001C02F592F838F708A3010F4805D01C0CF
:101BC0008F59888701C0712C8981853E11F485E089
:101BD0008983FE013C9685E1DF011D928A95E9F734
:101BE000F80180A18C8781A192A19C8F8B8F83A10A
:101BF00094A1A5A1B6A18D8F9E8FAF8FB8A3F0E25F
:101C00007F9EC0011124A7019601280F391F411D95
